Component: ARM Compiler 5.06 update 7 (build 960) Tool: armlink [4d3601]

==============================================================================

Section Cross References

    bios.o(i.ADC1_Init) refers to stm32f10x_rcc.o(i.RCC_APB2PeriphClockCmd) for RCC_APB2PeriphClockCmd
    bios.o(i.ADC1_Init) refers to stm32f10x_adc.o(i.ADC_StructInit) for ADC_StructInit
    bios.o(i.ADC1_Init) refers to stm32f10x_adc.o(i.ADC_Init) for ADC_Init
    bios.o(i.ADC1_Init) refers to stm32f10x_adc.o(i.ADC_RegularChannelConfig) for ADC_RegularChannelConfig
    bios.o(i.ADC1_Init) refers to stm32f10x_adc.o(i.ADC_TempSensorVrefintCmd) for ADC_TempSensorVrefintCmd
    bios.o(i.ADC1_Init) refers to stm32f10x_adc.o(i.ADC_Cmd) for ADC_Cmd
    bios.o(i.ADC1_Init) refers to stm32f10x_adc.o(i.ADC_ResetCalibration) for ADC_ResetCalibration
    bios.o(i.ADC1_Init) refers to stm32f10x_adc.o(i.ADC_GetResetCalibrationStatus) for ADC_GetResetCalibrationStatus
    bios.o(i.ADC1_Init) refers to stm32f10x_adc.o(i.ADC_StartCalibration) for ADC_StartCalibration
    bios.o(i.ADC1_Init) refers to stm32f10x_adc.o(i.ADC_GetCalibrationStatus) for ADC_GetCalibrationStatus
    bios.o(i.GPIO_InPutset) refers to stm32f10x_rcc.o(i.RCC_APB2PeriphClockCmd) for RCC_APB2PeriphClockCmd
    bios.o(i.GPIO_InPutset) refers to stm32f10x_gpio.o(i.GPIO_Init) for GPIO_Init
    bios.o(i.InstrumentTypeRead) refers to stm32f10x_gpio.o(i.GPIO_ReadInputDataBit) for GPIO_ReadInputDataBit
    bios.o(i.Read_Internal_Temperature) refers to stm32f10x_adc.o(i.ADC_SoftwareStartConvCmd) for ADC_SoftwareStartConvCmd
    bios.o(i.Read_Internal_Temperature) refers to stm32f10x_adc.o(i.ADC_GetFlagStatus) for ADC_GetFlagStatus
    bios.o(i.Read_Internal_Temperature) refers to stm32f10x_adc.o(i.ADC_GetConversionValue) for ADC_GetConversionValue
    bios.o(i.SafeCheck) refers to stm32f10x_gpio.o(i.GPIO_ReadInputDataBit) for GPIO_ReadInputDataBit
    i2c.o(i.I2C2_ACK) refers to stm32f10x_gpio.o(i.GPIO_ResetBits) for GPIO_ResetBits
    i2c.o(i.I2C2_ACK) refers to delay.o(i.delay_us) for delay_us
    i2c.o(i.I2C2_ACK) refers to stm32f10x_gpio.o(i.GPIO_SetBits) for GPIO_SetBits
    i2c.o(i.I2C2_Init) refers to stm32f10x_rcc.o(i.RCC_APB2PeriphClockCmd) for RCC_APB2PeriphClockCmd
    i2c.o(i.I2C2_Init) refers to stm32f10x_gpio.o(i.GPIO_Init) for GPIO_Init
    i2c.o(i.I2C2_Init) refers to stm32f10x_gpio.o(i.GPIO_SetBits) for GPIO_SetBits
    i2c.o(i.I2C2_NACK) refers to stm32f10x_gpio.o(i.GPIO_ResetBits) for GPIO_ResetBits
    i2c.o(i.I2C2_NACK) refers to stm32f10x_gpio.o(i.GPIO_SetBits) for GPIO_SetBits
    i2c.o(i.I2C2_NACK) refers to delay.o(i.delay_us) for delay_us
    i2c.o(i.I2C2_ReadByte) refers to stm32f10x_gpio.o(i.GPIO_SetBits) for GPIO_SetBits
    i2c.o(i.I2C2_ReadByte) refers to stm32f10x_gpio.o(i.GPIO_ResetBits) for GPIO_ResetBits
    i2c.o(i.I2C2_ReadByte) refers to delay.o(i.delay_us) for delay_us
    i2c.o(i.I2C2_ReadByte) refers to stm32f10x_gpio.o(i.GPIO_ReadInputDataBit) for GPIO_ReadInputDataBit
    i2c.o(i.I2C2_ReadByte) refers to i2c.o(i.I2C2_NACK) for I2C2_NACK
    i2c.o(i.I2C2_ReadByte) refers to i2c.o(i.I2C2_ACK) for I2C2_ACK
    i2c.o(i.I2C2_SendByte) refers to stm32f10x_gpio.o(i.GPIO_ResetBits) for GPIO_ResetBits
    i2c.o(i.I2C2_SendByte) refers to delay.o(i.delay_us) for delay_us
    i2c.o(i.I2C2_SendByte) refers to stm32f10x_gpio.o(i.GPIO_SetBits) for GPIO_SetBits
    i2c.o(i.I2C2_Start) refers to stm32f10x_gpio.o(i.GPIO_SetBits) for GPIO_SetBits
    i2c.o(i.I2C2_Start) refers to delay.o(i.delay_us) for delay_us
    i2c.o(i.I2C2_Start) refers to stm32f10x_gpio.o(i.GPIO_ResetBits) for GPIO_ResetBits
    i2c.o(i.I2C2_Stop) refers to stm32f10x_gpio.o(i.GPIO_ResetBits) for GPIO_ResetBits
    i2c.o(i.I2C2_Stop) refers to delay.o(i.delay_us) for delay_us
    i2c.o(i.I2C2_Stop) refers to stm32f10x_gpio.o(i.GPIO_SetBits) for GPIO_SetBits
    i2c.o(i.I2C2_Wait_ACK) refers to stm32f10x_gpio.o(i.GPIO_SetBits) for GPIO_SetBits
    i2c.o(i.I2C2_Wait_ACK) refers to delay.o(i.delay_us) for delay_us
    i2c.o(i.I2C2_Wait_ACK) refers to i2c.o(i.I2C2_Stop) for I2C2_Stop
    i2c.o(i.I2C2_Wait_ACK) refers to stm32f10x_gpio.o(i.GPIO_ReadInputDataBit) for GPIO_ReadInputDataBit
    i2c.o(i.I2C2_Wait_ACK) refers to stm32f10x_gpio.o(i.GPIO_ResetBits) for GPIO_ResetBits
    i2c.o(i.I2C_ACK) refers to stm32f10x_gpio.o(i.GPIO_ResetBits) for GPIO_ResetBits
    i2c.o(i.I2C_ACK) refers to delay.o(i.delay_us) for delay_us
    i2c.o(i.I2C_ACK) refers to stm32f10x_gpio.o(i.GPIO_SetBits) for GPIO_SetBits
    i2c.o(i.I2C_Init) refers to stm32f10x_rcc.o(i.RCC_APB2PeriphClockCmd) for RCC_APB2PeriphClockCmd
    i2c.o(i.I2C_Init) refers to stm32f10x_gpio.o(i.GPIO_Init) for GPIO_Init
    i2c.o(i.I2C_Init) refers to stm32f10x_gpio.o(i.GPIO_SetBits) for GPIO_SetBits
    i2c.o(i.I2C_NACK) refers to stm32f10x_gpio.o(i.GPIO_ResetBits) for GPIO_ResetBits
    i2c.o(i.I2C_NACK) refers to stm32f10x_gpio.o(i.GPIO_SetBits) for GPIO_SetBits
    i2c.o(i.I2C_NACK) refers to delay.o(i.delay_us) for delay_us
    i2c.o(i.I2C_ReadByte) refers to stm32f10x_gpio.o(i.GPIO_SetBits) for GPIO_SetBits
    i2c.o(i.I2C_ReadByte) refers to delay.o(i.delay_us) for delay_us
    i2c.o(i.I2C_ReadByte) refers to stm32f10x_gpio.o(i.GPIO_ResetBits) for GPIO_ResetBits
    i2c.o(i.I2C_ReadByte) refers to stm32f10x_gpio.o(i.GPIO_ReadInputDataBit) for GPIO_ReadInputDataBit
    i2c.o(i.I2C_ReadByte) refers to i2c.o(i.I2C_NACK) for I2C_NACK
    i2c.o(i.I2C_ReadByte) refers to i2c.o(i.I2C_ACK) for I2C_ACK
    i2c.o(i.I2C_SendByte) refers to stm32f10x_gpio.o(i.GPIO_ResetBits) for GPIO_ResetBits
    i2c.o(i.I2C_SendByte) refers to delay.o(i.delay_us) for delay_us
    i2c.o(i.I2C_SendByte) refers to stm32f10x_gpio.o(i.GPIO_SetBits) for GPIO_SetBits
    i2c.o(i.I2C_Start) refers to stm32f10x_gpio.o(i.GPIO_SetBits) for GPIO_SetBits
    i2c.o(i.I2C_Start) refers to delay.o(i.delay_us) for delay_us
    i2c.o(i.I2C_Start) refers to stm32f10x_gpio.o(i.GPIO_ResetBits) for GPIO_ResetBits
    i2c.o(i.I2C_Stop) refers to stm32f10x_gpio.o(i.GPIO_ResetBits) for GPIO_ResetBits
    i2c.o(i.I2C_Stop) refers to delay.o(i.delay_us) for delay_us
    i2c.o(i.I2C_Stop) refers to stm32f10x_gpio.o(i.GPIO_SetBits) for GPIO_SetBits
    i2c.o(i.I2C_Wait_ACK) refers to stm32f10x_gpio.o(i.GPIO_SetBits) for GPIO_SetBits
    i2c.o(i.I2C_Wait_ACK) refers to delay.o(i.delay_us) for delay_us
    i2c.o(i.I2C_Wait_ACK) refers to i2c.o(i.I2C_Stop) for I2C_Stop
    i2c.o(i.I2C_Wait_ACK) refers to stm32f10x_gpio.o(i.GPIO_ReadInputDataBit) for GPIO_ReadInputDataBit
    i2c.o(i.I2C_Wait_ACK) refers to stm32f10x_gpio.o(i.GPIO_ResetBits) for GPIO_ResetBits
    i2c.o(i.WS100T10_Ctrl) refers to delay.o(i.delay_us) for delay_us
    i2c.o(i.WS100T10_Init) refers to stm32f10x_rcc.o(i.RCC_APB2PeriphClockCmd) for RCC_APB2PeriphClockCmd
    i2c.o(i.WS100T10_Init) refers to stm32f10x_gpio.o(i.GPIO_ResetBits) for GPIO_ResetBits
    i2c.o(i.WS100T10_Init) refers to stm32f10x_gpio.o(i.GPIO_Init) for GPIO_Init
    spi.o(i.SPI1_Configuration) refers to stm32f10x_rcc.o(i.RCC_APB2PeriphClockCmd) for RCC_APB2PeriphClockCmd
    spi.o(i.SPI1_Configuration) refers to stm32f10x_gpio.o(i.GPIO_Init) for GPIO_Init
    spi.o(i.SPI1_Configuration) refers to stm32f10x_spi.o(i.SPI_Init) for SPI_Init
    spi.o(i.SPI1_Configuration) refers to stm32f10x_spi.o(i.SPI_Cmd) for SPI_Cmd
    spi.o(i.SPI1_ReadWrite) refers to stm32f10x_spi.o(i.SPI_I2S_GetFlagStatus) for SPI_I2S_GetFlagStatus
    spi.o(i.SPI1_ReadWrite) refers to stm32f10x_spi.o(i.SPI_I2S_SendData) for SPI_I2S_SendData
    spi.o(i.SPI1_ReadWrite) refers to stm32f10x_spi.o(i.SPI_I2S_ReceiveData) for SPI_I2S_ReceiveData
    spi.o(i.SPI2_Configuration) refers to spi.o(i.bus_SPIxPortInit) for bus_SPIxPortInit
    spi.o(i.SPI2_ReadWrite) refers to spi.o(i.bus_SPIxShift) for bus_SPIxShift
    spi.o(i.bus_SPIxShift) refers to delay.o(i.delay_us) for delay_us
    spi.o(i.bus_SPIxShift1) refers to delay.o(i.delay_us) for delay_us
    usart.o(i.BIOS_USART2_Init) refers to system_stm32f10x.o(.data) for SystemCoreClock
    usart.o(i.BIOS_USART3_Init) refers to stm32f10x_usart.o(i.USART_ITConfig) for USART_ITConfig
    usart.o(i.BIOS_USART3_Init) refers to system_stm32f10x.o(.data) for SystemCoreClock
    usart.o(i.USART2Print) refers to usart.o(i.USART2_Send) for USART2_Send
    usart.o(i.USART2Print) refers to delay.o(i.delay_us) for delay_us
    fm24.o(i.FM24Init) refers to i2c.o(i.I2C2_Init) for I2C2_Init
    fm24.o(i.FM24_Read) refers to i2c.o(i.I2C2_Start) for I2C2_Start
    fm24.o(i.FM24_Read) refers to i2c.o(i.I2C2_SendByte) for I2C2_SendByte
    fm24.o(i.FM24_Read) refers to i2c.o(i.I2C2_Wait_ACK) for I2C2_Wait_ACK
    fm24.o(i.FM24_Read) refers to i2c.o(i.I2C2_ReadByte) for I2C2_ReadByte
    fm24.o(i.FM24_Read) refers to i2c.o(i.I2C2_Stop) for I2C2_Stop
    fm24.o(i.FM24_Write) refers to i2c.o(i.I2C2_Start) for I2C2_Start
    fm24.o(i.FM24_Write) refers to i2c.o(i.I2C2_SendByte) for I2C2_SendByte
    fm24.o(i.FM24_Write) refers to i2c.o(i.I2C2_Wait_ACK) for I2C2_Wait_ACK
    fm24.o(i.FM24_Write) refers to i2c.o(i.I2C2_Stop) for I2C2_Stop
    cs5552.o(i.GET_ADC_CH0) refers to rt_cmsis.o(i.osDelay) for osDelay
    cs5552.o(i.GET_ADC_CH0) refers to delay.o(i.delay_us) for delay_us
    cs5552.o(i.GET_ADC_CH0) refers to cs5552.o(i.Read_Register) for Read_Register
    cs5552.o(i.GET_ADC_CH0) refers to fflt_clz.o(x$fpl$fflt) for __aeabi_i2f
    cs5552.o(i.GET_ADC_CH0) refers to cs5552.o(i.bubbleSort) for bubbleSort
    cs5552.o(i.GET_ADC_CH0) refers to faddsub_clz.o(x$fpl$fadd) for __aeabi_fadd
    cs5552.o(i.GET_ADC_CH0) refers to f2d.o(x$fpl$f2d) for __aeabi_f2d
    cs5552.o(i.GET_ADC_CH0) refers to ddiv.o(x$fpl$ddiv) for __aeabi_ddiv
    cs5552.o(i.GET_ADC_CH0) refers to d2f.o(x$fpl$d2f) for __aeabi_d2f
    cs5552.o(i.GET_ADC_CH0) refers to ffix.o(x$fpl$ffix) for __aeabi_f2iz
    cs5552.o(i.GET_ADC_CH0) refers to dflt_clz.o(x$fpl$dflt) for __aeabi_i2d
    cs5552.o(i.GET_ADC_CH0) refers to dmul.o(x$fpl$dmul) for __aeabi_dmul
    cs5552.o(i.GET_ADC_CH0) refers to cs5552.o(.data) for ADvalue
    cs5552.o(i.GET_ADC_CH0) refers to cs5552.o(.bss) for bufferdata
    cs5552.o(i.INIT_CS555X) refers to spi.o(i.SPI2_Configuration) for SPI2_Configuration
    cs5552.o(i.INIT_CS555X) refers to rt_cmsis.o(i.osDelay) for osDelay
    cs5552.o(i.INIT_CS555X) refers to cs5552.o(i.RESET_SPI) for RESET_SPI
    cs5552.o(i.INIT_CS555X) refers to cs5552.o(i.Write_Register) for Write_Register
    cs5552.o(i.INIT_CS555X) refers to spi.o(i.SPI2_ReadWrite) for SPI2_ReadWrite
    cs5552.o(i.INIT_CS555X) refers to rt_cmsis.o(i.osThreadCreate) for osThreadCreate
    cs5552.o(i.INIT_CS555X) refers to cs5552.o(.bss) for CalibrateWeight
    cs5552.o(i.INIT_CS555X) refers to cs5552.o(.constdata) for os_thread_def_GET_ADC_CH0
    cs5552.o(i.RESET_SPI) refers to spi.o(i.SPI2_ReadWrite) for SPI2_ReadWrite
    cs5552.o(i.Read_Register) refers to spi.o(i.SPI2_ReadWrite) for SPI2_ReadWrite
    cs5552.o(i.Read_Register) refers to delay.o(i.delay_us) for delay_us
    cs5552.o(i.WaitForReady) refers to delay.o(i.delay_us) for delay_us
    cs5552.o(i.WaitForReady) refers to stm32f10x_gpio.o(i.GPIO_ReadInputDataBit) for GPIO_ReadInputDataBit
    cs5552.o(i.Write_Register) refers to spi.o(i.SPI2_ReadWrite) for SPI2_ReadWrite
    cs5552.o(i.bubbleSort) refers to frleqf.o(x$fpl$frleqf) for __aeabi_cfrcmple
    cs5552.o(.constdata) refers to cs5552.o(i.GET_ADC_CH0) for GET_ADC_CH0
    ad7190.o(i.AD7190_Init) refers to spi.o(i.SPI1_Configuration) for SPI1_Configuration
    ad7190.o(i.AD7190_Init) refers to spi.o(i.SPI1_ReadWrite) for SPI1_ReadWrite
    ad7190.o(i.AD7190_Init) refers to rt_cmsis.o(i.osDelay) for osDelay
    ad7190.o(i.AD7190_Init) refers to ad7190.o(i.AD7190_ReadRegisterOnce) for AD7190_ReadRegisterOnce
    ad7190.o(i.AD7190_Init) refers to ad7190.o(i.AD7190_WriteRegisterOnce) for AD7190_WriteRegisterOnce
    ad7190.o(i.AD7190_Init) refers to ad7190.o(i.AD7190_WriteRegister) for AD7190_WriteRegister
    ad7190.o(i.AD7190_Init) refers to ad7190.o(i.AD7190_ReadRegister) for AD7190_ReadRegister
    ad7190.o(i.AD7190_Init) refers to ad7190.o(i.AD7190_WaitForReady) for AD7190_WaitForReady
    ad7190.o(i.AD7190_Init) refers to rt_cmsis.o(i.osThreadCreate) for osThreadCreate
    ad7190.o(i.AD7190_Init) refers to ad7190.o(.bss) for CalibrateWeight2
    ad7190.o(i.AD7190_Init) refers to ad7190.o(.constdata) for os_thread_def_AD7190_Run
    ad7190.o(i.AD7190_ReadData) refers to ad7190.o(i.AD7190_WaitForReady) for AD7190_WaitForReady
    ad7190.o(i.AD7190_ReadData) refers to ad7190.o(i.AD7190_ReadRegister) for AD7190_ReadRegister
    ad7190.o(i.AD7190_ReadData) refers to spi.o(i.SPI1_Configuration) for SPI1_Configuration
    ad7190.o(i.AD7190_ReadData) refers to spi.o(i.SPI1_ReadWrite) for SPI1_ReadWrite
    ad7190.o(i.AD7190_ReadData) refers to rt_cmsis.o(i.osDelay) for osDelay
    ad7190.o(i.AD7190_ReadData) refers to ad7190.o(i.AD7190_ReadRegisterOnce) for AD7190_ReadRegisterOnce
    ad7190.o(i.AD7190_ReadData) refers to ad7190.o(i.AD7190_WriteRegisterOnce) for AD7190_WriteRegisterOnce
    ad7190.o(i.AD7190_ReadData) refers to ad7190.o(i.AD7190_WriteRegister) for AD7190_WriteRegister
    ad7190.o(i.AD7190_ReadData) refers to ad7190.o(.data) for ErrCount
    ad7190.o(i.AD7190_ReadRegister) refers to spi.o(i.SPI1_ReadWrite) for SPI1_ReadWrite
    ad7190.o(i.AD7190_ReadRegisterOnce) refers to spi.o(i.SPI1_ReadWrite) for SPI1_ReadWrite
    ad7190.o(i.AD7190_Run) refers to rt_cmsis.o(i.osDelay) for osDelay
    ad7190.o(i.AD7190_Run) refers to ad7190.o(i.AD7190_ReadData) for AD7190_ReadData
    ad7190.o(i.AD7190_Run) refers to fflt_clz.o(x$fpl$fflt) for __aeabi_i2f
    ad7190.o(i.AD7190_Run) refers to ffix.o(x$fpl$ffix) for __aeabi_f2iz
    ad7190.o(i.AD7190_Run) refers to ad7190.o(i.kalman_filter_init2) for kalman_filter_init2
    ad7190.o(i.AD7190_Run) refers to ad7190.o(i.kalman_filter_update2) for kalman_filter_update2
    ad7190.o(i.AD7190_Run) refers to dflt_clz.o(x$fpl$dflt) for __aeabi_i2d
    ad7190.o(i.AD7190_Run) refers to dmul.o(x$fpl$dmul) for __aeabi_dmul
    ad7190.o(i.AD7190_Run) refers to d2f.o(x$fpl$d2f) for __aeabi_d2f
    ad7190.o(i.AD7190_Run) refers to f2d.o(x$fpl$f2d) for __aeabi_f2d
    ad7190.o(i.AD7190_Run) refers to faddsub_clz.o(x$fpl$fsub) for __aeabi_fsub
    ad7190.o(i.AD7190_Run) refers to dleqf.o(x$fpl$dleqf) for __aeabi_cdcmple
    ad7190.o(i.AD7190_Run) refers to fmul.o(x$fpl$fmul) for __aeabi_fmul
    ad7190.o(i.AD7190_Run) refers to fflt_clz.o(x$fpl$ffltu) for __aeabi_ui2f
    ad7190.o(i.AD7190_Run) refers to frleqf.o(x$fpl$frleqf) for __aeabi_cfrcmple
    ad7190.o(i.AD7190_Run) refers to faddsub_clz.o(x$fpl$frsb) for __aeabi_frsub
    ad7190.o(i.AD7190_Run) refers to faddsub_clz.o(x$fpl$fadd) for __aeabi_fadd
    ad7190.o(i.AD7190_Run) refers to ad7190.o(.data) for ADvalue2
    ad7190.o(i.AD7190_Run) refers to ad7190.o(.bss) for kf2
    ad7190.o(i.AD7190_Run) refers to hmi.o(.bss) for Set
    ad7190.o(i.AD7190_Run) refers to drleqf.o(x$fpl$drleqf) for __aeabi_cdrcmple
    ad7190.o(i.AD7190_Run) refers to fdiv.o(x$fpl$fdiv) for __aeabi_fdiv
    ad7190.o(i.AD7190_WaitForReady) refers to delay.o(i.delay_us) for delay_us
    ad7190.o(i.AD7190_WaitForReady) refers to stm32f10x_gpio.o(i.GPIO_ReadInputDataBit) for GPIO_ReadInputDataBit
    ad7190.o(i.AD7190_WriteRegister) refers to spi.o(i.SPI1_ReadWrite) for SPI1_ReadWrite
    ad7190.o(i.AD7190_WriteRegisterOnce) refers to spi.o(i.SPI1_ReadWrite) for SPI1_ReadWrite
    ad7190.o(i.kalman_filter_update2) refers to faddsub_clz.o(x$fpl$fadd) for __aeabi_fadd
    ad7190.o(i.kalman_filter_update2) refers to fdiv.o(x$fpl$fdiv) for __aeabi_fdiv
    ad7190.o(i.kalman_filter_update2) refers to faddsub_clz.o(x$fpl$fsub) for __aeabi_fsub
    ad7190.o(i.kalman_filter_update2) refers to fmul.o(x$fpl$fmul) for __aeabi_fmul
    ad7190.o(.constdata) refers to ad7190.o(i.AD7190_Run) for AD7190_Run
    ws100t10.o(i.ACCMD) refers to stm32f10x_gpio.o(i.GPIO_ResetBits) for GPIO_ResetBits
    ws100t10.o(i.ACCMD) refers to stm32f10x_gpio.o(i.GPIO_SetBits) for GPIO_SetBits
    ws100t10.o(i.ACCtrl) refers to fflt_clz.o(x$fpl$ffltu) for __aeabi_ui2f
    ws100t10.o(i.ACCtrl) refers to fmul.o(x$fpl$fmul) for __aeabi_fmul
    ws100t10.o(i.ACCtrl) refers to ffixu.o(x$fpl$ffixu) for __aeabi_f2uiz
    ws100t10.o(i.ACCtrl) refers to i2c.o(i.WS100T10_Ctrl) for WS100T10_Ctrl
    ws100t10.o(i.AC_CTRL_Init) refers to rt_cmsis.o(i.osThreadCreate) for osThreadCreate
    ws100t10.o(i.AC_CTRL_Init) refers to ws100t10.o(.constdata) for os_thread_def__task_ACCtrl
    ws100t10.o(i.HeatPID_Task) refers to fflt_clz.o(x$fpl$ffltu) for __aeabi_ui2f
    ws100t10.o(i.HeatPID_Task) refers to rt_cmsis.o(i.osDelay) for osDelay
    ws100t10.o(i.HeatPID_Task) refers to ws100t10.o(i.ACCMD) for ACCMD
    ws100t10.o(i.HeatPID_Task) refers to rt_cmsis.o(i.osKernelSysTick) for osKernelSysTick
    ws100t10.o(i.HeatPID_Task) refers to faddsub_clz.o(x$fpl$fsub) for __aeabi_fsub
    ws100t10.o(i.HeatPID_Task) refers to frleqf.o(x$fpl$frleqf) for __aeabi_cfrcmple
    ws100t10.o(i.HeatPID_Task) refers to fmul.o(x$fpl$fmul) for __aeabi_fmul
    ws100t10.o(i.HeatPID_Task) refers to ffixu.o(x$fpl$ffixu) for __aeabi_f2uiz
    ws100t10.o(i.HeatPID_Task) refers to faddsub_clz.o(x$fpl$fadd) for __aeabi_fadd
    ws100t10.o(i.HeatPID_Task) refers to fleqf.o(x$fpl$fleqf) for __aeabi_cfcmple
    ws100t10.o(i.HeatPID_Task) refers to hmi.o(.bss) for Set
    ws100t10.o(i.HeatPID_Task) refers to ws100t10.o(.data) for Kp
    ws100t10.o(i.HeatPID_Task) refers to rtx_conf_cm.o(.constdata) for os_tickus_i
    ws100t10.o(i.HeatPID_Task) refers to max6675.o(.data) for Temperature
    ws100t10.o(i.HeatTask_Init) refers to rt_cmsis.o(i.osThreadCreate) for osThreadCreate
    ws100t10.o(i.HeatTask_Init) refers to ws100t10.o(.constdata) for os_thread_def_HeatTask_Socket
    ws100t10.o(i.HeatTask_Socket) refers to ws100t10.o(i.HeatPID_Task) for HeatPID_Task
    ws100t10.o(i.HeatTask_Socket) refers to rt_cmsis.o(i.osThreadGetId) for osThreadGetId
    ws100t10.o(i.HeatTask_Socket) refers to rt_cmsis.o(i.osThreadTerminate) for osThreadTerminate
    ws100t10.o(i.Pump_GetOutput) refers to ws100t10.o(.data) for HeatOp_State
    ws100t10.o(i.Pump_OutCmd) refers to ws100t10.o(i.HeatTask_Init) for HeatTask_Init
    ws100t10.o(i.Pump_OutCmd) refers to ws100t10.o(.data) for HeatOp_State
    ws100t10.o(i._task_ACCtrl) refers to i2c.o(i.WS100T10_Init) for WS100T10_Init
    ws100t10.o(i._task_ACCtrl) refers to ws100t10.o(i.ACCtrl) for ACCtrl
    ws100t10.o(i._task_ACCtrl) refers to rt_cmsis.o(i.osDelay) for osDelay
    ws100t10.o(i._task_ACCtrl) refers to ws100t10.o(.data) for Percent
    ws100t10.o(.constdata) refers to ws100t10.o(i._task_ACCtrl) for _task_ACCtrl
    ws100t10.o(.constdata) refers to ws100t10.o(i.HeatTask_Socket) for HeatTask_Socket
    max6675.o(i.MAX6675_ConvertTemperature) refers to max6675.o(i.kalman_filter_init) for kalman_filter_init
    max6675.o(i.MAX6675_ConvertTemperature) refers to rt_cmsis.o(i.osDelay) for osDelay
    max6675.o(i.MAX6675_ConvertTemperature) refers to max6675.o(i.MAX6675_ReadData) for MAX6675_ReadData
    max6675.o(i.MAX6675_ConvertTemperature) refers to fflt_clz.o(x$fpl$ffltu) for __aeabi_ui2f
    max6675.o(i.MAX6675_ConvertTemperature) refers to fmul.o(x$fpl$fmul) for __aeabi_fmul
    max6675.o(i.MAX6675_ConvertTemperature) refers to fflt_clz.o(x$fpl$fflt) for __aeabi_i2f
    max6675.o(i.MAX6675_ConvertTemperature) refers to max6675.o(i.kalman_filter_update) for kalman_filter_update
    max6675.o(i.MAX6675_ConvertTemperature) refers to faddsub_clz.o(x$fpl$fadd) for __aeabi_fadd
    max6675.o(i.MAX6675_ConvertTemperature) refers to max6675.o(.bss) for kf
    max6675.o(i.MAX6675_ConvertTemperature) refers to hmi.o(.bss) for Set
    max6675.o(i.MAX6675_ConvertTemperature) refers to max6675.o(.data) for Temperature
    max6675.o(i.MAX6675_Init) refers to stm32f10x_gpio.o(i.GPIO_SetBits) for GPIO_SetBits
    max6675.o(i.MAX6675_Init) refers to stm32f10x_gpio.o(i.GPIO_Init) for GPIO_Init
    max6675.o(i.MAX6675_Init) refers to rt_cmsis.o(i.osThreadCreate) for osThreadCreate
    max6675.o(i.MAX6675_Init) refers to max6675.o(.constdata) for os_thread_def_MAX6675_ConvertTemperature
    max6675.o(i.MAX6675_ReadData) refers to stm32f10x_gpio.o(i.GPIO_ResetBits) for GPIO_ResetBits
    max6675.o(i.MAX6675_ReadData) refers to delay.o(i.delay_us) for delay_us
    max6675.o(i.MAX6675_ReadData) refers to stm32f10x_gpio.o(i.GPIO_ReadInputDataBit) for GPIO_ReadInputDataBit
    max6675.o(i.MAX6675_ReadData) refers to stm32f10x_gpio.o(i.GPIO_SetBits) for GPIO_SetBits
    max6675.o(i.kalman_filter_update) refers to faddsub_clz.o(x$fpl$fadd) for __aeabi_fadd
    max6675.o(i.kalman_filter_update) refers to fdiv.o(x$fpl$fdiv) for __aeabi_fdiv
    max6675.o(i.kalman_filter_update) refers to faddsub_clz.o(x$fpl$fsub) for __aeabi_fsub
    max6675.o(i.kalman_filter_update) refers to fmul.o(x$fpl$fmul) for __aeabi_fmul
    max6675.o(.constdata) refers to max6675.o(i.MAX6675_ConvertTemperature) for MAX6675_ConvertTemperature
    usarthmi.o(i.BIOS_TIM2_TIMER_Init) refers to usarthmi.o(i.__NVIC_EnableIRQ) for __NVIC_EnableIRQ
    usarthmi.o(i.BIOS_TIM2_TIMER_Init) refers to system_stm32f10x.o(.data) for SystemCoreClock
    usarthmi.o(i.BIOS_USART1_Init) refers to stm32f10x_usart.o(i.USART_ITConfig) for USART_ITConfig
    usarthmi.o(i.BIOS_USART1_Init) refers to usarthmi.o(i.__NVIC_EnableIRQ) for __NVIC_EnableIRQ
    usarthmi.o(i.BIOS_USART1_Init) refers to rt_cmsis.o(i.osMutexCreate) for osMutexCreate
    usarthmi.o(i.BIOS_USART1_Init) refers to system_stm32f10x.o(.data) for SystemCoreClock
    usarthmi.o(i.BIOS_USART1_Init) refers to usarthmi.o(.data) for USART_Mutex_ID
    usarthmi.o(i.DataPrint) refers to rt_cmsis.o(i.osMutexWait) for osMutexWait
    usarthmi.o(i.DataPrint) refers to usarthmi.o(i.UART1_Send) for UART1_Send
    usarthmi.o(i.DataPrint) refers to delay.o(i.delay_us) for delay_us
    usarthmi.o(i.DataPrint) refers to rt_cmsis.o(i.osMutexRelease) for osMutexRelease
    usarthmi.o(i.DataPrint) refers to usarthmi.o(.data) for USART_Mutex_ID
    usarthmi.o(i.DataRec) refers to usarthmi.o(i.UART1_Received) for UART1_Received
    usarthmi.o(i.TIM2_IRQHandler) refers to rt_cmsis.o(i.osSemaphoreRelease) for osSemaphoreRelease
    usarthmi.o(i.TIM2_IRQHandler) refers to usarthmi.o(.data) for RxFlag
    usarthmi.o(i.TIM2_IRQHandler) refers to usarthmi.o(.bss) for DataInbuf
    usarthmi.o(i.UART1_Send) refers to delay.o(i.delay_us) for delay_us
    usarthmi.o(i.USART1_IRQHandler) refers to usarthmi.o(i.DataRec) for DataRec
    usarthmi.o(i.USART1_IRQHandler) refers to usarthmi.o(.bss) for DataInbuf
    usarthmi.o(i.USART1_IRQHandler) refers to usarthmi.o(.data) for RxFlag
    usarthmi.o(i.USARTHMIInit) refers to rt_cmsis.o(i.osSemaphoreCreate) for osSemaphoreCreate
    usarthmi.o(i.USARTHMIInit) refers to usarthmi.o(i.BIOS_TIM2_TIMER_Init) for BIOS_TIM2_TIMER_Init
    usarthmi.o(i.USARTHMIInit) refers to usarthmi.o(i.BIOS_USART1_Init) for BIOS_USART1_Init
    usarthmi.o(i.USARTHMIInit) refers to usarthmi.o(.constdata) for os_semaphore_def_semDataBack
    usarthmi.o(i.USARTHMIInit) refers to usarthmi.o(.data) for semDataBack
    usarthmi.o(.constdata) refers to usarthmi.o(.data) for os_semaphore_cb_semDataBack
    moisture.o(i.main) refers to stm32f10x_rcc.o(i.RCC_APB2PeriphClockCmd) for RCC_APB2PeriphClockCmd
    moisture.o(i.main) refers to stm32f10x_gpio.o(i.GPIO_PinRemapConfig) for GPIO_PinRemapConfig
    moisture.o(i.main) refers to bios.o(i.GPIO_InPutset) for GPIO_InPutset
    moisture.o(i.main) refers to ws100t10.o(i.AC_CTRL_Init) for AC_CTRL_Init
    moisture.o(i.main) refers to max6675.o(i.MAX6675_Init) for MAX6675_Init
    moisture.o(i.main) refers to fm24.o(i.FM24Init) for FM24Init
    moisture.o(i.main) refers to rt_cmsis.o(i.osDelay) for osDelay
    moisture.o(i.main) refers to ad7190.o(i.AD7190_Init) for AD7190_Init
    moisture.o(i.main) refers to ffix.o(x$fpl$ffix) for __aeabi_f2iz
    moisture.o(i.main) refers to bios.o(i.InstrumentTypeRead) for InstrumentTypeRead
    moisture.o(i.main) refers to usarthmi.o(i.USARTHMIInit) for USARTHMIInit
    moisture.o(i.main) refers to hmi.o(i.HMICMDInit) for HMICMDInit
    moisture.o(i.main) refers to ad7190.o(.data) for ADvalue2filter
    moisture.o(i.main) refers to ad7190.o(.bss) for CalibrateWeight2
    moisture.o(i.main) refers to hmi.o(.data) for MaxWeight
    hmi.o(i.DataUnpack) refers to _printf_pad.o(.text) for _printf_pre_padding
    hmi.o(i.DataUnpack) refers to _printf_percent.o(.ARM.Collect$$_printf_percent$$00000000) for _printf_percent
    hmi.o(i.DataUnpack) refers to _printf_d.o(.ARM.Collect$$_printf_percent$$00000009) for _printf_d
    hmi.o(i.DataUnpack) refers to _printf_dec.o(.text) for _printf_int_dec
    hmi.o(i.DataUnpack) refers to _printf_f.o(.ARM.Collect$$_printf_percent$$00000003) for _printf_f
    hmi.o(i.DataUnpack) refers to _printf_s.o(.ARM.Collect$$_printf_percent$$00000014) for _printf_s
    hmi.o(i.DataUnpack) refers to printf1.o(x$fpl$printf1) for _printf_fp_dec
    hmi.o(i.DataUnpack) refers to _printf_str.o(.text) for _printf_str
    hmi.o(i.DataUnpack) refers to rt_cmsis.o(i.osSemaphoreCreate) for osSemaphoreCreate
    hmi.o(i.DataUnpack) refers to rt_cmsis.o(i.osSemaphoreWait) for osSemaphoreWait
    hmi.o(i.DataUnpack) refers to noretval__2sprintf.o(.text) for __2sprintf
    hmi.o(i.DataUnpack) refers to strlen.o(.text) for strlen
    hmi.o(i.DataUnpack) refers to usarthmi.o(i.DataPrint) for DataPrint
    hmi.o(i.DataUnpack) refers to fleqf.o(x$fpl$fleqf) for __aeabi_cfcmple
    hmi.o(i.DataUnpack) refers to fflt_clz.o(x$fpl$ffltu) for __aeabi_ui2f
    hmi.o(i.DataUnpack) refers to bios.o(i.SafeCheck) for SafeCheck
    hmi.o(i.DataUnpack) refers to rt_cmsis.o(i.osDelay) for osDelay
    hmi.o(i.DataUnpack) refers to fm24.o(i.FM24_Write) for FM24_Write
    hmi.o(i.DataUnpack) refers to fflt_clz.o(x$fpl$fflt) for __aeabi_i2f
    hmi.o(i.DataUnpack) refers to faddsub_clz.o(x$fpl$fsub) for __aeabi_fsub
    hmi.o(i.DataUnpack) refers to f2d.o(x$fpl$f2d) for __aeabi_f2d
    hmi.o(i.DataUnpack) refers to drleqf.o(x$fpl$drleqf) for __aeabi_cdrcmple
    hmi.o(i.DataUnpack) refers to ffix.o(x$fpl$ffix) for __aeabi_f2iz
    hmi.o(i.DataUnpack) refers to hmi.o(.data) for semDataChange
    hmi.o(i.DataUnpack) refers to usarthmi.o(.data) for semDataBack
    hmi.o(i.DataUnpack) refers to usarthmi.o(.bss) for DataInbuf
    hmi.o(i.DataUnpack) refers to ad7190.o(.data) for weightChanging
    hmi.o(i.DataUnpack) refers to hmi.o(.ARM.__AT_0x20001000) for buf
    hmi.o(i.DataUnpack) refers to hmi.o(.bss) for startTime
    hmi.o(i.DataUnpack) refers to ad7190.o(.bss) for CalibrateWeight2
    hmi.o(i.DataUnpack) refers to usart.o(i.USART2Print) for USART2Print
    hmi.o(i.DataUnpack) refers to hmi.o(.constdata) for .constdata
    hmi.o(i.DataUnpack) refers to fdiv.o(x$fpl$fdiv) for __aeabi_fdiv
    hmi.o(i.DataUnpack) refers to max6675.o(.data) for Temperature
    hmi.o(i.DataUnpack) refers to usart.o(i.BIOS_USART2_Init) for BIOS_USART2_Init
    hmi.o(i.DataUnpack) refers to strcmpv7m.o(.text) for strcmp
    hmi.o(i.DataUnpack) refers to strcpy.o(.text) for strcpy
    hmi.o(i.DataUnpack) refers to rt_cmsis.o(i.osSemaphoreRelease) for osSemaphoreRelease
    hmi.o(i.FM24DataCRC) refers to fm24.o(i.FM24_Read) for FM24_Read
    hmi.o(i.FM24DataCRC) refers to dleqf.o(x$fpl$dleqf) for __aeabi_cdcmple
    hmi.o(i.FM24DataCRC) refers to noretval__2sprintf.o(.text) for __2sprintf
    hmi.o(i.FM24DataCRC) refers to hmi.o(.bss) for Set
    hmi.o(i.FM24DataCRC) refers to ad7190.o(.bss) for CalibrateWeight2
    hmi.o(i.HMICMDInit) refers to rt_cmsis.o(i.osThreadCreate) for osThreadCreate
    hmi.o(i.HMICMDInit) refers to hmi.o(i.MoisturingRun) for MoisturingRun
    hmi.o(i.HMICMDInit) refers to hmi.o(.constdata) for os_thread_def_DataUnpack
    hmi.o(i.Moisturing) refers to _printf_pad.o(.text) for _printf_pre_padding
    hmi.o(i.Moisturing) refers to _printf_percent.o(.ARM.Collect$$_printf_percent$$00000000) for _printf_percent
    hmi.o(i.Moisturing) refers to _printf_d.o(.ARM.Collect$$_printf_percent$$00000009) for _printf_d
    hmi.o(i.Moisturing) refers to _printf_f.o(.ARM.Collect$$_printf_percent$$00000003) for _printf_f
    hmi.o(i.Moisturing) refers to _printf_dec.o(.text) for _printf_int_dec
    hmi.o(i.Moisturing) refers to printf1.o(x$fpl$printf1) for _printf_fp_dec
    hmi.o(i.Moisturing) refers to _printf_s.o(.ARM.Collect$$_printf_percent$$00000014) for _printf_s
    hmi.o(i.Moisturing) refers to _printf_str.o(.text) for _printf_str
    hmi.o(i.Moisturing) refers to hmi.o(i.FM24DataCRC) for FM24DataCRC
    hmi.o(i.Moisturing) refers to rt_cmsis.o(i.osDelay) for osDelay
    hmi.o(i.Moisturing) refers to ffix.o(x$fpl$ffix) for __aeabi_f2iz
    hmi.o(i.Moisturing) refers to usart.o(i.BIOS_USART2_Init) for BIOS_USART2_Init
    hmi.o(i.Moisturing) refers to f2d.o(x$fpl$f2d) for __aeabi_f2d
    hmi.o(i.Moisturing) refers to noretval__2sprintf.o(.text) for __2sprintf
    hmi.o(i.Moisturing) refers to strlen.o(.text) for strlen
    hmi.o(i.Moisturing) refers to usarthmi.o(i.DataPrint) for DataPrint
    hmi.o(i.Moisturing) refers to fdiv.o(x$fpl$fdiv) for __aeabi_fdiv
    hmi.o(i.Moisturing) refers to faddsub_clz.o(x$fpl$fadd) for __aeabi_fadd
    hmi.o(i.Moisturing) refers to fflt_clz.o(x$fpl$fflt) for __aeabi_i2f
    hmi.o(i.Moisturing) refers to fmul.o(x$fpl$fmul) for __aeabi_fmul
    hmi.o(i.Moisturing) refers to fflt_clz.o(x$fpl$ffltu) for __aeabi_ui2f
    hmi.o(i.Moisturing) refers to frleqf.o(x$fpl$frleqf) for __aeabi_cfrcmple
    hmi.o(i.Moisturing) refers to rt_cmsis.o(i.osSemaphoreWait) for osSemaphoreWait
    hmi.o(i.Moisturing) refers to hmi.o(.bss) for Set
    hmi.o(i.Moisturing) refers to ad7190.o(.data) for ADvalue2filter
    hmi.o(i.Moisturing) refers to ad7190.o(.bss) for CalibrateWeight2
    hmi.o(i.Moisturing) refers to hmi.o(.data) for Resolution
    hmi.o(i.Moisturing) refers to hmi.o(.ARM.__AT_0x20001200) for buf
    hmi.o(i.Moisturing) refers to max6675.o(.data) for Temperature
    hmi.o(i.Moisturing) refers to ws100t10.o(.data) for OutputMax
    hmi.o(i.Moisturing) refers to bios.o(i.SafeCheck) for SafeCheck
    hmi.o(i.Moisturing) refers to ws100t10.o(i.Pump_OutCmd) for Pump_OutCmd
    hmi.o(i.Moisturing) refers to rt_cmsis.o(i.osKernelSysTick) for osKernelSysTick
    hmi.o(i.Moisturing) refers to faddsub_clz.o(x$fpl$fsub) for __aeabi_fsub
    hmi.o(i.Moisturing) refers to rtx_conf_cm.o(.constdata) for os_tickus_i
    hmi.o(i.Moisturing) refers to feqf.o(x$fpl$feqf) for __aeabi_cfcmpeq
    hmi.o(i.Moisturing) refers to ffixu.o(x$fpl$ffixu) for __aeabi_f2uiz
    hmi.o(i.Moisturing) refers to fleqf.o(x$fpl$fleqf) for __aeabi_cfcmple
    hmi.o(i.MoisturingRun) refers to rt_cmsis.o(i.osThreadCreate) for osThreadCreate
    hmi.o(i.MoisturingRun) refers to hmi.o(.constdata) for os_thread_def_Moisturing
    hmi.o(.constdata) refers to hmi.o(i.Moisturing) for Moisturing
    hmi.o(.constdata) refers to hmi.o(i.DataUnpack) for DataUnpack
    rtx_conf_cm.o(.emb_text) refers to rt_cmsis.o(i.osKernelInitialize) for osKernelInitialize
    rtx_conf_cm.o(.emb_text) refers to rt_cmsis.o(i.osThreadCreate) for osThreadCreate
    rtx_conf_cm.o(.emb_text) refers to rt_cmsis.o(i.osKernelStart) for osKernelStart
    rtx_conf_cm.o(.emb_text) refers to exit.o(.text) for exit
    rtx_conf_cm.o(.emb_text) refers to rtx_conf_cm.o(.constdata) for os_thread_def_main
    rtx_conf_cm.o(i.__user_perthread_libspace) refers to rt_task.o(i.rt_tsk_self) for rt_tsk_self
    rtx_conf_cm.o(i.__user_perthread_libspace) refers to rt_cmsis.o(.data) for os_running
    rtx_conf_cm.o(i.__user_perthread_libspace) refers to rtx_conf_cm.o(.bss) for .bss
    rtx_conf_cm.o(i.__user_perthread_libspace) refers to libspace.o(.bss) for __libspace_start
    rtx_conf_cm.o(i._mutex_acquire) refers to rt_cmsis.o(.data) for os_running
    rtx_conf_cm.o(i._mutex_acquire) refers to rt_mutex.o(i.rt_mut_wait) for rt_mut_wait
    rtx_conf_cm.o(i._mutex_initialize) refers to rt_mutex.o(i.rt_mut_init) for rt_mut_init
    rtx_conf_cm.o(i._mutex_initialize) refers to rtx_conf_cm.o(.data) for .data
    rtx_conf_cm.o(i._mutex_initialize) refers to rtx_conf_cm.o(.bss) for .bss
    rtx_conf_cm.o(i._mutex_release) refers to rt_cmsis.o(.data) for os_running
    rtx_conf_cm.o(i._mutex_release) refers to rt_mutex.o(i.rt_mut_release) for rt_mut_release
    rtx_conf_cm.o(.constdata) refers to rtx_conf_cm.o(.bss) for os_messageQ_q_osTimerMessageQ
    rtx_conf_cm.o(.constdata) refers to moisture.o(i.main) for main
    stm32f10x_adc.o(i.ADC_DeInit) refers to stm32f10x_rcc.o(i.RCC_APB2PeriphResetCmd) for RCC_APB2PeriphResetCmd
    stm32f10x_gpio.o(i.GPIO_AFIODeInit) refers to stm32f10x_rcc.o(i.RCC_APB2PeriphResetCmd) for RCC_APB2PeriphResetCmd
    stm32f10x_gpio.o(i.GPIO_DeInit) refers to stm32f10x_rcc.o(i.RCC_APB2PeriphResetCmd) for RCC_APB2PeriphResetCmd
    stm32f10x_rcc.o(i.RCC_GetClocksFreq) refers to stm32f10x_rcc.o(.data) for APBAHBPrescTable
    stm32f10x_rcc.o(i.RCC_WaitForHSEStartUp) refers to stm32f10x_rcc.o(i.RCC_GetFlagStatus) for RCC_GetFlagStatus
    stm32f10x_spi.o(i.I2S_Init) refers to stm32f10x_rcc.o(i.RCC_GetClocksFreq) for RCC_GetClocksFreq
    stm32f10x_spi.o(i.SPI_I2S_DeInit) refers to stm32f10x_rcc.o(i.RCC_APB2PeriphResetCmd) for RCC_APB2PeriphResetCmd
    stm32f10x_spi.o(i.SPI_I2S_DeInit) refers to stm32f10x_rcc.o(i.RCC_APB1PeriphResetCmd) for RCC_APB1PeriphResetCmd
    stm32f10x_tim.o(i.TIM_DeInit) refers to stm32f10x_rcc.o(i.RCC_APB2PeriphResetCmd) for RCC_APB2PeriphResetCmd
    stm32f10x_tim.o(i.TIM_DeInit) refers to stm32f10x_rcc.o(i.RCC_APB1PeriphResetCmd) for RCC_APB1PeriphResetCmd
    stm32f10x_tim.o(i.TIM_ETRClockMode1Config) refers to stm32f10x_tim.o(i.TIM_ETRConfig) for TIM_ETRConfig
    stm32f10x_tim.o(i.TIM_ETRClockMode2Config) refers to stm32f10x_tim.o(i.TIM_ETRConfig) for TIM_ETRConfig
    stm32f10x_tim.o(i.TIM_ICInit) refers to stm32f10x_tim.o(i.TI1_Config) for TI1_Config
    stm32f10x_tim.o(i.TIM_ICInit) refers to stm32f10x_tim.o(i.TIM_SetIC1Prescaler) for TIM_SetIC1Prescaler
    stm32f10x_tim.o(i.TIM_ICInit) refers to stm32f10x_tim.o(i.TI2_Config) for TI2_Config
    stm32f10x_tim.o(i.TIM_ICInit) refers to stm32f10x_tim.o(i.TIM_SetIC2Prescaler) for TIM_SetIC2Prescaler
    stm32f10x_tim.o(i.TIM_ICInit) refers to stm32f10x_tim.o(i.TI3_Config) for TI3_Config
    stm32f10x_tim.o(i.TIM_ICInit) refers to stm32f10x_tim.o(i.TIM_SetIC3Prescaler) for TIM_SetIC3Prescaler
    stm32f10x_tim.o(i.TIM_ICInit) refers to stm32f10x_tim.o(i.TI4_Config) for TI4_Config
    stm32f10x_tim.o(i.TIM_ICInit) refers to stm32f10x_tim.o(i.TIM_SetIC4Prescaler) for TIM_SetIC4Prescaler
    stm32f10x_tim.o(i.TIM_ITRxExternalClockConfig) refers to stm32f10x_tim.o(i.TIM_SelectInputTrigger) for TIM_SelectInputTrigger
    stm32f10x_tim.o(i.TIM_PWMIConfig) refers to stm32f10x_tim.o(i.TI1_Config) for TI1_Config
    stm32f10x_tim.o(i.TIM_PWMIConfig) refers to stm32f10x_tim.o(i.TIM_SetIC1Prescaler) for TIM_SetIC1Prescaler
    stm32f10x_tim.o(i.TIM_PWMIConfig) refers to stm32f10x_tim.o(i.TI2_Config) for TI2_Config
    stm32f10x_tim.o(i.TIM_PWMIConfig) refers to stm32f10x_tim.o(i.TIM_SetIC2Prescaler) for TIM_SetIC2Prescaler
    stm32f10x_tim.o(i.TIM_TIxExternalClockConfig) refers to stm32f10x_tim.o(i.TI2_Config) for TI2_Config
    stm32f10x_tim.o(i.TIM_TIxExternalClockConfig) refers to stm32f10x_tim.o(i.TI1_Config) for TI1_Config
    stm32f10x_tim.o(i.TIM_TIxExternalClockConfig) refers to stm32f10x_tim.o(i.TIM_SelectInputTrigger) for TIM_SelectInputTrigger
    stm32f10x_usart.o(i.USART_DeInit) refers to stm32f10x_rcc.o(i.RCC_APB2PeriphResetCmd) for RCC_APB2PeriphResetCmd
    stm32f10x_usart.o(i.USART_DeInit) refers to stm32f10x_rcc.o(i.RCC_APB1PeriphResetCmd) for RCC_APB1PeriphResetCmd
    stm32f10x_usart.o(i.USART_Init) refers to stm32f10x_rcc.o(i.RCC_GetClocksFreq) for RCC_GetClocksFreq
    startup_stm32f10x_md.o(STACK) refers (Special) to heapauxi.o(.text) for __use_two_region_memory
    startup_stm32f10x_md.o(HEAP) refers (Special) to heapauxi.o(.text) for __use_two_region_memory
    startup_stm32f10x_md.o(RESET) refers (Special) to heapauxi.o(.text) for __use_two_region_memory
    startup_stm32f10x_md.o(RESET) refers to startup_stm32f10x_md.o(STACK) for __initial_sp
    startup_stm32f10x_md.o(RESET) refers to startup_stm32f10x_md.o(.text) for Reset_Handler
    startup_stm32f10x_md.o(RESET) refers to hal_cm3.o(.emb_text) for SVC_Handler
    startup_stm32f10x_md.o(RESET) refers to usarthmi.o(i.TIM2_IRQHandler) for TIM2_IRQHandler
    startup_stm32f10x_md.o(RESET) refers to usarthmi.o(i.USART1_IRQHandler) for USART1_IRQHandler
    startup_stm32f10x_md.o(.text) refers (Special) to heapauxi.o(.text) for __use_two_region_memory
    startup_stm32f10x_md.o(.text) refers to system_stm32f10x.o(i.SystemInit) for SystemInit
    startup_stm32f10x_md.o(.text) refers to __main.o(!!!main) for __main
    startup_stm32f10x_md.o(.text) refers to startup_stm32f10x_md.o(HEAP) for Heap_Mem
    startup_stm32f10x_md.o(.text) refers to startup_stm32f10x_md.o(STACK) for Stack_Mem
    system_stm32f10x.o(i.SetSysClock) refers to system_stm32f10x.o(i.SetSysClockTo72) for SetSysClockTo72
    system_stm32f10x.o(i.SystemCoreClockUpdate) refers to system_stm32f10x.o(.data) for SystemCoreClock
    system_stm32f10x.o(i.SystemInit) refers to system_stm32f10x.o(i.SetSysClock) for SetSysClock
    rt_cmsis.o(i.isrMessageGet) refers to rt_mailbox.o(i.isr_mbx_receive) for isr_mbx_receive
    rt_cmsis.o(i.isrMessagePut) refers to rt_mailbox.o(i.rt_mbx_check) for rt_mbx_check
    rt_cmsis.o(i.isrMessagePut) refers to rt_mailbox.o(i.isr_mbx_send) for isr_mbx_send
    rt_cmsis.o(i.isrSemaphoreRelease) refers to rt_cmsis.o(i.rt_id2obj) for rt_id2obj
    rt_cmsis.o(i.isrSemaphoreRelease) refers to rt_semaphore.o(i.isr_sem_send) for isr_sem_send
    rt_cmsis.o(i.isrSignalSet) refers to rt_cmsis.o(i.rt_tid2ptcb) for rt_tid2ptcb
    rt_cmsis.o(i.isrSignalSet) refers to rt_event.o(i.isr_evt_set) for isr_evt_set
    rt_cmsis.o(i.osDelay) refers to rt_cmsis.o(i.svcDelay) for svcDelay
    rt_cmsis.o(i.osKernelInitialize) refers to rt_cmsis.o(i.svcKernelInitialize) for svcKernelInitialize
    rt_cmsis.o(i.osKernelRunning) refers to rt_cmsis.o(i.svcKernelRunning) for svcKernelRunning
    rt_cmsis.o(i.osKernelRunning) refers to rt_cmsis.o(.data) for .data
    rt_cmsis.o(i.osKernelStart) refers to rtx_conf_cm.o(.constdata) for os_flags
    rt_cmsis.o(i.osKernelStart) refers to rt_cmsis.o(i.svcKernelStart) for svcKernelStart
    rt_cmsis.o(i.osKernelSysTick) refers to rt_cmsis.o(i.svcKernelSysTick) for svcKernelSysTick
    rt_cmsis.o(i.osMailAlloc) refers to rt_cmsis.o(i.sysMailAlloc) for sysMailAlloc
    rt_cmsis.o(i.osMailCAlloc) refers to rt_cmsis.o(i.sysMailAlloc) for sysMailAlloc
    rt_cmsis.o(i.osMailCAlloc) refers to rt_cmsis.o(i.rt_clr_box) for rt_clr_box
    rt_cmsis.o(i.osMailCreate) refers to rt_cmsis.o(i.svcMailCreate) for svcMailCreate
    rt_cmsis.o(i.osMailCreate) refers to rt_cmsis.o(.data) for .data
    rt_cmsis.o(i.osMailFree) refers to rt_cmsis.o(i.sysMailFree) for sysMailFree
    rt_cmsis.o(i.osMailGet) refers to rt_cmsis.o(i.osMessageGet) for osMessageGet
    rt_cmsis.o(i.osMailPut) refers to rt_cmsis.o(i.osMessagePut) for osMessagePut
    rt_cmsis.o(i.osMessageCreate) refers to rt_cmsis.o(i.svcMessageCreate) for svcMessageCreate
    rt_cmsis.o(i.osMessageCreate) refers to rt_cmsis.o(.data) for .data
    rt_cmsis.o(i.osMessageGet) refers to rt_cmsis.o(i.isrMessageGet) for isrMessageGet
    rt_cmsis.o(i.osMessageGet) refers to rt_cmsis.o(i.svcMessageGet) for svcMessageGet
    rt_cmsis.o(i.osMessagePut) refers to rt_cmsis.o(i.isrMessagePut) for isrMessagePut
    rt_cmsis.o(i.osMessagePut) refers to rt_cmsis.o(i.svcMessagePut) for svcMessagePut
    rt_cmsis.o(i.osMutexCreate) refers to rt_cmsis.o(i.svcMutexCreate) for svcMutexCreate
    rt_cmsis.o(i.osMutexCreate) refers to rt_cmsis.o(.data) for .data
    rt_cmsis.o(i.osMutexDelete) refers to rt_cmsis.o(i.svcMutexDelete) for svcMutexDelete
    rt_cmsis.o(i.osMutexRelease) refers to rt_cmsis.o(i.svcMutexRelease) for svcMutexRelease
    rt_cmsis.o(i.osMutexWait) refers to rt_cmsis.o(i.svcMutexWait) for svcMutexWait
    rt_cmsis.o(i.osPoolAlloc) refers to rt_cmsis.o(i.sysPoolAlloc) for sysPoolAlloc
    rt_cmsis.o(i.osPoolCAlloc) refers to rt_cmsis.o(i.rt_clr_box) for rt_clr_box
    rt_cmsis.o(i.osPoolCAlloc) refers to rt_cmsis.o(i.sysPoolAlloc) for sysPoolAlloc
    rt_cmsis.o(i.osPoolCreate) refers to rt_cmsis.o(i.svcPoolCreate) for svcPoolCreate
    rt_cmsis.o(i.osPoolCreate) refers to rt_cmsis.o(.data) for .data
    rt_cmsis.o(i.osPoolFree) refers to rt_cmsis.o(i.sysPoolFree) for sysPoolFree
    rt_cmsis.o(i.osSemaphoreCreate) refers to rt_cmsis.o(i.svcSemaphoreCreate) for svcSemaphoreCreate
    rt_cmsis.o(i.osSemaphoreCreate) refers to rt_cmsis.o(.data) for .data
    rt_cmsis.o(i.osSemaphoreDelete) refers to rt_cmsis.o(i.svcSemaphoreDelete) for svcSemaphoreDelete
    rt_cmsis.o(i.osSemaphoreRelease) refers to rt_cmsis.o(i.isrSemaphoreRelease) for isrSemaphoreRelease
    rt_cmsis.o(i.osSemaphoreRelease) refers to rt_cmsis.o(i.svcSemaphoreRelease) for svcSemaphoreRelease
    rt_cmsis.o(i.osSemaphoreWait) refers to rt_cmsis.o(i.svcSemaphoreWait) for svcSemaphoreWait
    rt_cmsis.o(i.osSignalClear) refers to rt_cmsis.o(i.svcSignalClear) for svcSignalClear
    rt_cmsis.o(i.osSignalSet) refers to rt_cmsis.o(i.isrSignalSet) for isrSignalSet
    rt_cmsis.o(i.osSignalSet) refers to rt_cmsis.o(i.svcSignalSet) for svcSignalSet
    rt_cmsis.o(i.osSignalWait) refers to rt_cmsis.o(i.svcSignalWait) for svcSignalWait
    rt_cmsis.o(i.osThreadCreate) refers to rt_cmsis.o(i.svcThreadCreate) for svcThreadCreate
    rt_cmsis.o(i.osThreadCreate) refers to rt_cmsis.o(.data) for .data
    rt_cmsis.o(i.osThreadExit) refers to rt_cmsis.o(i.svcThreadGetId) for svcThreadGetId
    rt_cmsis.o(i.osThreadExit) refers to rt_cmsis.o(i.svcThreadTerminate) for svcThreadTerminate
    rt_cmsis.o(i.osThreadGetId) refers to rt_cmsis.o(i.svcThreadGetId) for svcThreadGetId
    rt_cmsis.o(i.osThreadGetPriority) refers to rt_cmsis.o(i.svcThreadGetPriority) for svcThreadGetPriority
    rt_cmsis.o(i.osThreadSetPriority) refers to rt_cmsis.o(i.svcThreadSetPriority) for svcThreadSetPriority
    rt_cmsis.o(i.osThreadTerminate) refers to rt_cmsis.o(i.svcThreadTerminate) for svcThreadTerminate
    rt_cmsis.o(i.osThreadYield) refers to rt_cmsis.o(i.svcThreadYield) for svcThreadYield
    rt_cmsis.o(i.osTimerCall) refers to rt_cmsis.o(i.svcTimerCall) for svcTimerCall
    rt_cmsis.o(i.osTimerCreate) refers to rt_cmsis.o(i.svcTimerCreate) for svcTimerCreate
    rt_cmsis.o(i.osTimerCreate) refers to rt_cmsis.o(.data) for .data
    rt_cmsis.o(i.osTimerDelete) refers to rt_cmsis.o(i.svcTimerDelete) for svcTimerDelete
    rt_cmsis.o(i.osTimerStart) refers to rt_cmsis.o(i.svcTimerStart) for svcTimerStart
    rt_cmsis.o(i.osTimerStop) refers to rt_cmsis.o(i.svcTimerStop) for svcTimerStop
    rt_cmsis.o(i.osTimerThread) refers to rt_cmsis.o(i.osMessageGet) for osMessageGet
    rt_cmsis.o(i.osTimerThread) refers to rt_cmsis.o(i.osTimerCall) for osTimerCall
    rt_cmsis.o(i.osTimerThread) refers to rtx_conf_cm.o(.data) for osMessageQId_osTimerMessageQ
    rt_cmsis.o(i.os_resume) refers to rt_system.o(i.rt_resume) for rt_resume
    rt_cmsis.o(i.os_suspend) refers to rt_system.o(i.rt_suspend) for rt_suspend
    rt_cmsis.o(i.rt_ms2tick) refers to rtx_conf_cm.o(.constdata) for os_clockrate
    rt_cmsis.o(i.rt_timer_insert) refers to rt_cmsis.o(.data) for .data
    rt_cmsis.o(i.rt_timer_remove) refers to rt_cmsis.o(.data) for .data
    rt_cmsis.o(i.svcDelay) refers to rt_cmsis.o(i.rt_ms2tick) for rt_ms2tick
    rt_cmsis.o(i.svcDelay) refers to rt_time.o(i.rt_dly_wait) for rt_dly_wait
    rt_cmsis.o(i.svcKernelInitialize) refers to rt_memory.o(i.rt_init_mem) for rt_init_mem
    rt_cmsis.o(i.svcKernelInitialize) refers to rt_task.o(i.rt_sys_init) for rt_sys_init
    rt_cmsis.o(i.svcKernelInitialize) refers to rt_cmsis.o(i.svcMessageCreate) for svcMessageCreate
    rt_cmsis.o(i.svcKernelInitialize) refers to rt_cmsis.o(i.svcThreadCreate) for svcThreadCreate
    rt_cmsis.o(i.svcKernelInitialize) refers to rt_cmsis.o(.data) for .data
    rt_cmsis.o(i.svcKernelInitialize) refers to rtx_conf_cm.o(.bss) for os_stack_mem
    rt_cmsis.o(i.svcKernelInitialize) refers to rtx_conf_cm.o(.constdata) for os_stack_sz
    rt_cmsis.o(i.svcKernelInitialize) refers to rt_task.o(.data) for os_tsk
    rt_cmsis.o(i.svcKernelInitialize) refers to rtx_conf_cm.o(.data) for osMessageQId_osTimerMessageQ
    rt_cmsis.o(i.svcKernelRunning) refers to rt_cmsis.o(.data) for .data
    rt_cmsis.o(i.svcKernelStart) refers to rt_task.o(i.rt_tsk_prio) for rt_tsk_prio
    rt_cmsis.o(i.svcKernelStart) refers to rt_task.o(i.rt_sys_start) for rt_sys_start
    rt_cmsis.o(i.svcKernelStart) refers to rt_cmsis.o(.data) for .data
    rt_cmsis.o(i.svcKernelStart) refers to rt_task.o(.data) for os_tsk
    rt_cmsis.o(i.svcKernelSysTick) refers to rt_system.o(i.os_tick_val) for os_tick_val
    rt_cmsis.o(i.svcKernelSysTick) refers to rt_system.o(i.os_tick_ovf) for os_tick_ovf
    rt_cmsis.o(i.svcKernelSysTick) refers to rtx_conf_cm.o(.constdata) for os_trv
    rt_cmsis.o(i.svcKernelSysTick) refers to rt_time.o(.data) for os_time
    rt_cmsis.o(i.svcMailCreate) refers to rt_membox.o(i._init_box) for _init_box
    rt_cmsis.o(i.svcMailCreate) refers to rt_mailbox.o(i.rt_mbx_init) for rt_mbx_init
    rt_cmsis.o(i.svcMessageCreate) refers to rt_mailbox.o(i.rt_mbx_init) for rt_mbx_init
    rt_cmsis.o(i.svcMessageGet) refers to rt_cmsis.o(i.rt_ms2tick) for rt_ms2tick
    rt_cmsis.o(i.svcMessageGet) refers to rt_mailbox.o(i.rt_mbx_wait) for rt_mbx_wait
    rt_cmsis.o(i.svcMessagePut) refers to rt_cmsis.o(i.rt_ms2tick) for rt_ms2tick
    rt_cmsis.o(i.svcMessagePut) refers to rt_mailbox.o(i.rt_mbx_send) for rt_mbx_send
    rt_cmsis.o(i.svcMutexCreate) refers to rt_mutex.o(i.rt_mut_init) for rt_mut_init
    rt_cmsis.o(i.svcMutexDelete) refers to rt_cmsis.o(i.rt_id2obj) for rt_id2obj
    rt_cmsis.o(i.svcMutexDelete) refers to rt_mutex.o(i.rt_mut_delete) for rt_mut_delete
    rt_cmsis.o(i.svcMutexRelease) refers to rt_cmsis.o(i.rt_id2obj) for rt_id2obj
    rt_cmsis.o(i.svcMutexRelease) refers to rt_mutex.o(i.rt_mut_release) for rt_mut_release
    rt_cmsis.o(i.svcMutexWait) refers to rt_cmsis.o(i.rt_id2obj) for rt_id2obj
    rt_cmsis.o(i.svcMutexWait) refers to rt_cmsis.o(i.rt_ms2tick) for rt_ms2tick
    rt_cmsis.o(i.svcMutexWait) refers to rt_mutex.o(i.rt_mut_wait) for rt_mut_wait
    rt_cmsis.o(i.svcPoolCreate) refers to rt_membox.o(i._init_box) for _init_box
    rt_cmsis.o(i.svcSemaphoreCreate) refers to rt_semaphore.o(i.rt_sem_init) for rt_sem_init
    rt_cmsis.o(i.svcSemaphoreDelete) refers to rt_cmsis.o(i.rt_id2obj) for rt_id2obj
    rt_cmsis.o(i.svcSemaphoreDelete) refers to rt_semaphore.o(i.rt_sem_delete) for rt_sem_delete
    rt_cmsis.o(i.svcSemaphoreRelease) refers to rt_cmsis.o(i.rt_id2obj) for rt_id2obj
    rt_cmsis.o(i.svcSemaphoreRelease) refers to rt_semaphore.o(i.rt_sem_send) for rt_sem_send
    rt_cmsis.o(i.svcSemaphoreWait) refers to rt_cmsis.o(i.rt_id2obj) for rt_id2obj
    rt_cmsis.o(i.svcSemaphoreWait) refers to rt_cmsis.o(i.rt_ms2tick) for rt_ms2tick
    rt_cmsis.o(i.svcSemaphoreWait) refers to rt_semaphore.o(i.rt_sem_wait) for rt_sem_wait
    rt_cmsis.o(i.svcSignalClear) refers to rt_cmsis.o(i.rt_tid2ptcb) for rt_tid2ptcb
    rt_cmsis.o(i.svcSignalClear) refers to rt_event.o(i.rt_evt_clr) for rt_evt_clr
    rt_cmsis.o(i.svcSignalSet) refers to rt_cmsis.o(i.rt_tid2ptcb) for rt_tid2ptcb
    rt_cmsis.o(i.svcSignalSet) refers to rt_event.o(i.rt_evt_set) for rt_evt_set
    rt_cmsis.o(i.svcSignalWait) refers to rt_cmsis.o(i.rt_ms2tick) for rt_ms2tick
    rt_cmsis.o(i.svcSignalWait) refers to rt_event.o(i.rt_evt_wait) for rt_evt_wait
    rt_cmsis.o(i.svcSignalWait) refers to rt_task.o(.data) for os_tsk
    rt_cmsis.o(i.svcThreadCreate) refers to rt_memory.o(i.rt_alloc_mem) for rt_alloc_mem
    rt_cmsis.o(i.svcThreadCreate) refers to rt_task.o(i.rt_tsk_create) for rt_tsk_create
    rt_cmsis.o(i.svcThreadCreate) refers to rt_memory.o(i.rt_free_mem) for rt_free_mem
    rt_cmsis.o(i.svcThreadCreate) refers to rtx_conf_cm.o(.bss) for os_stack_mem
    rt_cmsis.o(i.svcThreadCreate) refers to rt_cmsis.o(i.osThreadExit) for osThreadExit
    rt_cmsis.o(i.svcThreadGetId) refers to rt_task.o(i.rt_tsk_self) for rt_tsk_self
    rt_cmsis.o(i.svcThreadGetId) refers to rtx_conf_cm.o(.bss) for os_active_TCB
    rt_cmsis.o(i.svcThreadGetPriority) refers to rt_cmsis.o(i.rt_tid2ptcb) for rt_tid2ptcb
    rt_cmsis.o(i.svcThreadSetPriority) refers to rt_cmsis.o(i.rt_tid2ptcb) for rt_tid2ptcb
    rt_cmsis.o(i.svcThreadSetPriority) refers to rt_task.o(i.rt_tsk_prio) for rt_tsk_prio
    rt_cmsis.o(i.svcThreadTerminate) refers to rt_cmsis.o(i.rt_tid2ptcb) for rt_tid2ptcb
    rt_cmsis.o(i.svcThreadTerminate) refers to rt_task.o(i.rt_tsk_delete) for rt_tsk_delete
    rt_cmsis.o(i.svcThreadTerminate) refers to rt_memory.o(i.rt_free_mem) for rt_free_mem
    rt_cmsis.o(i.svcThreadTerminate) refers to rtx_conf_cm.o(.bss) for os_stack_mem
    rt_cmsis.o(i.svcThreadYield) refers to rt_task.o(i.rt_tsk_pass) for rt_tsk_pass
    rt_cmsis.o(i.svcTimerCall) refers to rt_cmsis.o(i.rt_id2obj) for rt_id2obj
    rt_cmsis.o(i.svcTimerCreate) refers to rtx_conf_cm.o(.data) for osThreadId_osTimerThread
    rt_cmsis.o(i.svcTimerDelete) refers to rt_cmsis.o(i.rt_id2obj) for rt_id2obj
    rt_cmsis.o(i.svcTimerDelete) refers to rt_cmsis.o(i.rt_timer_remove) for rt_timer_remove
    rt_cmsis.o(i.svcTimerStart) refers to rt_cmsis.o(i.rt_id2obj) for rt_id2obj
    rt_cmsis.o(i.svcTimerStart) refers to lludivv7m.o(.text) for __aeabi_uldivmod
    rt_cmsis.o(i.svcTimerStart) refers to rt_cmsis.o(i.rt_timer_remove) for rt_timer_remove
    rt_cmsis.o(i.svcTimerStart) refers to rt_cmsis.o(i.rt_timer_insert) for rt_timer_insert
    rt_cmsis.o(i.svcTimerStart) refers to rtx_conf_cm.o(.constdata) for os_clockrate
    rt_cmsis.o(i.svcTimerStop) refers to rt_cmsis.o(i.rt_id2obj) for rt_id2obj
    rt_cmsis.o(i.svcTimerStop) refers to rt_cmsis.o(i.rt_timer_remove) for rt_timer_remove
    rt_cmsis.o(i.sysMailAlloc) refers to rt_membox.o(i.rt_alloc_box) for rt_alloc_box
    rt_cmsis.o(i.sysMailAlloc) refers to rt_list.o(i.rt_put_prio) for rt_put_prio
    rt_cmsis.o(i.sysMailAlloc) refers to rt_cmsis.o(i.rt_ms2tick) for rt_ms2tick
    rt_cmsis.o(i.sysMailAlloc) refers to rt_task.o(i.rt_block) for rt_block
    rt_cmsis.o(i.sysMailAlloc) refers to rt_task.o(.data) for os_tsk
    rt_cmsis.o(i.sysMailFree) refers to rt_membox.o(i.rt_free_box) for rt_free_box
    rt_cmsis.o(i.sysMailFree) refers to rt_list.o(i.rt_psq_enq) for rt_psq_enq
    rt_cmsis.o(i.sysMailFree) refers to rt_system.o(i.rt_psh_req) for rt_psh_req
    rt_cmsis.o(i.sysMailFree) refers to rt_membox.o(i.rt_alloc_box) for rt_alloc_box
    rt_cmsis.o(i.sysMailFree) refers to rt_list.o(i.rt_get_first) for rt_get_first
    rt_cmsis.o(i.sysMailFree) refers to hal_cm.o(i.rt_ret_val) for rt_ret_val
    rt_cmsis.o(i.sysMailFree) refers to rt_list.o(i.rt_rmv_dly) for rt_rmv_dly
    rt_cmsis.o(i.sysMailFree) refers to rt_task.o(i.rt_dispatch) for rt_dispatch
    rt_cmsis.o(i.sysPoolAlloc) refers to rt_membox.o(i.rt_alloc_box) for rt_alloc_box
    rt_cmsis.o(i.sysPoolFree) refers to rt_membox.o(i.rt_free_box) for rt_free_box
    rt_cmsis.o(i.sysTimerTick) refers to rt_cmsis.o(i.isrMessagePut) for isrMessagePut
    rt_cmsis.o(i.sysTimerTick) refers to rtx_conf_cm.o(i.os_error) for os_error
    rt_cmsis.o(i.sysTimerTick) refers to rt_cmsis.o(i.rt_timer_insert) for rt_timer_insert
    rt_cmsis.o(i.sysTimerTick) refers to rt_cmsis.o(.data) for .data
    rt_cmsis.o(i.sysTimerTick) refers to rtx_conf_cm.o(.data) for osMessageQId_osTimerMessageQ
    rt_cmsis.o(i.sysUserTimerUpdate) refers to rt_cmsis.o(i.sysTimerTick) for sysTimerTick
    rt_cmsis.o(i.sysUserTimerUpdate) refers to rt_cmsis.o(.data) for .data
    rt_cmsis.o(i.sysUserTimerWakeupTime) refers to rt_cmsis.o(.data) for .data
    rt_task.o(i.rt_block) refers to rt_list.o(i.rt_put_dly) for rt_put_dly
    rt_task.o(i.rt_block) refers to rt_list.o(i.rt_get_first) for rt_get_first
    rt_task.o(i.rt_block) refers to rt_task.o(i.rt_switch_req) for rt_switch_req
    rt_task.o(i.rt_block) refers to rt_task.o(.data) for .data
    rt_task.o(i.rt_block) refers to rt_list.o(.bss) for os_rdy
    rt_task.o(i.rt_dispatch) refers to rt_list.o(i.rt_put_rdy_first) for rt_put_rdy_first
    rt_task.o(i.rt_dispatch) refers to rt_task.o(i.rt_switch_req) for rt_switch_req
    rt_task.o(i.rt_dispatch) refers to rt_list.o(i.rt_get_first) for rt_get_first
    rt_task.o(i.rt_dispatch) refers to rt_list.o(i.rt_put_prio) for rt_put_prio
    rt_task.o(i.rt_dispatch) refers to rt_task.o(.data) for .data
    rt_task.o(i.rt_dispatch) refers to rt_list.o(.bss) for os_rdy
    rt_task.o(i.rt_init_context) refers to rt_membox.o(i.rt_alloc_box) for rt_alloc_box
    rt_task.o(i.rt_init_context) refers to hal_cm.o(i.rt_init_stack) for rt_init_stack
    rt_task.o(i.rt_init_context) refers to rtx_conf_cm.o(.bss) for mp_stk
    rt_task.o(i.rt_switch_req) refers to hal_cm.o(i.dbg_task_switch) for dbg_task_switch
    rt_task.o(i.rt_switch_req) refers to rt_task.o(.data) for .data
    rt_task.o(i.rt_switch_req) refers to hal_cm.o(.data) for dbg_msg
    rt_task.o(i.rt_sys_init) refers to hal_cm.o(i.dbg_init) for dbg_init
    rt_task.o(i.rt_sys_init) refers to rt_membox.o(i._init_box) for _init_box
    rt_task.o(i.rt_sys_init) refers to rt_task.o(i.rt_init_context) for rt_init_context
    rt_task.o(i.rt_sys_init) refers to rt_robin.o(i.rt_init_robin) for rt_init_robin
    rt_task.o(i.rt_sys_init) refers to rtx_conf_cm.o(.bss) for os_active_TCB
    rt_task.o(i.rt_sys_init) refers to rtx_conf_cm.o(.constdata) for os_maxtaskrun
    rt_task.o(i.rt_sys_init) refers to rtx_conf_cm.o(.data) for m_tmr
    rt_task.o(i.rt_sys_init) refers to rt_task.o(.bss) for .bss
    rt_task.o(i.rt_sys_init) refers to rtx_conf_cm.o(i.os_idle_demon) for os_idle_demon
    rt_task.o(i.rt_sys_init) refers to rt_list.o(.bss) for os_rdy
    rt_task.o(i.rt_sys_init) refers to rt_task.o(.data) for .data
    rt_task.o(i.rt_sys_start) refers to rt_system.o(i.os_tick_init) for os_tick_init
    rt_task.o(i.rt_sys_start) refers to rt_system.o(.data) for os_tick_irqn
    rt_task.o(i.rt_tsk_create) refers to rt_membox.o(i.rt_alloc_box) for rt_alloc_box
    rt_task.o(i.rt_tsk_create) refers to rt_task.o(i.rt_init_context) for rt_init_context
    rt_task.o(i.rt_tsk_create) refers to hal_cm.o(i.dbg_task_notify) for dbg_task_notify
    rt_task.o(i.rt_tsk_create) refers to rt_task.o(i.rt_dispatch) for rt_dispatch
    rt_task.o(i.rt_tsk_create) refers to rtx_conf_cm.o(.bss) for mp_tcb
    rt_task.o(i.rt_tsk_create) refers to rtx_conf_cm.o(.constdata) for os_maxtaskrun
    rt_task.o(i.rt_tsk_create) refers to hal_cm.o(.data) for dbg_msg
    rt_task.o(i.rt_tsk_delete) refers to hal_cm3.o(.emb_text) for rt_get_PSP
    rt_task.o(i.rt_tsk_delete) refers to rt_system.o(i.rt_stk_check) for rt_stk_check
    rt_task.o(i.rt_tsk_delete) refers to rt_list.o(i.rt_get_first) for rt_get_first
    rt_task.o(i.rt_tsk_delete) refers to hal_cm.o(i.rt_ret_val) for rt_ret_val
    rt_task.o(i.rt_tsk_delete) refers to rt_list.o(i.rt_rmv_dly) for rt_rmv_dly
    rt_task.o(i.rt_tsk_delete) refers to rt_list.o(i.rt_put_prio) for rt_put_prio
    rt_task.o(i.rt_tsk_delete) refers to rt_membox.o(i.rt_free_box) for rt_free_box
    rt_task.o(i.rt_tsk_delete) refers to hal_cm.o(i.dbg_task_notify) for dbg_task_notify
    rt_task.o(i.rt_tsk_delete) refers to rt_list.o(i.rt_rmv_list) for rt_rmv_list
    rt_task.o(i.rt_tsk_delete) refers to rt_task.o(i.rt_dispatch) for rt_dispatch
    rt_task.o(i.rt_tsk_delete) refers to hal_cm.o(.data) for dbg_msg
    rt_task.o(i.rt_tsk_delete) refers to rtx_conf_cm.o(.bss) for os_active_TCB
    rt_task.o(i.rt_tsk_delete) refers to rt_task.o(.data) for .data
    rt_task.o(i.rt_tsk_delete) refers to rt_list.o(.bss) for os_rdy
    rt_task.o(i.rt_tsk_delete) refers to rtx_conf_cm.o(.constdata) for os_maxtaskrun
    rt_task.o(i.rt_tsk_pass) refers to rt_list.o(i.rt_get_same_rdy_prio) for rt_get_same_rdy_prio
    rt_task.o(i.rt_tsk_pass) refers to rt_list.o(i.rt_put_prio) for rt_put_prio
    rt_task.o(i.rt_tsk_pass) refers to rt_task.o(i.rt_switch_req) for rt_switch_req
    rt_task.o(i.rt_tsk_pass) refers to rt_task.o(.data) for .data
    rt_task.o(i.rt_tsk_pass) refers to rt_list.o(.bss) for os_rdy
    rt_task.o(i.rt_tsk_prio) refers to rt_list.o(i.rt_put_prio) for rt_put_prio
    rt_task.o(i.rt_tsk_prio) refers to rt_list.o(i.rt_resort_prio) for rt_resort_prio
    rt_task.o(i.rt_tsk_prio) refers to rt_list.o(i.rt_get_first) for rt_get_first
    rt_task.o(i.rt_tsk_prio) refers to rt_task.o(i.rt_dispatch) for rt_dispatch
    rt_task.o(i.rt_tsk_prio) refers to rt_task.o(.data) for .data
    rt_task.o(i.rt_tsk_prio) refers to rtx_conf_cm.o(.constdata) for os_maxtaskrun
    rt_task.o(i.rt_tsk_prio) refers to rtx_conf_cm.o(.bss) for os_active_TCB
    rt_task.o(i.rt_tsk_prio) refers to rt_list.o(.bss) for os_rdy
    rt_task.o(i.rt_tsk_self) refers to rt_task.o(.data) for .data
    rt_mutex.o(i.rt_mut_delete) refers to rt_list.o(i.rt_resort_prio) for rt_resort_prio
    rt_mutex.o(i.rt_mut_delete) refers to rt_list.o(i.rt_get_first) for rt_get_first
    rt_mutex.o(i.rt_mut_delete) refers to hal_cm.o(i.rt_ret_val) for rt_ret_val
    rt_mutex.o(i.rt_mut_delete) refers to rt_list.o(i.rt_rmv_dly) for rt_rmv_dly
    rt_mutex.o(i.rt_mut_delete) refers to rt_list.o(i.rt_put_prio) for rt_put_prio
    rt_mutex.o(i.rt_mut_delete) refers to rt_task.o(i.rt_dispatch) for rt_dispatch
    rt_mutex.o(i.rt_mut_delete) refers to rt_task.o(.data) for os_tsk
    rt_mutex.o(i.rt_mut_delete) refers to rt_list.o(.bss) for os_rdy
    rt_mutex.o(i.rt_mut_release) refers to rt_list.o(i.rt_get_first) for rt_get_first
    rt_mutex.o(i.rt_mut_release) refers to hal_cm.o(i.rt_ret_val) for rt_ret_val
    rt_mutex.o(i.rt_mut_release) refers to rt_list.o(i.rt_rmv_dly) for rt_rmv_dly
    rt_mutex.o(i.rt_mut_release) refers to rt_list.o(i.rt_put_prio) for rt_put_prio
    rt_mutex.o(i.rt_mut_release) refers to rt_task.o(i.rt_dispatch) for rt_dispatch
    rt_mutex.o(i.rt_mut_release) refers to rt_task.o(.data) for os_tsk
    rt_mutex.o(i.rt_mut_release) refers to rt_list.o(.bss) for os_rdy
    rt_mutex.o(i.rt_mut_wait) refers to rt_list.o(i.rt_resort_prio) for rt_resort_prio
    rt_mutex.o(i.rt_mut_wait) refers to rt_list.o(i.rt_put_prio) for rt_put_prio
    rt_mutex.o(i.rt_mut_wait) refers to rt_task.o(i.rt_block) for rt_block
    rt_mutex.o(i.rt_mut_wait) refers to rt_task.o(.data) for os_tsk
    rt_system.o(i.os_tick_init) refers to rtx_conf_cm.o(.constdata) for os_trv
    rt_system.o(i.os_tick_val) refers to rtx_conf_cm.o(.constdata) for os_trv
    rt_system.o(i.rt_pop_req) refers to rt_list.o(i.rt_put_rdy_first) for rt_put_rdy_first
    rt_system.o(i.rt_pop_req) refers to rt_semaphore.o(i.rt_sem_psh) for rt_sem_psh
    rt_system.o(i.rt_pop_req) refers to rt_list.o(i.rt_get_first) for rt_get_first
    rt_system.o(i.rt_pop_req) refers to rt_task.o(i.rt_switch_req) for rt_switch_req
    rt_system.o(i.rt_pop_req) refers to rt_event.o(i.rt_evt_psh) for rt_evt_psh
    rt_system.o(i.rt_pop_req) refers to rt_mailbox.o(i.rt_mbx_psh) for rt_mbx_psh
    rt_system.o(i.rt_pop_req) refers to rt_task.o(.data) for os_tsk
    rt_system.o(i.rt_pop_req) refers to rtx_conf_cm.o(.bss) for os_fifo
    rt_system.o(i.rt_pop_req) refers to rt_list.o(.bss) for os_rdy
    rt_system.o(i.rt_psh_req) refers to rt_system.o(.data) for .data
    rt_system.o(i.rt_resume) refers to rt_list.o(i.rt_put_rdy_first) for rt_put_rdy_first
    rt_system.o(i.rt_resume) refers to rt_list.o(i.rt_dec_dly) for rt_dec_dly
    rt_system.o(i.rt_resume) refers to rt_cmsis.o(i.sysUserTimerUpdate) for sysUserTimerUpdate
    rt_system.o(i.rt_resume) refers to rt_list.o(i.rt_get_first) for rt_get_first
    rt_system.o(i.rt_resume) refers to rt_task.o(i.rt_switch_req) for rt_switch_req
    rt_system.o(i.rt_resume) refers to rt_system.o(i.rt_tsk_unlock) for rt_tsk_unlock
    rt_system.o(i.rt_resume) refers to rt_task.o(.data) for os_tsk
    rt_system.o(i.rt_resume) refers to rt_robin.o(.data) for os_robin
    rt_system.o(i.rt_resume) refers to rt_list.o(.bss) for os_dly
    rt_system.o(i.rt_resume) refers to rt_time.o(.data) for os_time
    rt_system.o(i.rt_stk_check) refers to rtx_conf_cm.o(i.os_error) for os_error
    rt_system.o(i.rt_stk_check) refers to rt_task.o(.data) for os_tsk
    rt_system.o(i.rt_suspend) refers to rt_system.o(i.rt_tsk_lock) for rt_tsk_lock
    rt_system.o(i.rt_suspend) refers to rt_cmsis.o(i.sysUserTimerWakeupTime) for sysUserTimerWakeupTime
    rt_system.o(i.rt_suspend) refers to rt_list.o(.bss) for os_dly
    rt_system.o(i.rt_systick) refers to rt_list.o(i.rt_put_rdy_first) for rt_put_rdy_first
    rt_system.o(i.rt_systick) refers to rt_robin.o(i.rt_chk_robin) for rt_chk_robin
    rt_system.o(i.rt_systick) refers to rt_list.o(i.rt_dec_dly) for rt_dec_dly
    rt_system.o(i.rt_systick) refers to rt_cmsis.o(i.sysTimerTick) for sysTimerTick
    rt_system.o(i.rt_systick) refers to rt_list.o(i.rt_get_first) for rt_get_first
    rt_system.o(i.rt_systick) refers to rt_task.o(i.rt_switch_req) for rt_switch_req
    rt_system.o(i.rt_systick) refers to rt_task.o(.data) for os_tsk
    rt_system.o(i.rt_systick) refers to rt_time.o(.data) for os_time
    rt_system.o(i.rt_systick) refers to rt_list.o(.bss) for os_rdy
    rt_system.o(i.rt_tsk_lock) refers to rt_system.o(.data) for .data
    rt_system.o(i.rt_tsk_unlock) refers to rt_system.o(.data) for .data
    rt_event.o(i.isr_evt_set) refers to rt_list.o(i.rt_psq_enq) for rt_psq_enq
    rt_event.o(i.isr_evt_set) refers to rt_system.o(i.rt_psh_req) for rt_psh_req
    rt_event.o(i.isr_evt_set) refers to rtx_conf_cm.o(.bss) for os_active_TCB
    rt_event.o(i.rt_evt_clr) refers to rtx_conf_cm.o(.bss) for os_active_TCB
    rt_event.o(i.rt_evt_get) refers to rt_task.o(.data) for os_tsk
    rt_event.o(i.rt_evt_psh) refers to rt_list.o(i.rt_rmv_dly) for rt_rmv_dly
    rt_event.o(i.rt_evt_psh) refers to hal_cm.o(i.rt_ret_val2) for rt_ret_val2
    rt_event.o(i.rt_evt_psh) refers to rt_list.o(i.rt_put_prio) for rt_put_prio
    rt_event.o(i.rt_evt_psh) refers to rt_list.o(.bss) for os_rdy
    rt_event.o(i.rt_evt_set) refers to rt_list.o(i.rt_rmv_dly) for rt_rmv_dly
    rt_event.o(i.rt_evt_set) refers to hal_cm.o(i.rt_ret_val2) for rt_ret_val2
    rt_event.o(i.rt_evt_set) refers to rt_task.o(i.rt_dispatch) for rt_dispatch
    rt_event.o(i.rt_evt_set) refers to rtx_conf_cm.o(.bss) for os_active_TCB
    rt_event.o(i.rt_evt_wait) refers to rt_task.o(i.rt_block) for rt_block
    rt_event.o(i.rt_evt_wait) refers to rt_task.o(.data) for os_tsk
    rt_list.o(i.rt_dec_dly) refers to rt_list.o(i.rt_put_prio) for rt_put_prio
    rt_list.o(i.rt_dec_dly) refers to rt_list.o(.bss) for .bss
    rt_list.o(i.rt_dec_dly) refers to rt_time.o(.data) for os_time
    rt_list.o(i.rt_get_same_rdy_prio) refers to rt_list.o(.bss) for .bss
    rt_list.o(i.rt_get_same_rdy_prio) refers to rt_task.o(.data) for os_tsk
    rt_list.o(i.rt_psq_enq) refers to rtx_conf_cm.o(i.os_error) for os_error
    rt_list.o(i.rt_psq_enq) refers to rtx_conf_cm.o(.bss) for os_fifo
    rt_list.o(i.rt_put_dly) refers to rt_list.o(.bss) for .bss
    rt_list.o(i.rt_put_rdy_first) refers to rt_list.o(.bss) for .bss
    rt_list.o(i.rt_resort_prio) refers to rt_list.o(i.rt_rmv_list) for rt_rmv_list
    rt_list.o(i.rt_resort_prio) refers to rt_list.o(i.rt_put_prio) for rt_put_prio
    rt_list.o(i.rt_resort_prio) refers to rt_list.o(.bss) for .bss
    rt_list.o(i.rt_rmv_list) refers to rt_list.o(.bss) for .bss
    rt_mailbox.o(i.isr_mbx_receive) refers to rt_list.o(i.rt_psq_enq) for rt_psq_enq
    rt_mailbox.o(i.isr_mbx_receive) refers to rt_system.o(i.rt_psh_req) for rt_psh_req
    rt_mailbox.o(i.isr_mbx_send) refers to rt_list.o(i.rt_psq_enq) for rt_psq_enq
    rt_mailbox.o(i.isr_mbx_send) refers to rt_system.o(i.rt_psh_req) for rt_psh_req
    rt_mailbox.o(i.rt_mbx_psh) refers to rt_membox.o(i.rt_alloc_box) for rt_alloc_box
    rt_mailbox.o(i.rt_mbx_psh) refers to rt_list.o(i.rt_get_first) for rt_get_first
    rt_mailbox.o(i.rt_mbx_psh) refers to hal_cm.o(i.rt_ret_val) for rt_ret_val
    rt_mailbox.o(i.rt_mbx_psh) refers to rt_list.o(i.rt_rmv_dly) for rt_rmv_dly
    rt_mailbox.o(i.rt_mbx_psh) refers to rt_list.o(i.rt_put_prio) for rt_put_prio
    rt_mailbox.o(i.rt_mbx_psh) refers to hal_cm.o(i.rt_ret_val2) for rt_ret_val2
    rt_mailbox.o(i.rt_mbx_psh) refers to rtx_conf_cm.o(i.os_error) for os_error
    rt_mailbox.o(i.rt_mbx_psh) refers to rt_list.o(.bss) for os_rdy
    rt_mailbox.o(i.rt_mbx_send) refers to rt_list.o(i.rt_put_prio) for rt_put_prio
    rt_mailbox.o(i.rt_mbx_send) refers to rt_list.o(i.rt_get_first) for rt_get_first
    rt_mailbox.o(i.rt_mbx_send) refers to hal_cm.o(i.rt_ret_val2) for rt_ret_val2
    rt_mailbox.o(i.rt_mbx_send) refers to rt_list.o(i.rt_rmv_dly) for rt_rmv_dly
    rt_mailbox.o(i.rt_mbx_send) refers to rt_task.o(i.rt_dispatch) for rt_dispatch
    rt_mailbox.o(i.rt_mbx_send) refers to rt_task.o(i.rt_block) for rt_block
    rt_mailbox.o(i.rt_mbx_send) refers to rt_task.o(.data) for os_tsk
    rt_mailbox.o(i.rt_mbx_wait) refers to rt_list.o(i.rt_get_first) for rt_get_first
    rt_mailbox.o(i.rt_mbx_wait) refers to hal_cm.o(i.rt_ret_val) for rt_ret_val
    rt_mailbox.o(i.rt_mbx_wait) refers to rt_list.o(i.rt_rmv_dly) for rt_rmv_dly
    rt_mailbox.o(i.rt_mbx_wait) refers to rt_task.o(i.rt_dispatch) for rt_dispatch
    rt_mailbox.o(i.rt_mbx_wait) refers to rt_list.o(i.rt_put_prio) for rt_put_prio
    rt_mailbox.o(i.rt_mbx_wait) refers to rt_task.o(i.rt_block) for rt_block
    rt_mailbox.o(i.rt_mbx_wait) refers to rt_task.o(.data) for os_tsk
    rt_semaphore.o(i.isr_sem_send) refers to rt_list.o(i.rt_psq_enq) for rt_psq_enq
    rt_semaphore.o(i.isr_sem_send) refers to rt_system.o(i.rt_psh_req) for rt_psh_req
    rt_semaphore.o(i.rt_sem_delete) refers to rt_list.o(i.rt_get_first) for rt_get_first
    rt_semaphore.o(i.rt_sem_delete) refers to hal_cm.o(i.rt_ret_val) for rt_ret_val
    rt_semaphore.o(i.rt_sem_delete) refers to rt_list.o(i.rt_rmv_dly) for rt_rmv_dly
    rt_semaphore.o(i.rt_sem_delete) refers to rt_list.o(i.rt_put_prio) for rt_put_prio
    rt_semaphore.o(i.rt_sem_delete) refers to rt_task.o(i.rt_dispatch) for rt_dispatch
    rt_semaphore.o(i.rt_sem_delete) refers to rt_list.o(.bss) for os_rdy
    rt_semaphore.o(i.rt_sem_delete) refers to rt_task.o(.data) for os_tsk
    rt_semaphore.o(i.rt_sem_psh) refers to rt_list.o(i.rt_get_first) for rt_get_first
    rt_semaphore.o(i.rt_sem_psh) refers to rt_list.o(i.rt_rmv_dly) for rt_rmv_dly
    rt_semaphore.o(i.rt_sem_psh) refers to hal_cm.o(i.rt_ret_val) for rt_ret_val
    rt_semaphore.o(i.rt_sem_psh) refers to rt_list.o(i.rt_put_prio) for rt_put_prio
    rt_semaphore.o(i.rt_sem_psh) refers to rt_list.o(.bss) for os_rdy
    rt_semaphore.o(i.rt_sem_send) refers to rt_list.o(i.rt_get_first) for rt_get_first
    rt_semaphore.o(i.rt_sem_send) refers to hal_cm.o(i.rt_ret_val) for rt_ret_val
    rt_semaphore.o(i.rt_sem_send) refers to rt_list.o(i.rt_rmv_dly) for rt_rmv_dly
    rt_semaphore.o(i.rt_sem_send) refers to rt_task.o(i.rt_dispatch) for rt_dispatch
    rt_semaphore.o(i.rt_sem_wait) refers to rt_list.o(i.rt_put_prio) for rt_put_prio
    rt_semaphore.o(i.rt_sem_wait) refers to rt_task.o(i.rt_block) for rt_block
    rt_semaphore.o(i.rt_sem_wait) refers to rt_task.o(.data) for os_tsk
    rt_time.o(i.rt_dly_wait) refers to rt_task.o(i.rt_block) for rt_block
    rt_time.o(i.rt_itv_set) refers to rt_task.o(.data) for os_tsk
    rt_time.o(i.rt_itv_set) refers to rt_time.o(.data) for .data
    rt_time.o(i.rt_itv_wait) refers to rt_task.o(i.rt_block) for rt_block
    rt_time.o(i.rt_itv_wait) refers to rt_task.o(.data) for os_tsk
    rt_time.o(i.rt_itv_wait) refers to rt_time.o(.data) for .data
    rt_time.o(i.rt_time_get) refers to rt_time.o(.data) for .data
    rt_robin.o(i.rt_chk_robin) refers to rt_list.o(i.rt_get_first) for rt_get_first
    rt_robin.o(i.rt_chk_robin) refers to rt_list.o(i.rt_put_prio) for rt_put_prio
    rt_robin.o(i.rt_chk_robin) refers to rt_robin.o(.data) for .data
    rt_robin.o(i.rt_chk_robin) refers to rt_list.o(.bss) for os_rdy
    rt_robin.o(i.rt_chk_robin) refers to rt_time.o(.data) for os_time
    rt_robin.o(i.rt_init_robin) refers to rt_robin.o(.data) for .data
    rt_robin.o(i.rt_init_robin) refers to rtx_conf_cm.o(.constdata) for os_rrobin
    rt_membox.o(i._calloc_box) refers to hal_cm3.o(.emb_text) for _alloc_box
    hal_cm.o(i.dbg_init) refers to hal_cm.o(.data) for .data
    hal_cm.o(i.rt_init_stack) refers to rtx_conf_cm.o(.constdata) for os_stackinfo
    hal_cm3.o(.emb_text) refers to rtx_conf_cm.o(.constdata) for os_flags
    hal_cm3.o(.emb_text) refers to rt_membox.o(i.rt_alloc_box) for rt_alloc_box
    hal_cm3.o(.emb_text) refers to rt_membox.o(i.rt_free_box) for rt_free_box
    hal_cm3.o(.emb_text) refers to rt_system.o(i.rt_stk_check) for rt_stk_check
    hal_cm3.o(.emb_text) refers to rt_task.o(.data) for os_tsk
    hal_cm3.o(.emb_text) refers to svc_table.o(SVC_TABLE) for SVC_Count
    hal_cm3.o(.emb_text) refers to rt_system.o(i.rt_pop_req) for rt_pop_req
    hal_cm3.o(.emb_text) refers to rt_system.o(i.rt_systick) for rt_systick
    hal_cm3.o(.emb_text) refers to rt_system.o(i.os_tick_irqack) for os_tick_irqack
    libspace.o(.text) refers to libspace.o(.bss) for __libspace_start
    __2sprintf.o(.text) refers to _printf_char_common.o(.text) for _printf_char_common
    __2sprintf.o(.text) refers to _sputc.o(.text) for _sputc
    noretval__2sprintf.o(.text) refers to _printf_char_common.o(.text) for _printf_char_common
    noretval__2sprintf.o(.text) refers to _sputc.o(.text) for _sputc
    __printf.o(.text) refers to _printf_percent.o(.ARM.Collect$$_printf_percent$$00000000) for _printf_percent
    _printf_str.o(.text) refers (Special) to _printf_char.o(.text) for _printf_cs_common
    _printf_str.o(.text) refers (Weak) to _printf_pad.o(.text) for _printf_pre_padding
    _printf_str.o(.text) refers (Weak) to _printf_pad.o(.text) for _printf_post_padding
    _printf_dec.o(.text) refers to _printf_intcommon.o(.text) for _printf_int_common
    __printf_flags.o(.text) refers to _printf_percent.o(.ARM.Collect$$_printf_percent$$00000000) for _printf_percent
    __printf_flags.o(.text) refers to __printf_flags.o(.constdata) for .constdata
    __printf_ss.o(.text) refers to _printf_percent.o(.ARM.Collect$$_printf_percent$$00000000) for _printf_percent
    __printf_flags_ss.o(.text) refers to _printf_percent.o(.ARM.Collect$$_printf_percent$$00000000) for _printf_percent
    __printf_flags_ss.o(.text) refers to __printf_flags_ss.o(.constdata) for .constdata
    __printf_wp.o(.text) refers to __printf_wp.o(i._is_digit) for _is_digit
    __printf_wp.o(.text) refers to _printf_percent.o(.ARM.Collect$$_printf_percent$$00000000) for _printf_percent
    __printf_flags_wp.o(.text) refers to __printf_wp.o(i._is_digit) for _is_digit
    __printf_flags_wp.o(.text) refers to _printf_percent.o(.ARM.Collect$$_printf_percent$$00000000) for _printf_percent
    __printf_flags_wp.o(.text) refers to __printf_flags_wp.o(.constdata) for .constdata
    __printf_ss_wp.o(.text) refers to __printf_wp.o(i._is_digit) for _is_digit
    __printf_ss_wp.o(.text) refers to _printf_percent.o(.ARM.Collect$$_printf_percent$$00000000) for _printf_percent
    __printf_flags_ss_wp.o(.text) refers to __printf_wp.o(i._is_digit) for _is_digit
    __printf_flags_ss_wp.o(.text) refers to _printf_percent.o(.ARM.Collect$$_printf_percent$$00000000) for _printf_percent
    __printf_flags_ss_wp.o(.text) refers to __printf_flags_ss_wp.o(.constdata) for .constdata
    _printf_s.o(.ARM.Collect$$_printf_percent$$00000014) refers (Weak) to _printf_char.o(.text) for _printf_string
    _printf_d.o(.ARM.Collect$$_printf_percent$$00000009) refers (Weak) to _printf_dec.o(.text) for _printf_int_dec
    _printf_f.o(.ARM.Collect$$_printf_percent$$00000003) refers (Weak) to printf1.o(x$fpl$printf1) for _printf_fp_dec
    _printf_percent.o(.ARM.Collect$$_printf_percent$$00000000) refers (Special) to _printf_percent_end.o(.ARM.Collect$$_printf_percent$$00000017) for _printf_percent_end
    exit.o(.text) refers to rtexit.o(.ARM.Collect$$rtexit$$00000000) for __rt_exit
    __main.o(!!!main) refers to __rtentry.o(.ARM.Collect$$rtentry$$00000000) for __rt_entry
    d2f.o(x$fpl$d2f) refers (Special) to usenofp.o(x$fpl$usenofp) for __I$use$fp
    d2f.o(x$fpl$d2f) refers to fretinf.o(x$fpl$fretinf) for __fpl_fretinf
    d2f.o(x$fpl$d2f) refers to dnaninf.o(x$fpl$dnaninf) for __fpl_dnaninf
    ddiv.o(x$fpl$drdiv) refers (Special) to usenofp.o(x$fpl$usenofp) for __I$use$fp
    ddiv.o(x$fpl$drdiv) refers to ddiv.o(x$fpl$ddiv) for ddiv_entry
    ddiv.o(x$fpl$ddiv) refers (Special) to usenofp.o(x$fpl$usenofp) for __I$use$fp
    ddiv.o(x$fpl$ddiv) refers to dretinf.o(x$fpl$dretinf) for __fpl_dretinf
    ddiv.o(x$fpl$ddiv) refers to dnaninf.o(x$fpl$dnaninf) for __fpl_dnaninf
    dflt_clz.o(x$fpl$dfltu) refers (Special) to usenofp.o(x$fpl$usenofp) for __I$use$fp
    dflt_clz.o(x$fpl$dflt) refers (Special) to usenofp.o(x$fpl$usenofp) for __I$use$fp
    dflt_clz.o(x$fpl$dfltn) refers (Special) to usenofp.o(x$fpl$usenofp) for __I$use$fp
    dleqf.o(x$fpl$dleqf) refers (Special) to usenofp.o(x$fpl$usenofp) for __I$use$fp
    dleqf.o(x$fpl$dleqf) refers to dnaninf.o(x$fpl$dnaninf) for __fpl_dnaninf
    dleqf.o(x$fpl$dleqf) refers to dcmpi.o(x$fpl$dcmpinf) for __fpl_dcmp_Inf
    dmul.o(x$fpl$dmul) refers (Special) to usenofp.o(x$fpl$usenofp) for __I$use$fp
    dmul.o(x$fpl$dmul) refers to dretinf.o(x$fpl$dretinf) for __fpl_dretinf
    dmul.o(x$fpl$dmul) refers to dnaninf.o(x$fpl$dnaninf) for __fpl_dnaninf
    drleqf.o(x$fpl$drleqf) refers (Special) to usenofp.o(x$fpl$usenofp) for __I$use$fp
    drleqf.o(x$fpl$drleqf) refers to dleqf.o(x$fpl$dleqf) for __fpl_dcmple_InfNaN
    f2d.o(x$fpl$f2d) refers (Special) to usenofp.o(x$fpl$usenofp) for __I$use$fp
    f2d.o(x$fpl$f2d) refers to fnaninf.o(x$fpl$fnaninf) for __fpl_fnaninf
    f2d.o(x$fpl$f2d) refers to dretinf.o(x$fpl$dretinf) for __fpl_dretinf
    faddsub_clz.o(x$fpl$fadd) refers (Special) to usenofp.o(x$fpl$usenofp) for __I$use$fp
    faddsub_clz.o(x$fpl$fadd) refers to faddsub_clz.o(x$fpl$fsub) for _fsub1
    faddsub_clz.o(x$fpl$fadd) refers to fretinf.o(x$fpl$fretinf) for __fpl_fretinf
    faddsub_clz.o(x$fpl$fadd) refers to fnaninf.o(x$fpl$fnaninf) for __fpl_fnaninf
    faddsub_clz.o(x$fpl$frsb) refers (Special) to usenofp.o(x$fpl$usenofp) for __I$use$fp
    faddsub_clz.o(x$fpl$frsb) refers to faddsub_clz.o(x$fpl$fadd) for _fadd1
    faddsub_clz.o(x$fpl$frsb) refers to faddsub_clz.o(x$fpl$fsub) for _fsub1
    faddsub_clz.o(x$fpl$fsub) refers (Special) to usenofp.o(x$fpl$usenofp) for __I$use$fp
    faddsub_clz.o(x$fpl$fsub) refers to faddsub_clz.o(x$fpl$fadd) for _fadd1
    faddsub_clz.o(x$fpl$fsub) refers to fnaninf.o(x$fpl$fnaninf) for __fpl_fnaninf
    fdiv.o(x$fpl$frdiv) refers (Special) to usenofp.o(x$fpl$usenofp) for __I$use$fp
    fdiv.o(x$fpl$frdiv) refers to fdiv.o(x$fpl$fdiv) for _fdiv1
    fdiv.o(x$fpl$fdiv) refers (Special) to usenofp.o(x$fpl$usenofp) for __I$use$fp
    fdiv.o(x$fpl$fdiv) refers to fretinf.o(x$fpl$fretinf) for __fpl_fretinf
    fdiv.o(x$fpl$fdiv) refers to fnaninf.o(x$fpl$fnaninf) for __fpl_fnaninf
    feqf.o(x$fpl$feqf) refers (Special) to usenofp.o(x$fpl$usenofp) for __I$use$fp
    feqf.o(x$fpl$feqf) refers to fnaninf.o(x$fpl$fnaninf) for __fpl_fnaninf
    feqf.o(x$fpl$feqf) refers to fcmpi.o(x$fpl$fcmpinf) for __fpl_fcmp_Inf
    ffix.o(x$fpl$ffix) refers (Special) to usenofp.o(x$fpl$usenofp) for __I$use$fp
    ffix.o(x$fpl$ffix) refers to fnaninf.o(x$fpl$fnaninf) for __fpl_fnaninf
    ffix.o(x$fpl$ffixr) refers (Special) to usenofp.o(x$fpl$usenofp) for __I$use$fp
    ffix.o(x$fpl$ffixr) refers to fnaninf.o(x$fpl$fnaninf) for __fpl_fnaninf
    ffixu.o(x$fpl$ffixu) refers (Special) to usenofp.o(x$fpl$usenofp) for __I$use$fp
    ffixu.o(x$fpl$ffixu) refers to fnaninf.o(x$fpl$fnaninf) for __fpl_fnaninf
    ffixu.o(x$fpl$ffixur) refers (Special) to usenofp.o(x$fpl$usenofp) for __I$use$fp
    ffixu.o(x$fpl$ffixur) refers to fnaninf.o(x$fpl$fnaninf) for __fpl_fnaninf
    fflt_clz.o(x$fpl$ffltu) refers (Special) to usenofp.o(x$fpl$usenofp) for __I$use$fp
    fflt_clz.o(x$fpl$fflt) refers (Special) to usenofp.o(x$fpl$usenofp) for __I$use$fp
    fflt_clz.o(x$fpl$ffltn) refers (Special) to usenofp.o(x$fpl$usenofp) for __I$use$fp
    fleqf.o(x$fpl$fleqf) refers (Special) to usenofp.o(x$fpl$usenofp) for __I$use$fp
    fleqf.o(x$fpl$fleqf) refers to fnaninf.o(x$fpl$fnaninf) for __fpl_fnaninf
    fleqf.o(x$fpl$fleqf) refers to fcmpi.o(x$fpl$fcmpinf) for __fpl_fcmp_Inf
    fmul.o(x$fpl$fmul) refers (Special) to usenofp.o(x$fpl$usenofp) for __I$use$fp
    fmul.o(x$fpl$fmul) refers to fretinf.o(x$fpl$fretinf) for __fpl_fretinf
    fmul.o(x$fpl$fmul) refers to fnaninf.o(x$fpl$fnaninf) for __fpl_fnaninf
    frleqf.o(x$fpl$frleqf) refers (Special) to usenofp.o(x$fpl$usenofp) for __I$use$fp
    frleqf.o(x$fpl$frleqf) refers to fleqf.o(x$fpl$fleqf) for __fpl_fcmple_InfNaN
    printf1.o(x$fpl$printf1) refers to _printf_fp_dec.o(.text) for _printf_fp_dec_real
    __rtentry.o(.ARM.Collect$$rtentry$$00000000) refers (Special) to __rtentry2.o(.ARM.Collect$$rtentry$$0000000A) for __rt_entry_li
    __rtentry.o(.ARM.Collect$$rtentry$$00000000) refers (Special) to __rtentry2.o(.ARM.Collect$$rtentry$$0000000D) for __rt_entry_main
    __rtentry.o(.ARM.Collect$$rtentry$$00000000) refers (Special) to __rtentry2.o(.ARM.Collect$$rtentry$$0000000B) for __rt_entry_postli_1
    __rtentry.o(.ARM.Collect$$rtentry$$00000000) refers (Special) to __rtentry2.o(.ARM.Collect$$rtentry$$00000009) for __rt_entry_postsh_1
    __rtentry.o(.ARM.Collect$$rtentry$$00000000) refers (Special) to __rtentry2.o(.ARM.Collect$$rtentry$$00000002) for __rt_entry_presh_1
    __rtentry.o(.ARM.Collect$$rtentry$$00000000) refers (Special) to __rtentry4.o(.ARM.Collect$$rtentry$$00000004) for __rt_entry_sh
    rtexit.o(.ARM.Collect$$rtexit$$00000000) refers (Special) to rtexit2.o(.ARM.Collect$$rtexit$$00000004) for __rt_exit_exit
    rtexit.o(.ARM.Collect$$rtexit$$00000000) refers (Special) to rtexit2.o(.ARM.Collect$$rtexit$$00000003) for __rt_exit_ls
    rtexit.o(.ARM.Collect$$rtexit$$00000000) refers (Special) to rtexit2.o(.ARM.Collect$$rtexit$$00000002) for __rt_exit_prels_1
    rtexit.o(.ARM.exidx) refers (Special) to rtexit2.o(.ARM.Collect$$rtexit$$00000004) for __rt_exit_exit
    rtexit.o(.ARM.exidx) refers (Special) to rtexit2.o(.ARM.Collect$$rtexit$$00000003) for __rt_exit_ls
    rtexit.o(.ARM.exidx) refers (Special) to rtexit2.o(.ARM.Collect$$rtexit$$00000002) for __rt_exit_prels_1
    rtexit.o(.ARM.exidx) refers to rtexit.o(.ARM.Collect$$rtexit$$00000000) for .ARM.Collect$$rtexit$$00000000
    aeabi_ldiv0_sigfpe.o(.text) refers to rt_div0.o(.text) for __rt_div0
    _printf_intcommon.o(.text) refers (Weak) to _printf_pad.o(.text) for _printf_pre_padding
    _printf_intcommon.o(.text) refers (Weak) to _printf_pad.o(.text) for _printf_pre_padding
    _printf_intcommon.o(.text) refers (Weak) to _printf_pad.o(.text) for _printf_post_padding
    _printf_fp_dec.o(.text) refers (Special) to usenofp.o(x$fpl$usenofp) for __I$use$fp
    _printf_fp_dec.o(.text) refers (Special) to lc_numeric_c.o(locale$$code) for _get_lc_numeric
    _printf_fp_dec.o(.text) refers to bigflt0.o(.text) for _btod_etento
    _printf_fp_dec.o(.text) refers to btod.o(CL$$btod_d2e) for _btod_d2e
    _printf_fp_dec.o(.text) refers to btod.o(CL$$btod_ediv) for _btod_ediv
    _printf_fp_dec.o(.text) refers to btod.o(CL$$btod_emul) for _btod_emul
    _printf_fp_dec.o(.text) refers to lludiv10.o(.text) for _ll_udiv10
    _printf_fp_dec.o(.text) refers to fpclassify.o(i.__ARM_fpclassify) for __ARM_fpclassify
    _printf_fp_dec.o(.text) refers to _printf_fp_infnan.o(.text) for _printf_fp_infnan
    _printf_fp_dec.o(.text) refers (Weak) to _printf_pad.o(.text) for _printf_pre_padding
    _printf_fp_dec.o(.text) refers (Weak) to _printf_pad.o(.text) for _printf_pre_padding
    _printf_fp_dec.o(.text) refers to rt_locale_twolibspace.o(.text) for __rt_locale
    _printf_fp_dec.o(.text) refers (Weak) to _printf_pad.o(.text) for _printf_post_padding
    _printf_char_common.o(.text) refers to __printf_flags_wp.o(.text) for __printf
    _printf_char.o(.text) refers (Weak) to _printf_str.o(.text) for _printf_str
    dcmpi.o(x$fpl$dcmpinf) refers (Special) to usenofp.o(x$fpl$usenofp) for __I$use$fp
    dnaninf.o(x$fpl$dnaninf) refers (Special) to usenofp.o(x$fpl$usenofp) for __I$use$fp
    dretinf.o(x$fpl$dretinf) refers (Special) to usenofp.o(x$fpl$usenofp) for __I$use$fp
    fcmpi.o(x$fpl$fcmpinf) refers (Special) to usenofp.o(x$fpl$usenofp) for __I$use$fp
    fnaninf.o(x$fpl$fnaninf) refers (Special) to usenofp.o(x$fpl$usenofp) for __I$use$fp
    fretinf.o(x$fpl$fretinf) refers (Special) to usenofp.o(x$fpl$usenofp) for __I$use$fp
    __rtentry2.o(.ARM.Collect$$rtentry$$00000008) refers to boardinit2.o(.text) for _platform_post_stackheap_init
    __rtentry2.o(.ARM.Collect$$rtentry$$0000000A) refers to libinit.o(.ARM.Collect$$libinit$$00000000) for __rt_lib_init
    __rtentry2.o(.ARM.Collect$$rtentry$$0000000B) refers to rtx_conf_cm.o(.emb_text) for _platform_post_lib_init
    __rtentry2.o(.ARM.Collect$$rtentry$$0000000D) refers to moisture.o(i.main) for main
    __rtentry2.o(.ARM.Collect$$rtentry$$0000000D) refers to exit.o(.text) for exit
    __rtentry2.o(.ARM.exidx) refers to __rtentry2.o(.ARM.Collect$$rtentry$$00000001) for .ARM.Collect$$rtentry$$00000001
    __rtentry2.o(.ARM.exidx) refers to __rtentry2.o(.ARM.Collect$$rtentry$$00000008) for .ARM.Collect$$rtentry$$00000008
    __rtentry2.o(.ARM.exidx) refers to __rtentry2.o(.ARM.Collect$$rtentry$$0000000A) for .ARM.Collect$$rtentry$$0000000A
    __rtentry2.o(.ARM.exidx) refers to __rtentry2.o(.ARM.Collect$$rtentry$$0000000B) for .ARM.Collect$$rtentry$$0000000B
    __rtentry2.o(.ARM.exidx) refers to __rtentry2.o(.ARM.Collect$$rtentry$$0000000D) for .ARM.Collect$$rtentry$$0000000D
    __rtentry4.o(.ARM.Collect$$rtentry$$00000004) refers to sys_stackheap_outer.o(.text) for __user_setup_stackheap
    __rtentry4.o(.ARM.exidx) refers to __rtentry4.o(.ARM.Collect$$rtentry$$00000004) for .ARM.Collect$$rtentry$$00000004
    rtexit2.o(.ARM.Collect$$rtexit$$00000003) refers to libshutdown.o(.ARM.Collect$$libshutdown$$00000000) for __rt_lib_shutdown
    rtexit2.o(.ARM.Collect$$rtexit$$00000004) refers to sys_exit.o(.text) for _sys_exit
    rtexit2.o(.ARM.exidx) refers to rtexit2.o(.ARM.Collect$$rtexit$$00000001) for .ARM.Collect$$rtexit$$00000001
    rtexit2.o(.ARM.exidx) refers to rtexit2.o(.ARM.Collect$$rtexit$$00000003) for .ARM.Collect$$rtexit$$00000003
    rtexit2.o(.ARM.exidx) refers to rtexit2.o(.ARM.Collect$$rtexit$$00000004) for .ARM.Collect$$rtexit$$00000004
    rt_div0.o(.text) refers to defsig_fpe_outer.o(.text) for __rt_SIGFPE
    rt_locale.o(.text) refers to rt_locale.o(.bss) for __rt_locale_data
    rt_locale_intlibspace.o(.text) refers to libspace.o(.bss) for __libspace_start
    rt_locale_twolibspace.o(.text) refers to libspace.o(.text) for __user_perproc_libspace
    _printf_fp_infnan.o(.text) refers (Weak) to _printf_pad.o(.text) for _printf_pre_padding
    _printf_fp_infnan.o(.text) refers (Weak) to _printf_pad.o(.text) for _printf_post_padding
    bigflt0.o(.text) refers (Special) to usenofp.o(x$fpl$usenofp) for __I$use$fp
    bigflt0.o(.text) refers to btod.o(CL$$btod_emul) for _btod_emul
    bigflt0.o(.text) refers to btod.o(CL$$btod_ediv) for _btod_ediv
    bigflt0.o(.text) refers to bigflt0.o(.constdata) for .constdata
    bigflt0.o(.constdata) refers (Special) to usenofp.o(x$fpl$usenofp) for __I$use$fp
    btod.o(CL$$btod_d2e) refers (Special) to usenofp.o(x$fpl$usenofp) for __I$use$fp
    btod.o(CL$$btod_d2e) refers to btod.o(CL$$btod_d2e_norm_op1) for _d2e_norm_op1
    btod.o(CL$$btod_d2e_norm_op1) refers (Special) to usenofp.o(x$fpl$usenofp) for __I$use$fp
    btod.o(CL$$btod_d2e_norm_op1) refers to btod.o(CL$$btod_d2e_denorm_low) for _d2e_denorm_low
    btod.o(CL$$btod_d2e_denorm_low) refers (Special) to usenofp.o(x$fpl$usenofp) for __I$use$fp
    btod.o(CL$$btod_emul) refers (Special) to usenofp.o(x$fpl$usenofp) for __I$use$fp
    btod.o(CL$$btod_emul) refers to btod.o(CL$$btod_mult_common) for __btod_mult_common
    btod.o(CL$$btod_emul) refers to btod.o(CL$$btod_e2e) for _e2e
    btod.o(CL$$btod_ediv) refers (Special) to usenofp.o(x$fpl$usenofp) for __I$use$fp
    btod.o(CL$$btod_ediv) refers to btod.o(CL$$btod_div_common) for __btod_div_common
    btod.o(CL$$btod_ediv) refers to btod.o(CL$$btod_e2e) for _e2e
    btod.o(CL$$btod_emuld) refers (Special) to usenofp.o(x$fpl$usenofp) for __I$use$fp
    btod.o(CL$$btod_emuld) refers to btod.o(CL$$btod_mult_common) for __btod_mult_common
    btod.o(CL$$btod_emuld) refers to btod.o(CL$$btod_e2d) for _e2d
    btod.o(CL$$btod_edivd) refers (Special) to usenofp.o(x$fpl$usenofp) for __I$use$fp
    btod.o(CL$$btod_edivd) refers to btod.o(CL$$btod_div_common) for __btod_div_common
    btod.o(CL$$btod_edivd) refers to btod.o(CL$$btod_e2d) for _e2d
    btod.o(CL$$btod_e2e) refers (Special) to usenofp.o(x$fpl$usenofp) for __I$use$fp
    btod.o(CL$$btod_e2d) refers (Special) to usenofp.o(x$fpl$usenofp) for __I$use$fp
    btod.o(CL$$btod_e2d) refers to btod.o(CL$$btod_e2e) for _e2e
    btod.o(CL$$btod_mult_common) refers (Special) to usenofp.o(x$fpl$usenofp) for __I$use$fp
    btod.o(CL$$btod_div_common) refers (Special) to usenofp.o(x$fpl$usenofp) for __I$use$fp
    lc_numeric_c.o(locale$$data) refers (Special) to libinit2.o(.ARM.Collect$$libinit$$00000016) for __rt_lib_init_lc_numeric_2
    lc_numeric_c.o(locale$$code) refers (Special) to libinit2.o(.ARM.Collect$$libinit$$00000016) for __rt_lib_init_lc_numeric_2
    lc_numeric_c.o(locale$$code) refers to strcmpv7m.o(.text) for strcmp
    lc_numeric_c.o(locale$$code) refers to lc_numeric_c.o(locale$$data) for __lcnum_c_name
    istatus.o(x$fpl$ieeestatus) refers (Special) to usenofp.o(x$fpl$usenofp) for __I$use$fp
    fpclassify.o(i.__ARM_fpclassify) refers (Special) to usenofp.o(x$fpl$usenofp) for __I$use$fp
    sys_exit.o(.text) refers (Special) to use_no_semi.o(.text) for __I$use$semihosting
    sys_exit.o(.text) refers (Special) to indicate_semi.o(.text) for __semihosting_library_function
    sys_stackheap_outer.o(.text) refers to libspace.o(.text) for __user_perproc_libspace
    sys_stackheap_outer.o(.text) refers to startup_stm32f10x_md.o(.text) for __user_initial_stackheap
    defsig_fpe_outer.o(.text) refers to defsig_fpe_inner.o(.text) for __rt_SIGFPE_inner
    defsig_fpe_outer.o(.text) refers to defsig_exit.o(.text) for __sig_exit
    defsig_fpe_formal.o(.text) refers to rt_raise.o(.text) for __rt_raise
    libinit.o(.ARM.Collect$$libinit$$00000000) refers (Special) to libinit2.o(.ARM.Collect$$libinit$$0000002E) for __rt_lib_init_alloca_1
    libinit.o(.ARM.Collect$$libinit$$00000000) refers (Special) to libinit2.o(.ARM.Collect$$libinit$$0000002C) for __rt_lib_init_argv_1
    libinit.o(.ARM.Collect$$libinit$$00000000) refers (Special) to libinit2.o(.ARM.Collect$$libinit$$0000001B) for __rt_lib_init_atexit_1
    libinit.o(.ARM.Collect$$libinit$$00000000) refers (Special) to libinit2.o(.ARM.Collect$$libinit$$00000021) for __rt_lib_init_clock_1
    libinit.o(.ARM.Collect$$libinit$$00000000) refers (Special) to libinit2.o(.ARM.Collect$$libinit$$00000032) for __rt_lib_init_cpp_1
    libinit.o(.ARM.Collect$$libinit$$00000000) refers (Special) to libinit2.o(.ARM.Collect$$libinit$$00000030) for __rt_lib_init_exceptions_1
    libinit.o(.ARM.Collect$$libinit$$00000000) refers (Special) to libinit2.o(.ARM.Collect$$libinit$$00000002) for __rt_lib_init_fp_1
    libinit.o(.ARM.Collect$$libinit$$00000000) refers (Special) to libinit2.o(.ARM.Collect$$libinit$$0000001F) for __rt_lib_init_fp_trap_1
    libinit.o(.ARM.Collect$$libinit$$00000000) refers (Special) to libinit2.o(.ARM.Collect$$libinit$$00000023) for __rt_lib_init_getenv_1
    libinit.o(.ARM.Collect$$libinit$$00000000) refers (Special) to libinit2.o(.ARM.Collect$$libinit$$0000000A) for __rt_lib_init_heap_1
    libinit.o(.ARM.Collect$$libinit$$00000000) refers (Special) to libinit2.o(.ARM.Collect$$libinit$$00000011) for __rt_lib_init_lc_collate_1
    libinit.o(.ARM.Collect$$libinit$$00000000) refers (Special) to libinit2.o(.ARM.Collect$$libinit$$00000013) for __rt_lib_init_lc_ctype_1
    libinit.o(.ARM.Collect$$libinit$$00000000) refers (Special) to libinit2.o(.ARM.Collect$$libinit$$00000015) for __rt_lib_init_lc_monetary_1
    libinit.o(.ARM.Collect$$libinit$$00000000) refers (Special) to libinit2.o(.ARM.Collect$$libinit$$00000017) for __rt_lib_init_lc_numeric_1
    libinit.o(.ARM.Collect$$libinit$$00000000) refers (Special) to libinit2.o(.ARM.Collect$$libinit$$00000019) for __rt_lib_init_lc_time_1
    libinit.o(.ARM.Collect$$libinit$$00000000) refers (Special) to libinit2.o(.ARM.Collect$$libinit$$00000004) for __rt_lib_init_preinit_1
    libinit.o(.ARM.Collect$$libinit$$00000000) refers (Special) to libinit2.o(.ARM.Collect$$libinit$$0000000E) for __rt_lib_init_rand_1
    libinit.o(.ARM.Collect$$libinit$$00000000) refers (Special) to libinit2.o(.ARM.Collect$$libinit$$00000033) for __rt_lib_init_return
    libinit.o(.ARM.Collect$$libinit$$00000000) refers (Special) to libinit2.o(.ARM.Collect$$libinit$$0000001D) for __rt_lib_init_signal_1
    libinit.o(.ARM.Collect$$libinit$$00000000) refers (Special) to libinit2.o(.ARM.Collect$$libinit$$00000025) for __rt_lib_init_stdio_1
    libinit.o(.ARM.Collect$$libinit$$00000000) refers (Special) to libinit2.o(.ARM.Collect$$libinit$$0000000C) for __rt_lib_init_user_alloc_1
    libinit2.o(.ARM.Collect$$libinit$$0000000F) refers (Weak) to rt_locale_twolibspace.o(.text) for __rt_locale
    libinit2.o(.ARM.Collect$$libinit$$00000010) refers to libinit2.o(.ARM.Collect$$libinit$$0000000F) for .ARM.Collect$$libinit$$0000000F
    libinit2.o(.ARM.Collect$$libinit$$00000012) refers to libinit2.o(.ARM.Collect$$libinit$$0000000F) for .ARM.Collect$$libinit$$0000000F
    libinit2.o(.ARM.Collect$$libinit$$00000014) refers to libinit2.o(.ARM.Collect$$libinit$$0000000F) for .ARM.Collect$$libinit$$0000000F
    libinit2.o(.ARM.Collect$$libinit$$00000016) refers to libinit2.o(.ARM.Collect$$libinit$$0000000F) for .ARM.Collect$$libinit$$0000000F
    libinit2.o(.ARM.Collect$$libinit$$00000016) refers (Weak) to lc_numeric_c.o(locale$$code) for _get_lc_numeric
    libinit2.o(.ARM.Collect$$libinit$$00000018) refers to libinit2.o(.ARM.Collect$$libinit$$0000000F) for .ARM.Collect$$libinit$$0000000F
    libinit2.o(.ARM.Collect$$libinit$$00000026) refers to argv_veneer.o(.emb_text) for __ARM_argv_veneer
    libinit2.o(.ARM.Collect$$libinit$$00000027) refers to argv_veneer.o(.emb_text) for __ARM_argv_veneer
    libshutdown.o(.ARM.Collect$$libshutdown$$00000000) refers (Special) to libshutdown2.o(.ARM.Collect$$libshutdown$$00000004) for __rt_lib_shutdown_cpp_1
    libshutdown.o(.ARM.Collect$$libshutdown$$00000000) refers (Special) to libshutdown2.o(.ARM.Collect$$libshutdown$$00000002) for __rt_lib_shutdown_fini_1
    libshutdown.o(.ARM.Collect$$libshutdown$$00000000) refers (Special) to libshutdown2.o(.ARM.Collect$$libshutdown$$00000009) for __rt_lib_shutdown_fp_trap_1
    libshutdown.o(.ARM.Collect$$libshutdown$$00000000) refers (Special) to libshutdown2.o(.ARM.Collect$$libshutdown$$00000011) for __rt_lib_shutdown_heap_1
    libshutdown.o(.ARM.Collect$$libshutdown$$00000000) refers (Special) to libshutdown2.o(.ARM.Collect$$libshutdown$$00000012) for __rt_lib_shutdown_return
    libshutdown.o(.ARM.Collect$$libshutdown$$00000000) refers (Special) to libshutdown2.o(.ARM.Collect$$libshutdown$$0000000C) for __rt_lib_shutdown_signal_1
    libshutdown.o(.ARM.Collect$$libshutdown$$00000000) refers (Special) to libshutdown2.o(.ARM.Collect$$libshutdown$$00000006) for __rt_lib_shutdown_stdio_1
    libshutdown.o(.ARM.Collect$$libshutdown$$00000000) refers (Special) to libshutdown2.o(.ARM.Collect$$libshutdown$$0000000E) for __rt_lib_shutdown_user_alloc_1
    rt_raise.o(.text) refers to __raise.o(.text) for __raise
    rt_raise.o(.text) refers to sys_exit.o(.text) for _sys_exit
    defsig_exit.o(.text) refers to sys_exit.o(.text) for _sys_exit
    defsig_fpe_inner.o(.text) refers to defsig_general.o(.text) for __default_signal_display
    argv_veneer.o(.emb_text) refers to no_argv.o(.text) for __ARM_get_argv
    __raise.o(.text) refers to defsig.o(CL$$defsig) for __default_signal_handler
    defsig_general.o(.text) refers to sys_wrch.o(.text) for _ttywrch
    _get_argv_nomalloc.o(.text) refers (Special) to hrguard.o(.text) for __heap_region$guard
    _get_argv_nomalloc.o(.text) refers to defsig_rtmem_outer.o(.text) for __rt_SIGRTMEM
    _get_argv_nomalloc.o(.text) refers to sys_command.o(.text) for _sys_command_string
    sys_wrch.o(.text) refers (Special) to use_no_semi.o(.text) for __I$use$semihosting
    sys_wrch.o(.text) refers (Special) to indicate_semi.o(.text) for __semihosting_library_function
    sys_command.o(.text) refers (Special) to use_no_semi.o(.text) for __I$use$semihosting
    sys_command.o(.text) refers (Special) to indicate_semi.o(.text) for __semihosting_library_function
    defsig_rtmem_outer.o(.text) refers to defsig_rtmem_inner.o(.text) for __rt_SIGRTMEM_inner
    defsig_rtmem_outer.o(.text) refers to defsig_exit.o(.text) for __sig_exit
    defsig_rtmem_formal.o(.text) refers to rt_raise.o(.text) for __rt_raise
    defsig.o(CL$$defsig) refers to defsig_fpe_inner.o(.text) for __rt_SIGFPE_inner
    defsig.o(CL$$defsig) refers to defsig_rtmem_inner.o(.text) for __rt_SIGRTMEM_inner
    defsig_abrt_inner.o(.text) refers to defsig_general.o(.text) for __default_signal_display
    defsig_rtred_inner.o(.text) refers to defsig_general.o(.text) for __default_signal_display
    defsig_rtmem_inner.o(.text) refers to defsig_general.o(.text) for __default_signal_display
    defsig_stak_inner.o(.text) refers to defsig_general.o(.text) for __default_signal_display
    defsig_pvfn_inner.o(.text) refers to defsig_general.o(.text) for __default_signal_display
    defsig_cppl_inner.o(.text) refers to defsig_general.o(.text) for __default_signal_display
    defsig_segv_inner.o(.text) refers to defsig_general.o(.text) for __default_signal_display
    defsig_other.o(.text) refers to defsig_general.o(.text) for __default_signal_display


==============================================================================

Removing Unused input sections from the image.

    Removing bios.o(.rev16_text), (4 bytes).
    Removing bios.o(.revsh_text), (4 bytes).
    Removing bios.o(.rrx_text), (6 bytes).
    Removing bios.o(i.ADC1_Init), (112 bytes).
    Removing bios.o(i.BIOS_NVIC_Init), (40 bytes).
    Removing bios.o(i.Read_Internal_Temperature), (36 bytes).
    Removing delay.o(.rev16_text), (4 bytes).
    Removing delay.o(.revsh_text), (4 bytes).
    Removing delay.o(.rrx_text), (6 bytes).
    Removing i2c.o(.rev16_text), (4 bytes).
    Removing i2c.o(.revsh_text), (4 bytes).
    Removing i2c.o(.rrx_text), (6 bytes).
    Removing i2c.o(i.I2C_ACK), (52 bytes).
    Removing i2c.o(i.I2C_Init), (60 bytes).
    Removing i2c.o(i.I2C_NACK), (52 bytes).
    Removing i2c.o(i.I2C_ReadByte), (100 bytes).
    Removing i2c.o(i.I2C_SendByte), (92 bytes).
    Removing i2c.o(i.I2C_Start), (52 bytes).
    Removing i2c.o(i.I2C_Stop), (48 bytes).
    Removing i2c.o(i.I2C_Wait_ACK), (84 bytes).
    Removing spi.o(.rev16_text), (4 bytes).
    Removing spi.o(.revsh_text), (4 bytes).
    Removing spi.o(.rrx_text), (6 bytes).
    Removing spi.o(i.SPI2_Configuration), (8 bytes).
    Removing spi.o(i.SPI2_ReadWrite), (12 bytes).
    Removing spi.o(i.bus_SPIxPortInit), (84 bytes).
    Removing spi.o(i.bus_SPIxShift), (116 bytes).
    Removing spi.o(i.bus_SPIxShift1), (116 bytes).
    Removing usart.o(.rev16_text), (4 bytes).
    Removing usart.o(.revsh_text), (4 bytes).
    Removing usart.o(.rrx_text), (6 bytes).
    Removing usart.o(i.BIOS_USART3_Init), (160 bytes).
    Removing usart.o(i.UART3_Received), (24 bytes).
    Removing usart.o(i.UART3_Send), (24 bytes).
    Removing fm24.o(.rev16_text), (4 bytes).
    Removing fm24.o(.revsh_text), (4 bytes).
    Removing fm24.o(.rrx_text), (6 bytes).
    Removing cs5552.o(.rev16_text), (4 bytes).
    Removing cs5552.o(.revsh_text), (4 bytes).
    Removing cs5552.o(.rrx_text), (6 bytes).
    Removing cs5552.o(i.GET_ADC_CH0), (236 bytes).
    Removing cs5552.o(i.INIT_CS555X), (200 bytes).
    Removing cs5552.o(i.RESET_SPI), (28 bytes).
    Removing cs5552.o(i.Read_Register), (70 bytes).
    Removing cs5552.o(i.WaitForReady), (48 bytes).
    Removing cs5552.o(i.Write_Register), (50 bytes).
    Removing cs5552.o(i.bubbleSort), (70 bytes).
    Removing cs5552.o(.bss), (56 bytes).
    Removing cs5552.o(.constdata), (16 bytes).
    Removing cs5552.o(.data), (20 bytes).
    Removing ad7190.o(.rev16_text), (4 bytes).
    Removing ad7190.o(.revsh_text), (4 bytes).
    Removing ad7190.o(.rrx_text), (6 bytes).
    Removing ws100t10.o(.rev16_text), (4 bytes).
    Removing ws100t10.o(.revsh_text), (4 bytes).
    Removing ws100t10.o(.rrx_text), (6 bytes).
    Removing ws100t10.o(i.Pump_GetOutput), (28 bytes).
    Removing max6675.o(.rev16_text), (4 bytes).
    Removing max6675.o(.revsh_text), (4 bytes).
    Removing max6675.o(.rrx_text), (6 bytes).
    Removing usarthmi.o(.rev16_text), (4 bytes).
    Removing usarthmi.o(.revsh_text), (4 bytes).
    Removing usarthmi.o(.rrx_text), (6 bytes).
    Removing moisture.o(.rev16_text), (4 bytes).
    Removing moisture.o(.revsh_text), (4 bytes).
    Removing moisture.o(.rrx_text), (6 bytes).
    Removing hmi.o(.rev16_text), (4 bytes).
    Removing hmi.o(.revsh_text), (4 bytes).
    Removing hmi.o(.rrx_text), (6 bytes).
    Removing rtx_conf_cm.o(i.__user_perthread_libspace), (44 bytes).
    Removing rtx_conf_cm.o(i._mutex_initialize), (44 bytes).
    Removing misc.o(.rev16_text), (4 bytes).
    Removing misc.o(.revsh_text), (4 bytes).
    Removing misc.o(.rrx_text), (6 bytes).
    Removing misc.o(i.NVIC_Init), (112 bytes).
    Removing misc.o(i.NVIC_PriorityGroupConfig), (20 bytes).
    Removing misc.o(i.NVIC_SetVectorTable), (20 bytes).
    Removing misc.o(i.NVIC_SystemLPConfig), (32 bytes).
    Removing misc.o(i.SysTick_CLKSourceConfig), (40 bytes).
    Removing stm32f10x_adc.o(.rev16_text), (4 bytes).
    Removing stm32f10x_adc.o(.revsh_text), (4 bytes).
    Removing stm32f10x_adc.o(.rrx_text), (6 bytes).
    Removing stm32f10x_adc.o(i.ADC_AnalogWatchdogCmd), (20 bytes).
    Removing stm32f10x_adc.o(i.ADC_AnalogWatchdogSingleChannelConfig), (16 bytes).
    Removing stm32f10x_adc.o(i.ADC_AnalogWatchdogThresholdsConfig), (6 bytes).
    Removing stm32f10x_adc.o(i.ADC_AutoInjectedConvCmd), (22 bytes).
    Removing stm32f10x_adc.o(i.ADC_ClearFlag), (6 bytes).
    Removing stm32f10x_adc.o(i.ADC_ClearITPendingBit), (10 bytes).
    Removing stm32f10x_adc.o(i.ADC_Cmd), (22 bytes).
    Removing stm32f10x_adc.o(i.ADC_DMACmd), (22 bytes).
    Removing stm32f10x_adc.o(i.ADC_DeInit), (92 bytes).
    Removing stm32f10x_adc.o(i.ADC_DiscModeChannelCountConfig), (24 bytes).
    Removing stm32f10x_adc.o(i.ADC_DiscModeCmd), (22 bytes).
    Removing stm32f10x_adc.o(i.ADC_ExternalTrigConvCmd), (22 bytes).
    Removing stm32f10x_adc.o(i.ADC_ExternalTrigInjectedConvCmd), (22 bytes).
    Removing stm32f10x_adc.o(i.ADC_ExternalTrigInjectedConvConfig), (16 bytes).
    Removing stm32f10x_adc.o(i.ADC_GetCalibrationStatus), (20 bytes).
    Removing stm32f10x_adc.o(i.ADC_GetConversionValue), (8 bytes).
    Removing stm32f10x_adc.o(i.ADC_GetDualModeConversionValue), (12 bytes).
    Removing stm32f10x_adc.o(i.ADC_GetFlagStatus), (18 bytes).
    Removing stm32f10x_adc.o(i.ADC_GetITStatus), (36 bytes).
    Removing stm32f10x_adc.o(i.ADC_GetInjectedConversionValue), (28 bytes).
    Removing stm32f10x_adc.o(i.ADC_GetResetCalibrationStatus), (20 bytes).
    Removing stm32f10x_adc.o(i.ADC_GetSoftwareStartConvStatus), (20 bytes).
    Removing stm32f10x_adc.o(i.ADC_GetSoftwareStartInjectedConvCmdStatus), (20 bytes).
    Removing stm32f10x_adc.o(i.ADC_ITConfig), (24 bytes).
    Removing stm32f10x_adc.o(i.ADC_Init), (80 bytes).
    Removing stm32f10x_adc.o(i.ADC_InjectedChannelConfig), (130 bytes).
    Removing stm32f10x_adc.o(i.ADC_InjectedDiscModeCmd), (22 bytes).
    Removing stm32f10x_adc.o(i.ADC_InjectedSequencerLengthConfig), (24 bytes).
    Removing stm32f10x_adc.o(i.ADC_RegularChannelConfig), (184 bytes).
    Removing stm32f10x_adc.o(i.ADC_ResetCalibration), (10 bytes).
    Removing stm32f10x_adc.o(i.ADC_SetInjectedOffset), (20 bytes).
    Removing stm32f10x_adc.o(i.ADC_SoftwareStartConvCmd), (22 bytes).
    Removing stm32f10x_adc.o(i.ADC_SoftwareStartInjectedConvCmd), (22 bytes).
    Removing stm32f10x_adc.o(i.ADC_StartCalibration), (10 bytes).
    Removing stm32f10x_adc.o(i.ADC_StructInit), (18 bytes).
    Removing stm32f10x_adc.o(i.ADC_TempSensorVrefintCmd), (36 bytes).
    Removing stm32f10x_gpio.o(.rev16_text), (4 bytes).
    Removing stm32f10x_gpio.o(.revsh_text), (4 bytes).
    Removing stm32f10x_gpio.o(.rrx_text), (6 bytes).
    Removing stm32f10x_gpio.o(i.GPIO_AFIODeInit), (20 bytes).
    Removing stm32f10x_gpio.o(i.GPIO_DeInit), (200 bytes).
    Removing stm32f10x_gpio.o(i.GPIO_ETH_MediaInterfaceConfig), (12 bytes).
    Removing stm32f10x_gpio.o(i.GPIO_EXTILineConfig), (64 bytes).
    Removing stm32f10x_gpio.o(i.GPIO_EventOutputCmd), (12 bytes).
    Removing stm32f10x_gpio.o(i.GPIO_EventOutputConfig), (32 bytes).
    Removing stm32f10x_gpio.o(i.GPIO_PinLockConfig), (18 bytes).
    Removing stm32f10x_gpio.o(i.GPIO_ReadInputData), (8 bytes).
    Removing stm32f10x_gpio.o(i.GPIO_ReadOutputData), (8 bytes).
    Removing stm32f10x_gpio.o(i.GPIO_ReadOutputDataBit), (18 bytes).
    Removing stm32f10x_gpio.o(i.GPIO_StructInit), (16 bytes).
    Removing stm32f10x_gpio.o(i.GPIO_Write), (4 bytes).
    Removing stm32f10x_gpio.o(i.GPIO_WriteBit), (10 bytes).
    Removing stm32f10x_rcc.o(.rev16_text), (4 bytes).
    Removing stm32f10x_rcc.o(.revsh_text), (4 bytes).
    Removing stm32f10x_rcc.o(.rrx_text), (6 bytes).
    Removing stm32f10x_rcc.o(i.RCC_ADCCLKConfig), (24 bytes).
    Removing stm32f10x_rcc.o(i.RCC_AHBPeriphClockCmd), (32 bytes).
    Removing stm32f10x_rcc.o(i.RCC_APB1PeriphClockCmd), (32 bytes).
    Removing stm32f10x_rcc.o(i.RCC_APB1PeriphResetCmd), (32 bytes).
    Removing stm32f10x_rcc.o(i.RCC_APB2PeriphResetCmd), (32 bytes).
    Removing stm32f10x_rcc.o(i.RCC_AdjustHSICalibrationValue), (24 bytes).
    Removing stm32f10x_rcc.o(i.RCC_BackupResetCmd), (12 bytes).
    Removing stm32f10x_rcc.o(i.RCC_ClearFlag), (20 bytes).
    Removing stm32f10x_rcc.o(i.RCC_ClearITPendingBit), (12 bytes).
    Removing stm32f10x_rcc.o(i.RCC_ClockSecuritySystemCmd), (12 bytes).
    Removing stm32f10x_rcc.o(i.RCC_DeInit), (76 bytes).
    Removing stm32f10x_rcc.o(i.RCC_GetClocksFreq), (212 bytes).
    Removing stm32f10x_rcc.o(i.RCC_GetFlagStatus), (60 bytes).
    Removing stm32f10x_rcc.o(i.RCC_GetITStatus), (24 bytes).
    Removing stm32f10x_rcc.o(i.RCC_GetSYSCLKSource), (16 bytes).
    Removing stm32f10x_rcc.o(i.RCC_HCLKConfig), (24 bytes).
    Removing stm32f10x_rcc.o(i.RCC_HSEConfig), (76 bytes).
    Removing stm32f10x_rcc.o(i.RCC_HSICmd), (12 bytes).
    Removing stm32f10x_rcc.o(i.RCC_ITConfig), (32 bytes).
    Removing stm32f10x_rcc.o(i.RCC_LSEConfig), (52 bytes).
    Removing stm32f10x_rcc.o(i.RCC_LSICmd), (12 bytes).
    Removing stm32f10x_rcc.o(i.RCC_MCOConfig), (12 bytes).
    Removing stm32f10x_rcc.o(i.RCC_PCLK1Config), (24 bytes).
    Removing stm32f10x_rcc.o(i.RCC_PCLK2Config), (24 bytes).
    Removing stm32f10x_rcc.o(i.RCC_PLLCmd), (12 bytes).
    Removing stm32f10x_rcc.o(i.RCC_PLLConfig), (28 bytes).
    Removing stm32f10x_rcc.o(i.RCC_RTCCLKCmd), (12 bytes).
    Removing stm32f10x_rcc.o(i.RCC_RTCCLKConfig), (16 bytes).
    Removing stm32f10x_rcc.o(i.RCC_SYSCLKConfig), (24 bytes).
    Removing stm32f10x_rcc.o(i.RCC_USBCLKConfig), (12 bytes).
    Removing stm32f10x_rcc.o(i.RCC_WaitForHSEStartUp), (56 bytes).
    Removing stm32f10x_rcc.o(.data), (20 bytes).
    Removing stm32f10x_spi.o(.rev16_text), (4 bytes).
    Removing stm32f10x_spi.o(.revsh_text), (4 bytes).
    Removing stm32f10x_spi.o(.rrx_text), (6 bytes).
    Removing stm32f10x_spi.o(i.I2S_Cmd), (24 bytes).
    Removing stm32f10x_spi.o(i.I2S_Init), (232 bytes).
    Removing stm32f10x_spi.o(i.I2S_StructInit), (20 bytes).
    Removing stm32f10x_spi.o(i.SPI_BiDirectionalLineConfig), (28 bytes).
    Removing stm32f10x_spi.o(i.SPI_CalculateCRC), (24 bytes).
    Removing stm32f10x_spi.o(i.SPI_DataSizeConfig), (18 bytes).
    Removing stm32f10x_spi.o(i.SPI_GetCRC), (16 bytes).
    Removing stm32f10x_spi.o(i.SPI_GetCRCPolynomial), (6 bytes).
    Removing stm32f10x_spi.o(i.SPI_I2S_ClearFlag), (6 bytes).
    Removing stm32f10x_spi.o(i.SPI_I2S_ClearITPendingBit), (20 bytes).
    Removing stm32f10x_spi.o(i.SPI_I2S_DMACmd), (18 bytes).
    Removing stm32f10x_spi.o(i.SPI_I2S_DeInit), (88 bytes).
    Removing stm32f10x_spi.o(i.SPI_I2S_GetITStatus), (52 bytes).
    Removing stm32f10x_spi.o(i.SPI_I2S_ITConfig), (32 bytes).
    Removing stm32f10x_spi.o(i.SPI_NSSInternalSoftwareConfig), (30 bytes).
    Removing stm32f10x_spi.o(i.SPI_SSOutputCmd), (24 bytes).
    Removing stm32f10x_spi.o(i.SPI_StructInit), (24 bytes).
    Removing stm32f10x_spi.o(i.SPI_TransmitCRC), (10 bytes).
    Removing stm32f10x_tim.o(.rev16_text), (4 bytes).
    Removing stm32f10x_tim.o(.revsh_text), (4 bytes).
    Removing stm32f10x_tim.o(.rrx_text), (6 bytes).
    Removing stm32f10x_tim.o(i.TI1_Config), (128 bytes).
    Removing stm32f10x_tim.o(i.TI2_Config), (152 bytes).
    Removing stm32f10x_tim.o(i.TI3_Config), (144 bytes).
    Removing stm32f10x_tim.o(i.TI4_Config), (152 bytes).
    Removing stm32f10x_tim.o(i.TIM_ARRPreloadConfig), (24 bytes).
    Removing stm32f10x_tim.o(i.TIM_BDTRConfig), (32 bytes).
    Removing stm32f10x_tim.o(i.TIM_BDTRStructInit), (18 bytes).
    Removing stm32f10x_tim.o(i.TIM_CCPreloadControl), (24 bytes).
    Removing stm32f10x_tim.o(i.TIM_CCxCmd), (30 bytes).
    Removing stm32f10x_tim.o(i.TIM_CCxNCmd), (30 bytes).
    Removing stm32f10x_tim.o(i.TIM_ClearFlag), (6 bytes).
    Removing stm32f10x_tim.o(i.TIM_ClearITPendingBit), (6 bytes).
    Removing stm32f10x_tim.o(i.TIM_ClearOC1Ref), (18 bytes).
    Removing stm32f10x_tim.o(i.TIM_ClearOC2Ref), (24 bytes).
    Removing stm32f10x_tim.o(i.TIM_ClearOC3Ref), (18 bytes).
    Removing stm32f10x_tim.o(i.TIM_ClearOC4Ref), (24 bytes).
    Removing stm32f10x_tim.o(i.TIM_Cmd), (24 bytes).
    Removing stm32f10x_tim.o(i.TIM_CounterModeConfig), (18 bytes).
    Removing stm32f10x_tim.o(i.TIM_CtrlPWMOutputs), (30 bytes).
    Removing stm32f10x_tim.o(i.TIM_DMACmd), (18 bytes).
    Removing stm32f10x_tim.o(i.TIM_DMAConfig), (10 bytes).
    Removing stm32f10x_tim.o(i.TIM_DeInit), (488 bytes).
    Removing stm32f10x_tim.o(i.TIM_ETRClockMode1Config), (54 bytes).
    Removing stm32f10x_tim.o(i.TIM_ETRClockMode2Config), (32 bytes).
    Removing stm32f10x_tim.o(i.TIM_ETRConfig), (28 bytes).
    Removing stm32f10x_tim.o(i.TIM_EncoderInterfaceConfig), (66 bytes).
    Removing stm32f10x_tim.o(i.TIM_ForcedOC1Config), (18 bytes).
    Removing stm32f10x_tim.o(i.TIM_ForcedOC2Config), (26 bytes).
    Removing stm32f10x_tim.o(i.TIM_ForcedOC3Config), (18 bytes).
    Removing stm32f10x_tim.o(i.TIM_ForcedOC4Config), (26 bytes).
    Removing stm32f10x_tim.o(i.TIM_GenerateEvent), (4 bytes).
    Removing stm32f10x_tim.o(i.TIM_GetCapture1), (6 bytes).
    Removing stm32f10x_tim.o(i.TIM_GetCapture2), (6 bytes).
    Removing stm32f10x_tim.o(i.TIM_GetCapture3), (6 bytes).
    Removing stm32f10x_tim.o(i.TIM_GetCapture4), (8 bytes).
    Removing stm32f10x_tim.o(i.TIM_GetCounter), (6 bytes).
    Removing stm32f10x_tim.o(i.TIM_GetFlagStatus), (18 bytes).
    Removing stm32f10x_tim.o(i.TIM_GetITStatus), (34 bytes).
    Removing stm32f10x_tim.o(i.TIM_GetPrescaler), (6 bytes).
    Removing stm32f10x_tim.o(i.TIM_ICInit), (172 bytes).
    Removing stm32f10x_tim.o(i.TIM_ICStructInit), (18 bytes).
    Removing stm32f10x_tim.o(i.TIM_ITConfig), (18 bytes).
    Removing stm32f10x_tim.o(i.TIM_ITRxExternalClockConfig), (24 bytes).
    Removing stm32f10x_tim.o(i.TIM_InternalClockConfig), (12 bytes).
    Removing stm32f10x_tim.o(i.TIM_OC1FastConfig), (18 bytes).
    Removing stm32f10x_tim.o(i.TIM_OC1Init), (152 bytes).
    Removing stm32f10x_tim.o(i.TIM_OC1NPolarityConfig), (18 bytes).
    Removing stm32f10x_tim.o(i.TIM_OC1PolarityConfig), (18 bytes).
    Removing stm32f10x_tim.o(i.TIM_OC1PreloadConfig), (18 bytes).
    Removing stm32f10x_tim.o(i.TIM_OC2FastConfig), (26 bytes).
    Removing stm32f10x_tim.o(i.TIM_OC2Init), (164 bytes).
    Removing stm32f10x_tim.o(i.TIM_OC2NPolarityConfig), (26 bytes).
    Removing stm32f10x_tim.o(i.TIM_OC2PolarityConfig), (26 bytes).
    Removing stm32f10x_tim.o(i.TIM_OC2PreloadConfig), (26 bytes).
    Removing stm32f10x_tim.o(i.TIM_OC3FastConfig), (18 bytes).
    Removing stm32f10x_tim.o(i.TIM_OC3Init), (160 bytes).
    Removing stm32f10x_tim.o(i.TIM_OC3NPolarityConfig), (26 bytes).
    Removing stm32f10x_tim.o(i.TIM_OC3PolarityConfig), (26 bytes).
    Removing stm32f10x_tim.o(i.TIM_OC3PreloadConfig), (18 bytes).
    Removing stm32f10x_tim.o(i.TIM_OC4FastConfig), (26 bytes).
    Removing stm32f10x_tim.o(i.TIM_OC4Init), (124 bytes).
    Removing stm32f10x_tim.o(i.TIM_OC4PolarityConfig), (26 bytes).
    Removing stm32f10x_tim.o(i.TIM_OC4PreloadConfig), (26 bytes).
    Removing stm32f10x_tim.o(i.TIM_OCStructInit), (20 bytes).
    Removing stm32f10x_tim.o(i.TIM_PWMIConfig), (124 bytes).
    Removing stm32f10x_tim.o(i.TIM_PrescalerConfig), (6 bytes).
    Removing stm32f10x_tim.o(i.TIM_SelectCCDMA), (24 bytes).
    Removing stm32f10x_tim.o(i.TIM_SelectCOM), (24 bytes).
    Removing stm32f10x_tim.o(i.TIM_SelectHallSensor), (24 bytes).
    Removing stm32f10x_tim.o(i.TIM_SelectInputTrigger), (18 bytes).
    Removing stm32f10x_tim.o(i.TIM_SelectMasterSlaveMode), (18 bytes).
    Removing stm32f10x_tim.o(i.TIM_SelectOCxM), (82 bytes).
    Removing stm32f10x_tim.o(i.TIM_SelectOnePulseMode), (18 bytes).
    Removing stm32f10x_tim.o(i.TIM_SelectOutputTrigger), (18 bytes).
    Removing stm32f10x_tim.o(i.TIM_SelectSlaveMode), (18 bytes).
    Removing stm32f10x_tim.o(i.TIM_SetAutoreload), (4 bytes).
    Removing stm32f10x_tim.o(i.TIM_SetClockDivision), (18 bytes).
    Removing stm32f10x_tim.o(i.TIM_SetCompare1), (4 bytes).
    Removing stm32f10x_tim.o(i.TIM_SetCompare2), (4 bytes).
    Removing stm32f10x_tim.o(i.TIM_SetCompare3), (4 bytes).
    Removing stm32f10x_tim.o(i.TIM_SetCompare4), (6 bytes).
    Removing stm32f10x_tim.o(i.TIM_SetCounter), (4 bytes).
    Removing stm32f10x_tim.o(i.TIM_SetIC1Prescaler), (18 bytes).
    Removing stm32f10x_tim.o(i.TIM_SetIC2Prescaler), (26 bytes).
    Removing stm32f10x_tim.o(i.TIM_SetIC3Prescaler), (18 bytes).
    Removing stm32f10x_tim.o(i.TIM_SetIC4Prescaler), (26 bytes).
    Removing stm32f10x_tim.o(i.TIM_TIxExternalClockConfig), (62 bytes).
    Removing stm32f10x_tim.o(i.TIM_TimeBaseInit), (164 bytes).
    Removing stm32f10x_tim.o(i.TIM_TimeBaseStructInit), (18 bytes).
    Removing stm32f10x_tim.o(i.TIM_UpdateDisableConfig), (24 bytes).
    Removing stm32f10x_tim.o(i.TIM_UpdateRequestConfig), (24 bytes).
    Removing stm32f10x_usart.o(.rev16_text), (4 bytes).
    Removing stm32f10x_usart.o(.revsh_text), (4 bytes).
    Removing stm32f10x_usart.o(.rrx_text), (6 bytes).
    Removing stm32f10x_usart.o(i.USART_ClearFlag), (18 bytes).
    Removing stm32f10x_usart.o(i.USART_ClearITPendingBit), (30 bytes).
    Removing stm32f10x_usart.o(i.USART_ClockInit), (34 bytes).
    Removing stm32f10x_usart.o(i.USART_ClockStructInit), (12 bytes).
    Removing stm32f10x_usart.o(i.USART_Cmd), (24 bytes).
    Removing stm32f10x_usart.o(i.USART_DMACmd), (18 bytes).
    Removing stm32f10x_usart.o(i.USART_DeInit), (156 bytes).
    Removing stm32f10x_usart.o(i.USART_GetFlagStatus), (26 bytes).
    Removing stm32f10x_usart.o(i.USART_GetITStatus), (84 bytes).
    Removing stm32f10x_usart.o(i.USART_HalfDuplexCmd), (24 bytes).
    Removing stm32f10x_usart.o(i.USART_Init), (216 bytes).
    Removing stm32f10x_usart.o(i.USART_IrDACmd), (24 bytes).
    Removing stm32f10x_usart.o(i.USART_IrDAConfig), (18 bytes).
    Removing stm32f10x_usart.o(i.USART_LINBreakDetectLengthConfig), (18 bytes).
    Removing stm32f10x_usart.o(i.USART_LINCmd), (24 bytes).
    Removing stm32f10x_usart.o(i.USART_OneBitMethodCmd), (24 bytes).
    Removing stm32f10x_usart.o(i.USART_OverSampling8Cmd), (22 bytes).
    Removing stm32f10x_usart.o(i.USART_ReceiveData), (10 bytes).
    Removing stm32f10x_usart.o(i.USART_ReceiverWakeUpCmd), (24 bytes).
    Removing stm32f10x_usart.o(i.USART_SendBreak), (10 bytes).
    Removing stm32f10x_usart.o(i.USART_SendData), (8 bytes).
    Removing stm32f10x_usart.o(i.USART_SetAddress), (18 bytes).
    Removing stm32f10x_usart.o(i.USART_SetGuardTime), (16 bytes).
    Removing stm32f10x_usart.o(i.USART_SetPrescaler), (16 bytes).
    Removing stm32f10x_usart.o(i.USART_SmartCardCmd), (24 bytes).
    Removing stm32f10x_usart.o(i.USART_SmartCardNACKCmd), (24 bytes).
    Removing stm32f10x_usart.o(i.USART_StructInit), (24 bytes).
    Removing stm32f10x_usart.o(i.USART_WakeUpConfig), (18 bytes).
    Removing system_stm32f10x.o(.rev16_text), (4 bytes).
    Removing system_stm32f10x.o(.revsh_text), (4 bytes).
    Removing system_stm32f10x.o(.rrx_text), (6 bytes).
    Removing system_stm32f10x.o(i.SystemCoreClockUpdate), (164 bytes).
    Removing rt_cmsis.o(.rev16_text), (4 bytes).
    Removing rt_cmsis.o(.revsh_text), (4 bytes).
    Removing rt_cmsis.o(.rrx_text), (6 bytes).
    Removing rt_cmsis.o(i.isrMessageGet), (42 bytes).
    Removing rt_cmsis.o(i.isrSignalSet), (36 bytes).
    Removing rt_cmsis.o(i.osKernelRunning), (36 bytes).
    Removing rt_cmsis.o(i.osMailAlloc), (28 bytes).
    Removing rt_cmsis.o(i.osMailCAlloc), (48 bytes).
    Removing rt_cmsis.o(i.osMailCreate), (44 bytes).
    Removing rt_cmsis.o(i.osMailFree), (28 bytes).
    Removing rt_cmsis.o(i.osMailGet), (22 bytes).
    Removing rt_cmsis.o(i.osMailPut), (20 bytes).
    Removing rt_cmsis.o(i.osMessageCreate), (44 bytes).
    Removing rt_cmsis.o(i.osMessageGet), (24 bytes).
    Removing rt_cmsis.o(i.osMessagePut), (24 bytes).
    Removing rt_cmsis.o(i.osMutexDelete), (24 bytes).
    Removing rt_cmsis.o(i.osPoolAlloc), (32 bytes).
    Removing rt_cmsis.o(i.osPoolCAlloc), (52 bytes).
    Removing rt_cmsis.o(i.osPoolCreate), (44 bytes).
    Removing rt_cmsis.o(i.osPoolFree), (32 bytes).
    Removing rt_cmsis.o(i.osSemaphoreDelete), (24 bytes).
    Removing rt_cmsis.o(i.osSignalClear), (24 bytes).
    Removing rt_cmsis.o(i.osSignalSet), (24 bytes).
    Removing rt_cmsis.o(i.osSignalWait), (24 bytes).
    Removing rt_cmsis.o(i.osThreadGetPriority), (24 bytes).
    Removing rt_cmsis.o(i.osThreadSetPriority), (24 bytes).
    Removing rt_cmsis.o(i.osThreadYield), (24 bytes).
    Removing rt_cmsis.o(i.osTimerCall), (12 bytes).
    Removing rt_cmsis.o(i.osTimerCreate), (44 bytes).
    Removing rt_cmsis.o(i.osTimerDelete), (24 bytes).
    Removing rt_cmsis.o(i.osTimerStart), (24 bytes).
    Removing rt_cmsis.o(i.osTimerStop), (24 bytes).
    Removing rt_cmsis.o(i.osTimerThread), (44 bytes).
    Removing rt_cmsis.o(i.osWait), (4 bytes).
    Removing rt_cmsis.o(i.os_resume), (12 bytes).
    Removing rt_cmsis.o(i.os_suspend), (12 bytes).
    Removing rt_cmsis.o(i.rt_clr_box), (24 bytes).
    Removing rt_cmsis.o(i.rt_timer_remove), (60 bytes).
    Removing rt_cmsis.o(i.svcKernelRunning), (12 bytes).
    Removing rt_cmsis.o(i.svcMailCreate), (66 bytes).
    Removing rt_cmsis.o(i.svcMessageGet), (58 bytes).
    Removing rt_cmsis.o(i.svcMessagePut), (54 bytes).
    Removing rt_cmsis.o(i.svcMutexDelete), (26 bytes).
    Removing rt_cmsis.o(i.svcPoolCreate), (40 bytes).
    Removing rt_cmsis.o(i.svcSemaphoreDelete), (26 bytes).
    Removing rt_cmsis.o(i.svcSignalClear), (36 bytes).
    Removing rt_cmsis.o(i.svcSignalSet), (36 bytes).
    Removing rt_cmsis.o(i.svcSignalWait), (84 bytes).
    Removing rt_cmsis.o(i.svcThreadGetPriority), (18 bytes).
    Removing rt_cmsis.o(i.svcThreadSetPriority), (46 bytes).
    Removing rt_cmsis.o(i.svcThreadYield), (10 bytes).
    Removing rt_cmsis.o(i.svcTimerCall), (24 bytes).
    Removing rt_cmsis.o(i.svcTimerCreate), (56 bytes).
    Removing rt_cmsis.o(i.svcTimerDelete), (40 bytes).
    Removing rt_cmsis.o(i.svcTimerStart), (100 bytes).
    Removing rt_cmsis.o(i.svcTimerStop), (36 bytes).
    Removing rt_cmsis.o(i.sysMailAlloc), (88 bytes).
    Removing rt_cmsis.o(i.sysMailFree), (96 bytes).
    Removing rt_cmsis.o(i.sysPoolAlloc), (10 bytes).
    Removing rt_cmsis.o(i.sysPoolFree), (20 bytes).
    Removing rt_cmsis.o(i.sysUserTimerUpdate), (48 bytes).
    Removing rt_cmsis.o(i.sysUserTimerWakeupTime), (20 bytes).
    Removing rt_task.o(i.rt_tsk_pass), (48 bytes).
    Removing rt_mutex.o(i.rt_mut_delete), (176 bytes).
    Removing rt_system.o(.emb_text), (0 bytes).
    Removing rt_system.o(i.rt_resume), (136 bytes).
    Removing rt_system.o(i.rt_suspend), (36 bytes).
    Removing rt_system.o(i.rt_tsk_lock), (80 bytes).
    Removing rt_system.o(i.rt_tsk_unlock), (80 bytes).
    Removing rt_event.o(i.isr_evt_set), (40 bytes).
    Removing rt_event.o(i.rt_evt_clr), (28 bytes).
    Removing rt_event.o(i.rt_evt_get), (12 bytes).
    Removing rt_event.o(i.rt_evt_set), (92 bytes).
    Removing rt_event.o(i.rt_evt_wait), (60 bytes).
    Removing rt_list.o(i.rt_get_same_rdy_prio), (36 bytes).
    Removing rt_mailbox.o(i.isr_mbx_receive), (86 bytes).
    Removing rt_mailbox.o(i.rt_mbx_send), (152 bytes).
    Removing rt_mailbox.o(i.rt_mbx_wait), (180 bytes).
    Removing rt_semaphore.o(i.rt_sem_delete), (92 bytes).
    Removing rt_time.o(i.rt_itv_set), (24 bytes).
    Removing rt_time.o(i.rt_itv_wait), (40 bytes).
    Removing rt_time.o(i.rt_time_get), (12 bytes).
    Removing rt_membox.o(i._calloc_box), (30 bytes).

402 unused section(s) (total 14416 bytes) removed from the image.

==============================================================================

Image Symbol Table

    Local Symbols

    Symbol Name                              Value     Ov Type        Size  Object(Section)

    ../clib/angel/boardlib.s                 0x00000000   Number         0  boardinit1.o ABSOLUTE
    ../clib/angel/boardlib.s                 0x00000000   Number         0  boardinit2.o ABSOLUTE
    ../clib/angel/boardlib.s                 0x00000000   Number         0  boardshut.o ABSOLUTE
    ../clib/angel/handlers.s                 0x00000000   Number         0  __scatter_zi.o ABSOLUTE
    ../clib/angel/handlers.s                 0x00000000   Number         0  __scatter_copy.o ABSOLUTE
    ../clib/angel/kernel.s                   0x00000000   Number         0  rtexit.o ABSOLUTE
    ../clib/angel/kernel.s                   0x00000000   Number         0  __rtentry2.o ABSOLUTE
    ../clib/angel/kernel.s                   0x00000000   Number         0  __rtentry.o ABSOLUTE
    ../clib/angel/kernel.s                   0x00000000   Number         0  rtexit2.o ABSOLUTE
    ../clib/angel/kernel.s                   0x00000000   Number         0  __rtentry4.o ABSOLUTE
    ../clib/angel/rt.s                       0x00000000   Number         0  rt_raise.o ABSOLUTE
    ../clib/angel/rt.s                       0x00000000   Number         0  aeabi_ldiv0_sigfpe.o ABSOLUTE
    ../clib/angel/rt.s                       0x00000000   Number         0  aeabi_ldiv0.o ABSOLUTE
    ../clib/angel/rt.s                       0x00000000   Number         0  rt_locale_twolibspace.o ABSOLUTE
    ../clib/angel/rt.s                       0x00000000   Number         0  rt_locale_intlibspace.o ABSOLUTE
    ../clib/angel/rt.s                       0x00000000   Number         0  rt_locale.o ABSOLUTE
    ../clib/angel/rt.s                       0x00000000   Number         0  rt_div0.o ABSOLUTE
    ../clib/angel/scatter.s                  0x00000000   Number         0  __scatter.o ABSOLUTE
    ../clib/angel/startup.s                  0x00000000   Number         0  __main.o ABSOLUTE
    ../clib/angel/sys.s                      0x00000000   Number         0  use_no_semi.o ABSOLUTE
    ../clib/angel/sys.s                      0x00000000   Number         0  sys_stackheap_outer.o ABSOLUTE
    ../clib/angel/sys.s                      0x00000000   Number         0  indicate_semi.o ABSOLUTE
    ../clib/angel/sys.s                      0x00000000   Number         0  libspace.o ABSOLUTE
    ../clib/angel/sysapp.c                   0x00000000   Number         0  sys_wrch.o ABSOLUTE
    ../clib/angel/sysapp.c                   0x00000000   Number         0  sys_exit.o ABSOLUTE
    ../clib/angel/sysapp.c                   0x00000000   Number         0  sys_command.o ABSOLUTE
    ../clib/armsys.c                         0x00000000   Number         0  argv_veneer.o ABSOLUTE
    ../clib/armsys.c                         0x00000000   Number         0  no_argv.o ABSOLUTE
    ../clib/armsys.c                         0x00000000   Number         0  _get_argv_nomalloc.o ABSOLUTE
    ../clib/armsys.c                         0x00000000   Number         0  argv_veneer.o ABSOLUTE
    ../clib/bigflt.c                         0x00000000   Number         0  bigflt0.o ABSOLUTE
    ../clib/btod.s                           0x00000000   Number         0  btod.o ABSOLUTE
    ../clib/heapalloc.c                      0x00000000   Number         0  hrguard.o ABSOLUTE
    ../clib/heapaux.c                        0x00000000   Number         0  heapauxi.o ABSOLUTE
    ../clib/libinit.s                        0x00000000   Number         0  libshutdown2.o ABSOLUTE
    ../clib/libinit.s                        0x00000000   Number         0  libinit2.o ABSOLUTE
    ../clib/libinit.s                        0x00000000   Number         0  libinit.o ABSOLUTE
    ../clib/libinit.s                        0x00000000   Number         0  libshutdown.o ABSOLUTE
    ../clib/locale.s                         0x00000000   Number         0  lc_numeric_c.o ABSOLUTE
    ../clib/longlong.s                       0x00000000   Number         0  lludiv10.o ABSOLUTE
    ../clib/longlong.s                       0x00000000   Number         0  lludivv7m.o ABSOLUTE
    ../clib/memcpset.s                       0x00000000   Number         0  strcmpv7m.o ABSOLUTE
    ../clib/misc.s                           0x00000000   Number         0  printf_stubs.o ABSOLUTE
    ../clib/printf.c                         0x00000000   Number         0  __2sprintf.o ABSOLUTE
    ../clib/printf.c                         0x00000000   Number         0  __printf_nopercent.o ABSOLUTE
    ../clib/printf.c                         0x00000000   Number         0  __printf_flags_ss.o ABSOLUTE
    ../clib/printf.c                         0x00000000   Number         0  _printf_fp_infnan.o ABSOLUTE
    ../clib/printf.c                         0x00000000   Number         0  noretval__2sprintf.o ABSOLUTE
    ../clib/printf.c                         0x00000000   Number         0  _printf_char.o ABSOLUTE
    ../clib/printf.c                         0x00000000   Number         0  _sputc.o ABSOLUTE
    ../clib/printf.c                         0x00000000   Number         0  __printf.o ABSOLUTE
    ../clib/printf.c                         0x00000000   Number         0  _printf_pad.o ABSOLUTE
    ../clib/printf.c                         0x00000000   Number         0  _printf_char_common.o ABSOLUTE
    ../clib/printf.c                         0x00000000   Number         0  _printf_intcommon.o ABSOLUTE
    ../clib/printf.c                         0x00000000   Number         0  __printf_ss.o ABSOLUTE
    ../clib/printf.c                         0x00000000   Number         0  __printf_wp.o ABSOLUTE
    ../clib/printf.c                         0x00000000   Number         0  __printf_flags.o ABSOLUTE
    ../clib/printf.c                         0x00000000   Number         0  __printf_flags_wp.o ABSOLUTE
    ../clib/printf.c                         0x00000000   Number         0  __printf_ss_wp.o ABSOLUTE
    ../clib/printf.c                         0x00000000   Number         0  __printf_flags_ss_wp.o ABSOLUTE
    ../clib/printf.c                         0x00000000   Number         0  _printf_dec.o ABSOLUTE
    ../clib/printf.c                         0x00000000   Number         0  _printf_str.o ABSOLUTE
    ../clib/printf.c                         0x00000000   Number         0  _printf_fp_dec.o ABSOLUTE
    ../clib/printf_percent.s                 0x00000000   Number         0  _printf_percent_end.o ABSOLUTE
    ../clib/printf_percent.s                 0x00000000   Number         0  _printf_f.o ABSOLUTE
    ../clib/printf_percent.s                 0x00000000   Number         0  _printf_s.o ABSOLUTE
    ../clib/printf_percent.s                 0x00000000   Number         0  _printf_d.o ABSOLUTE
    ../clib/printf_percent.s                 0x00000000   Number         0  _printf_percent.o ABSOLUTE
    ../clib/signal.c                         0x00000000   Number         0  __raise.o ABSOLUTE
    ../clib/signal.c                         0x00000000   Number         0  defsig_general.o ABSOLUTE
    ../clib/signal.c                         0x00000000   Number         0  defsig_rtmem_outer.o ABSOLUTE
    ../clib/signal.c                         0x00000000   Number         0  defsig_rtmem_formal.o ABSOLUTE
    ../clib/signal.c                         0x00000000   Number         0  defsig_abrt_inner.o ABSOLUTE
    ../clib/signal.c                         0x00000000   Number         0  defsig_rtred_inner.o ABSOLUTE
    ../clib/signal.c                         0x00000000   Number         0  defsig_cppl_inner.o ABSOLUTE
    ../clib/signal.c                         0x00000000   Number         0  defsig_other.o ABSOLUTE
    ../clib/signal.c                         0x00000000   Number         0  defsig_segv_inner.o ABSOLUTE
    ../clib/signal.c                         0x00000000   Number         0  defsig_fpe_inner.o ABSOLUTE
    ../clib/signal.c                         0x00000000   Number         0  defsig_exit.o ABSOLUTE
    ../clib/signal.c                         0x00000000   Number         0  defsig_pvfn_inner.o ABSOLUTE
    ../clib/signal.c                         0x00000000   Number         0  defsig_stak_inner.o ABSOLUTE
    ../clib/signal.c                         0x00000000   Number         0  defsig_rtmem_inner.o ABSOLUTE
    ../clib/signal.c                         0x00000000   Number         0  defsig_fpe_formal.o ABSOLUTE
    ../clib/signal.c                         0x00000000   Number         0  defsig_fpe_outer.o ABSOLUTE
    ../clib/signal.s                         0x00000000   Number         0  defsig.o ABSOLUTE
    ../clib/stdlib.c                         0x00000000   Number         0  exit.o ABSOLUTE
    ../clib/string.c                         0x00000000   Number         0  strlen.o ABSOLUTE
    ../clib/string.c                         0x00000000   Number         0  strcpy.o ABSOLUTE
    ../fplib/d2f.s                           0x00000000   Number         0  d2f.o ABSOLUTE
    ../fplib/dcmpi.s                         0x00000000   Number         0  dcmpi.o ABSOLUTE
    ../fplib/ddiv.s                          0x00000000   Number         0  ddiv.o ABSOLUTE
    ../fplib/dflt.s                          0x00000000   Number         0  dflt_clz.o ABSOLUTE
    ../fplib/dleqf.s                         0x00000000   Number         0  dleqf.o ABSOLUTE
    ../fplib/dmul.s                          0x00000000   Number         0  dmul.o ABSOLUTE
    ../fplib/dnaninf.s                       0x00000000   Number         0  dnaninf.o ABSOLUTE
    ../fplib/dretinf.s                       0x00000000   Number         0  dretinf.o ABSOLUTE
    ../fplib/drleqf.s                        0x00000000   Number         0  drleqf.o ABSOLUTE
    ../fplib/f2d.s                           0x00000000   Number         0  f2d.o ABSOLUTE
    ../fplib/faddsub.s                       0x00000000   Number         0  faddsub_clz.o ABSOLUTE
    ../fplib/fcmpi.s                         0x00000000   Number         0  fcmpi.o ABSOLUTE
    ../fplib/fdiv.s                          0x00000000   Number         0  fdiv.o ABSOLUTE
    ../fplib/feqf.s                          0x00000000   Number         0  feqf.o ABSOLUTE
    ../fplib/ffix.s                          0x00000000   Number         0  ffix.o ABSOLUTE
    ../fplib/ffixu.s                         0x00000000   Number         0  ffixu.o ABSOLUTE
    ../fplib/fflt.s                          0x00000000   Number         0  fflt_clz.o ABSOLUTE
    ../fplib/fleqf.s                         0x00000000   Number         0  fleqf.o ABSOLUTE
    ../fplib/fmul.s                          0x00000000   Number         0  fmul.o ABSOLUTE
    ../fplib/fnaninf.s                       0x00000000   Number         0  fnaninf.o ABSOLUTE
    ../fplib/fpinit.s                        0x00000000   Number         0  fpinit.o ABSOLUTE
    ../fplib/fretinf.s                       0x00000000   Number         0  fretinf.o ABSOLUTE
    ../fplib/frleqf.s                        0x00000000   Number         0  frleqf.o ABSOLUTE
    ../fplib/istatus.s                       0x00000000   Number         0  istatus.o ABSOLUTE
    ../fplib/printf1.s                       0x00000000   Number         0  printf1.o ABSOLUTE
    ../fplib/usenofp.s                       0x00000000   Number         0  usenofp.o ABSOLUTE
    ../mathlib/fpclassify.c                  0x00000000   Number         0  fpclassify.o ABSOLUTE
    ..\HAL_CM.c                              0x00000000   Number         0  hal_cm.o ABSOLUTE
    ..\\rt_CMSIS.c                           0x00000000   Number         0  rt_cmsis.o ABSOLUTE
    ..\\rt_System.c                          0x00000000   Number         0  rt_system.o ABSOLUTE
    ..\rt_CMSIS.c                            0x00000000   Number         0  rt_cmsis.o ABSOLUTE
    ..\rt_Event.c                            0x00000000   Number         0  rt_event.o ABSOLUTE
    ..\rt_List.c                             0x00000000   Number         0  rt_list.o ABSOLUTE
    ..\rt_Mailbox.c                          0x00000000   Number         0  rt_mailbox.o ABSOLUTE
    ..\rt_MemBox.c                           0x00000000   Number         0  rt_membox.o ABSOLUTE
    ..\rt_Memory.c                           0x00000000   Number         0  rt_memory.o ABSOLUTE
    ..\rt_Mutex.c                            0x00000000   Number         0  rt_mutex.o ABSOLUTE
    ..\rt_Robin.c                            0x00000000   Number         0  rt_robin.o ABSOLUTE
    ..\rt_Semaphore.c                        0x00000000   Number         0  rt_semaphore.o ABSOLUTE
    ..\rt_System.c                           0x00000000   Number         0  rt_system.o ABSOLUTE
    ..\rt_Task.c                             0x00000000   Number         0  rt_task.o ABSOLUTE
    ..\rt_Time.c                             0x00000000   Number         0  rt_time.o ABSOLUTE
    C:/Users/YT01/AppData/Local/Arm/Packs/Keil/STM32F1xx_DFP/2.4.1/Device/StdPeriph_Driver/src/misc.c 0x00000000   Number         0  misc.o ABSOLUTE
    C:/Users/YT01/AppData/Local/Arm/Packs/Keil/STM32F1xx_DFP/2.4.1/Device/StdPeriph_Driver/src/stm32f10x_adc.c 0x00000000   Number         0  stm32f10x_adc.o ABSOLUTE
    C:/Users/YT01/AppData/Local/Arm/Packs/Keil/STM32F1xx_DFP/2.4.1/Device/StdPeriph_Driver/src/stm32f10x_gpio.c 0x00000000   Number         0  stm32f10x_gpio.o ABSOLUTE
    C:/Users/YT01/AppData/Local/Arm/Packs/Keil/STM32F1xx_DFP/2.4.1/Device/StdPeriph_Driver/src/stm32f10x_rcc.c 0x00000000   Number         0  stm32f10x_rcc.o ABSOLUTE
    C:/Users/YT01/AppData/Local/Arm/Packs/Keil/STM32F1xx_DFP/2.4.1/Device/StdPeriph_Driver/src/stm32f10x_spi.c 0x00000000   Number         0  stm32f10x_spi.o ABSOLUTE
    C:/Users/YT01/AppData/Local/Arm/Packs/Keil/STM32F1xx_DFP/2.4.1/Device/StdPeriph_Driver/src/stm32f10x_tim.c 0x00000000   Number         0  stm32f10x_tim.o ABSOLUTE
    C:/Users/YT01/AppData/Local/Arm/Packs/Keil/STM32F1xx_DFP/2.4.1/Device/StdPeriph_Driver/src/stm32f10x_usart.c 0x00000000   Number         0  stm32f10x_usart.o ABSOLUTE
    C:\Users\YT01\AppData\Local\Arm\Packs\Keil\STM32F1xx_DFP\2.4.1\Device\StdPeriph_Driver\src\misc.c 0x00000000   Number         0  misc.o ABSOLUTE
    C:\Users\YT01\AppData\Local\Arm\Packs\Keil\STM32F1xx_DFP\2.4.1\Device\StdPeriph_Driver\src\stm32f10x_adc.c 0x00000000   Number         0  stm32f10x_adc.o ABSOLUTE
    C:\Users\YT01\AppData\Local\Arm\Packs\Keil\STM32F1xx_DFP\2.4.1\Device\StdPeriph_Driver\src\stm32f10x_gpio.c 0x00000000   Number         0  stm32f10x_gpio.o ABSOLUTE
    C:\Users\YT01\AppData\Local\Arm\Packs\Keil\STM32F1xx_DFP\2.4.1\Device\StdPeriph_Driver\src\stm32f10x_rcc.c 0x00000000   Number         0  stm32f10x_rcc.o ABSOLUTE
    C:\Users\YT01\AppData\Local\Arm\Packs\Keil\STM32F1xx_DFP\2.4.1\Device\StdPeriph_Driver\src\stm32f10x_spi.c 0x00000000   Number         0  stm32f10x_spi.o ABSOLUTE
    C:\Users\YT01\AppData\Local\Arm\Packs\Keil\STM32F1xx_DFP\2.4.1\Device\StdPeriph_Driver\src\stm32f10x_tim.c 0x00000000   Number         0  stm32f10x_tim.o ABSOLUTE
    C:\Users\YT01\AppData\Local\Arm\Packs\Keil\STM32F1xx_DFP\2.4.1\Device\StdPeriph_Driver\src\stm32f10x_usart.c 0x00000000   Number         0  stm32f10x_usart.o ABSOLUTE
    HAL_CM3.c                                0x00000000   Number         0  hal_cm3.o ABSOLUTE
    HAL_CM3.c                                0x00000000   Number         0  hal_cm3.o ABSOLUTE
    RTE/CMSIS/RTX_Conf_CM.c                  0x00000000   Number         0  rtx_conf_cm.o ABSOLUTE
    RTE/Device/STM32F103C8/startup_stm32f10x_md.s 0x00000000   Number         0  startup_stm32f10x_md.o ABSOLUTE
    RTE/Device/STM32F103C8/system_stm32f10x.c 0x00000000   Number         0  system_stm32f10x.o ABSOLUTE
    RTE\CMSIS\RTX_Conf_CM.c                  0x00000000   Number         0  rtx_conf_cm.o ABSOLUTE
    RTE\Device\STM32F103C8\system_stm32f10x.c 0x00000000   Number         0  system_stm32f10x.o ABSOLUTE
    SVC_Table.s                              0x00000000   Number         0  svc_table.o ABSOLUTE
    Source\AD7190.c                          0x00000000   Number         0  ad7190.o ABSOLUTE
    Source\BIOS.c                            0x00000000   Number         0  bios.o ABSOLUTE
    Source\CS5552.c                          0x00000000   Number         0  cs5552.o ABSOLUTE
    Source\Delay.c                           0x00000000   Number         0  delay.o ABSOLUTE
    Source\FM24.c                            0x00000000   Number         0  fm24.o ABSOLUTE
    Source\HMI.c                             0x00000000   Number         0  hmi.o ABSOLUTE
    Source\Moisture.c                        0x00000000   Number         0  moisture.o ABSOLUTE
    Source\USARTHMI.c                        0x00000000   Number         0  usarthmi.o ABSOLUTE
    Source\WS100T10.c                        0x00000000   Number         0  ws100t10.o ABSOLUTE
    Source\\AD7190.c                         0x00000000   Number         0  ad7190.o ABSOLUTE
    Source\\BIOS.c                           0x00000000   Number         0  bios.o ABSOLUTE
    Source\\CS5552.c                         0x00000000   Number         0  cs5552.o ABSOLUTE
    Source\\Delay.c                          0x00000000   Number         0  delay.o ABSOLUTE
    Source\\FM24.c                           0x00000000   Number         0  fm24.o ABSOLUTE
    Source\\HMI.c                            0x00000000   Number         0  hmi.o ABSOLUTE
    Source\\Moisture.c                       0x00000000   Number         0  moisture.o ABSOLUTE
    Source\\USARTHMI.c                       0x00000000   Number         0  usarthmi.o ABSOLUTE
    Source\\WS100T10.c                       0x00000000   Number         0  ws100t10.o ABSOLUTE
    Source\\i2c.c                            0x00000000   Number         0  i2c.o ABSOLUTE
    Source\\max6675.c                        0x00000000   Number         0  max6675.o ABSOLUTE
    Source\\spi.c                            0x00000000   Number         0  spi.o ABSOLUTE
    Source\\usart.c                          0x00000000   Number         0  usart.o ABSOLUTE
    Source\i2c.c                             0x00000000   Number         0  i2c.o ABSOLUTE
    Source\max6675.c                         0x00000000   Number         0  max6675.o ABSOLUTE
    Source\spi.c                             0x00000000   Number         0  spi.o ABSOLUTE
    Source\usart.c                           0x00000000   Number         0  usart.o ABSOLUTE
    dc.s                                     0x00000000   Number         0  dc.o ABSOLUTE
    RESET                                    0x08000000   Section      236  startup_stm32f10x_md.o(RESET)
    !!!main                                  0x080000ec   Section        8  __main.o(!!!main)
    !!!scatter                               0x080000f4   Section       52  __scatter.o(!!!scatter)
    !!handler_copy                           0x08000128   Section       26  __scatter_copy.o(!!handler_copy)
    !!handler_zi                             0x08000144   Section       28  __scatter_zi.o(!!handler_zi)
    .ARM.Collect$$_printf_percent$$00000000  0x08000160   Section        0  _printf_percent.o(.ARM.Collect$$_printf_percent$$00000000)
    .ARM.Collect$$_printf_percent$$00000003  0x08000160   Section        6  _printf_f.o(.ARM.Collect$$_printf_percent$$00000003)
    .ARM.Collect$$_printf_percent$$00000009  0x08000166   Section        6  _printf_d.o(.ARM.Collect$$_printf_percent$$00000009)
    .ARM.Collect$$_printf_percent$$00000014  0x0800016c   Section        6  _printf_s.o(.ARM.Collect$$_printf_percent$$00000014)
    .ARM.Collect$$_printf_percent$$00000017  0x08000172   Section        4  _printf_percent_end.o(.ARM.Collect$$_printf_percent$$00000017)
    .ARM.Collect$$libinit$$00000000          0x08000176   Section        2  libinit.o(.ARM.Collect$$libinit$$00000000)
    .ARM.Collect$$libinit$$00000002          0x08000178   Section        0  libinit2.o(.ARM.Collect$$libinit$$00000002)
    .ARM.Collect$$libinit$$00000004          0x08000178   Section        0  libinit2.o(.ARM.Collect$$libinit$$00000004)
    .ARM.Collect$$libinit$$0000000A          0x08000178   Section        0  libinit2.o(.ARM.Collect$$libinit$$0000000A)
    .ARM.Collect$$libinit$$0000000C          0x08000178   Section        0  libinit2.o(.ARM.Collect$$libinit$$0000000C)
    .ARM.Collect$$libinit$$0000000E          0x08000178   Section        0  libinit2.o(.ARM.Collect$$libinit$$0000000E)
    .ARM.Collect$$libinit$$0000000F          0x08000178   Section        6  libinit2.o(.ARM.Collect$$libinit$$0000000F)
    .ARM.Collect$$libinit$$00000011          0x0800017e   Section        0  libinit2.o(.ARM.Collect$$libinit$$00000011)
    .ARM.Collect$$libinit$$00000013          0x0800017e   Section        0  libinit2.o(.ARM.Collect$$libinit$$00000013)
    .ARM.Collect$$libinit$$00000015          0x0800017e   Section        0  libinit2.o(.ARM.Collect$$libinit$$00000015)
    .ARM.Collect$$libinit$$00000016          0x0800017e   Section       10  libinit2.o(.ARM.Collect$$libinit$$00000016)
    .ARM.Collect$$libinit$$00000017          0x08000188   Section        0  libinit2.o(.ARM.Collect$$libinit$$00000017)
    .ARM.Collect$$libinit$$00000019          0x08000188   Section        0  libinit2.o(.ARM.Collect$$libinit$$00000019)
    .ARM.Collect$$libinit$$0000001B          0x08000188   Section        0  libinit2.o(.ARM.Collect$$libinit$$0000001B)
    .ARM.Collect$$libinit$$0000001D          0x08000188   Section        0  libinit2.o(.ARM.Collect$$libinit$$0000001D)
    .ARM.Collect$$libinit$$0000001F          0x08000188   Section        0  libinit2.o(.ARM.Collect$$libinit$$0000001F)
    .ARM.Collect$$libinit$$00000021          0x08000188   Section        0  libinit2.o(.ARM.Collect$$libinit$$00000021)
    .ARM.Collect$$libinit$$00000023          0x08000188   Section        0  libinit2.o(.ARM.Collect$$libinit$$00000023)
    .ARM.Collect$$libinit$$00000025          0x08000188   Section        0  libinit2.o(.ARM.Collect$$libinit$$00000025)
    .ARM.Collect$$libinit$$0000002C          0x08000188   Section        0  libinit2.o(.ARM.Collect$$libinit$$0000002C)
    .ARM.Collect$$libinit$$0000002E          0x08000188   Section        0  libinit2.o(.ARM.Collect$$libinit$$0000002E)
    .ARM.Collect$$libinit$$00000030          0x08000188   Section        0  libinit2.o(.ARM.Collect$$libinit$$00000030)
    .ARM.Collect$$libinit$$00000032          0x08000188   Section        0  libinit2.o(.ARM.Collect$$libinit$$00000032)
    .ARM.Collect$$libinit$$00000033          0x08000188   Section        2  libinit2.o(.ARM.Collect$$libinit$$00000033)
    .ARM.Collect$$libshutdown$$00000000      0x0800018a   Section        2  libshutdown.o(.ARM.Collect$$libshutdown$$00000000)
    .ARM.Collect$$libshutdown$$00000002      0x0800018c   Section        0  libshutdown2.o(.ARM.Collect$$libshutdown$$00000002)
    .ARM.Collect$$libshutdown$$00000004      0x0800018c   Section        0  libshutdown2.o(.ARM.Collect$$libshutdown$$00000004)
    .ARM.Collect$$libshutdown$$00000006      0x0800018c   Section        0  libshutdown2.o(.ARM.Collect$$libshutdown$$00000006)
    .ARM.Collect$$libshutdown$$00000009      0x0800018c   Section        0  libshutdown2.o(.ARM.Collect$$libshutdown$$00000009)
    .ARM.Collect$$libshutdown$$0000000C      0x0800018c   Section        0  libshutdown2.o(.ARM.Collect$$libshutdown$$0000000C)
    .ARM.Collect$$libshutdown$$0000000E      0x0800018c   Section        0  libshutdown2.o(.ARM.Collect$$libshutdown$$0000000E)
    .ARM.Collect$$libshutdown$$00000011      0x0800018c   Section        0  libshutdown2.o(.ARM.Collect$$libshutdown$$00000011)
    .ARM.Collect$$libshutdown$$00000012      0x0800018c   Section        2  libshutdown2.o(.ARM.Collect$$libshutdown$$00000012)
    .ARM.Collect$$rtentry$$00000000          0x0800018e   Section        0  __rtentry.o(.ARM.Collect$$rtentry$$00000000)
    .ARM.Collect$$rtentry$$00000002          0x0800018e   Section        0  __rtentry2.o(.ARM.Collect$$rtentry$$00000002)
    .ARM.Collect$$rtentry$$00000004          0x0800018e   Section        6  __rtentry4.o(.ARM.Collect$$rtentry$$00000004)
    .ARM.Collect$$rtentry$$00000009          0x08000194   Section        0  __rtentry2.o(.ARM.Collect$$rtentry$$00000009)
    .ARM.Collect$$rtentry$$0000000A          0x08000194   Section        4  __rtentry2.o(.ARM.Collect$$rtentry$$0000000A)
    .ARM.Collect$$rtentry$$0000000B          0x08000198   Section        8  __rtentry2.o(.ARM.Collect$$rtentry$$0000000B)
    .ARM.Collect$$rtentry$$0000000D          0x080001a0   Section        8  __rtentry2.o(.ARM.Collect$$rtentry$$0000000D)
    .ARM.Collect$$rtexit$$00000000           0x080001a8   Section        2  rtexit.o(.ARM.Collect$$rtexit$$00000000)
    .ARM.Collect$$rtexit$$00000002           0x080001aa   Section        0  rtexit2.o(.ARM.Collect$$rtexit$$00000002)
    .ARM.Collect$$rtexit$$00000003           0x080001aa   Section        4  rtexit2.o(.ARM.Collect$$rtexit$$00000003)
    .ARM.Collect$$rtexit$$00000004           0x080001ae   Section        6  rtexit2.o(.ARM.Collect$$rtexit$$00000004)
    .emb_text                                0x080001b4   Section       28  rtx_conf_cm.o(.emb_text)
    .emb_text                                0x080001d0   Section      304  hal_cm3.o(.emb_text)
    .text                                    0x08000300   Section       64  startup_stm32f10x_md.o(.text)
    .text                                    0x08000340   Section        8  libspace.o(.text)
    .text                                    0x08000348   Section        0  noretval__2sprintf.o(.text)
    .text                                    0x08000370   Section        0  _printf_pad.o(.text)
    .text                                    0x080003be   Section        0  _printf_str.o(.text)
    .text                                    0x08000410   Section        0  _printf_dec.o(.text)
    .text                                    0x08000488   Section        0  __printf_flags_wp.o(.text)
    .text                                    0x080005c0   Section        0  exit.o(.text)
    .text                                    0x080005d2   Section        0  strcpy.o(.text)
    .text                                    0x0800061a   Section        0  strlen.o(.text)
    .text                                    0x08000658   Section      128  strcmpv7m.o(.text)
    .text                                    0x080006d8   Section        0  heapauxi.o(.text)
    .text                                    0x080006de   Section        0  _printf_intcommon.o(.text)
    .text                                    0x08000790   Section        0  _printf_fp_dec.o(.text)
    _fp_digits                               0x08000793   Thumb Code   432  _printf_fp_dec.o(.text)
    .text                                    0x08000bb0   Section        0  _printf_char_common.o(.text)
    _printf_input_char                       0x08000bb1   Thumb Code    10  _printf_char_common.o(.text)
    .text                                    0x08000be0   Section        0  _sputc.o(.text)
    .text                                    0x08000bea   Section        0  _printf_char.o(.text)
    .text                                    0x08000c16   Section       10  rt_locale_twolibspace.o(.text)
    .text                                    0x08000c20   Section      138  lludiv10.o(.text)
    .text                                    0x08000cac   Section        0  _printf_fp_infnan.o(.text)
    .text                                    0x08000d2c   Section        0  bigflt0.o(.text)
    .text                                    0x08000e10   Section        0  sys_exit.o(.text)
    .text                                    0x08000e1c   Section       74  sys_stackheap_outer.o(.text)
    .text                                    0x08000e66   Section        2  use_no_semi.o(.text)
    .text                                    0x08000e68   Section        0  indicate_semi.o(.text)
    CL$$btod_d2e                             0x08000e68   Section       62  btod.o(CL$$btod_d2e)
    CL$$btod_d2e_denorm_low                  0x08000ea6   Section       70  btod.o(CL$$btod_d2e_denorm_low)
    CL$$btod_d2e_norm_op1                    0x08000eec   Section       96  btod.o(CL$$btod_d2e_norm_op1)
    CL$$btod_div_common                      0x08000f4c   Section      824  btod.o(CL$$btod_div_common)
    CL$$btod_e2e                             0x08001284   Section      220  btod.o(CL$$btod_e2e)
    CL$$btod_ediv                            0x08001360   Section       42  btod.o(CL$$btod_ediv)
    CL$$btod_emul                            0x0800138a   Section       42  btod.o(CL$$btod_emul)
    CL$$btod_mult_common                     0x080013b4   Section      580  btod.o(CL$$btod_mult_common)
    SVC_TABLE                                0x080015f8   Section        4  svc_table.o(SVC_TABLE)
    i.ACCMD                                  0x080015fc   Section        0  ws100t10.o(i.ACCMD)
    i.ACCtrl                                 0x08001620   Section        0  ws100t10.o(i.ACCtrl)
    i.AC_CTRL_Init                           0x08001664   Section        0  ws100t10.o(i.AC_CTRL_Init)
    i.AD7190_Init                            0x08001674   Section        0  ad7190.o(i.AD7190_Init)
    i.AD7190_ReadData                        0x0800175c   Section        0  ad7190.o(i.AD7190_ReadData)
    i.AD7190_ReadRegister                    0x0800188c   Section        0  ad7190.o(i.AD7190_ReadRegister)
    i.AD7190_ReadRegisterOnce                0x080018ba   Section        0  ad7190.o(i.AD7190_ReadRegisterOnce)
    i.AD7190_Run                             0x080018d4   Section        0  ad7190.o(i.AD7190_Run)
    i.AD7190_WaitForReady                    0x08001dd8   Section        0  ad7190.o(i.AD7190_WaitForReady)
    i.AD7190_WriteRegister                   0x08001e08   Section        0  ad7190.o(i.AD7190_WriteRegister)
    i.AD7190_WriteRegisterOnce               0x08001e2c   Section        0  ad7190.o(i.AD7190_WriteRegisterOnce)
    i.BIOS_TIM2_TIMER_Init                   0x08001e40   Section        0  usarthmi.o(i.BIOS_TIM2_TIMER_Init)
    i.BIOS_USART1_Init                       0x08001ea0   Section        0  usarthmi.o(i.BIOS_USART1_Init)
    i.BIOS_USART2_Init                       0x08001f40   Section        0  usart.o(i.BIOS_USART2_Init)
    i.DataPrint                              0x08001fac   Section        0  usarthmi.o(i.DataPrint)
    i.DataRec                                0x08001ffc   Section        0  usarthmi.o(i.DataRec)
    i.DataUnpack                             0x08002008   Section        0  hmi.o(i.DataUnpack)
    i.FM24DataCRC                            0x080035a0   Section        0  hmi.o(i.FM24DataCRC)
    i.FM24Init                               0x080036ec   Section        0  fm24.o(i.FM24Init)
    i.FM24_Read                              0x080036f4   Section        0  fm24.o(i.FM24_Read)
    i.FM24_Write                             0x08003750   Section        0  fm24.o(i.FM24_Write)
    i.GPIO_InPutset                          0x08003798   Section        0  bios.o(i.GPIO_InPutset)
    i.GPIO_Init                              0x080037c4   Section        0  stm32f10x_gpio.o(i.GPIO_Init)
    i.GPIO_PinRemapConfig                    0x080038dc   Section        0  stm32f10x_gpio.o(i.GPIO_PinRemapConfig)
    i.GPIO_ReadInputDataBit                  0x0800396c   Section        0  stm32f10x_gpio.o(i.GPIO_ReadInputDataBit)
    i.GPIO_ResetBits                         0x0800397e   Section        0  stm32f10x_gpio.o(i.GPIO_ResetBits)
    i.GPIO_SetBits                           0x08003982   Section        0  stm32f10x_gpio.o(i.GPIO_SetBits)
    i.HMICMDInit                             0x08003988   Section        0  hmi.o(i.HMICMDInit)
    i.HeatPID_Task                           0x0800399c   Section        0  ws100t10.o(i.HeatPID_Task)
    HeatPID_Task                             0x0800399d   Thumb Code   512  ws100t10.o(i.HeatPID_Task)
    i.HeatTask_Init                          0x08003be8   Section        0  ws100t10.o(i.HeatTask_Init)
    HeatTask_Init                            0x08003be9   Thumb Code    12  ws100t10.o(i.HeatTask_Init)
    i.HeatTask_Socket                        0x08003bf8   Section        0  ws100t10.o(i.HeatTask_Socket)
    HeatTask_Socket                          0x08003bf9   Thumb Code    20  ws100t10.o(i.HeatTask_Socket)
    i.I2C2_ACK                               0x08003c0c   Section        0  i2c.o(i.I2C2_ACK)
    i.I2C2_Init                              0x08003c48   Section        0  i2c.o(i.I2C2_Init)
    i.I2C2_NACK                              0x08003c88   Section        0  i2c.o(i.I2C2_NACK)
    i.I2C2_ReadByte                          0x08003cc4   Section        0  i2c.o(i.I2C2_ReadByte)
    i.I2C2_SendByte                          0x08003d28   Section        0  i2c.o(i.I2C2_SendByte)
    i.I2C2_Start                             0x08003d90   Section        0  i2c.o(i.I2C2_Start)
    i.I2C2_Stop                              0x08003dcc   Section        0  i2c.o(i.I2C2_Stop)
    i.I2C2_Wait_ACK                          0x08003e04   Section        0  i2c.o(i.I2C2_Wait_ACK)
    i.InstrumentTypeRead                     0x08003e68   Section        0  bios.o(i.InstrumentTypeRead)
    i.MAX6675_ConvertTemperature             0x08003ea8   Section        0  max6675.o(i.MAX6675_ConvertTemperature)
    i.MAX6675_Init                           0x08003f28   Section        0  max6675.o(i.MAX6675_Init)
    i.MAX6675_ReadData                       0x08003f90   Section        0  max6675.o(i.MAX6675_ReadData)
    i.Moisturing                             0x08003fe8   Section        0  hmi.o(i.Moisturing)
    i.MoisturingRun                          0x08005300   Section        0  hmi.o(i.MoisturingRun)
    i.Pump_OutCmd                            0x08005310   Section        0  ws100t10.o(i.Pump_OutCmd)
    i.RCC_APB2PeriphClockCmd                 0x08005338   Section        0  stm32f10x_rcc.o(i.RCC_APB2PeriphClockCmd)
    i.SPI1_Configuration                     0x08005358   Section        0  spi.o(i.SPI1_Configuration)
    i.SPI1_ReadWrite                         0x080053dc   Section        0  spi.o(i.SPI1_ReadWrite)
    i.SPI_Cmd                                0x08005414   Section        0  stm32f10x_spi.o(i.SPI_Cmd)
    i.SPI_I2S_GetFlagStatus                  0x0800542c   Section        0  stm32f10x_spi.o(i.SPI_I2S_GetFlagStatus)
    i.SPI_I2S_ReceiveData                    0x0800543e   Section        0  stm32f10x_spi.o(i.SPI_I2S_ReceiveData)
    i.SPI_I2S_SendData                       0x08005444   Section        0  stm32f10x_spi.o(i.SPI_I2S_SendData)
    i.SPI_Init                               0x08005448   Section        0  stm32f10x_spi.o(i.SPI_Init)
    i.SafeCheck                              0x08005484   Section        0  bios.o(i.SafeCheck)
    i.SetSysClock                            0x080054a0   Section        0  system_stm32f10x.o(i.SetSysClock)
    SetSysClock                              0x080054a1   Thumb Code     8  system_stm32f10x.o(i.SetSysClock)
    i.SetSysClockTo72                        0x080054a8   Section        0  system_stm32f10x.o(i.SetSysClockTo72)
    SetSysClockTo72                          0x080054a9   Thumb Code   214  system_stm32f10x.o(i.SetSysClockTo72)
    i.SystemInit                             0x08005588   Section        0  system_stm32f10x.o(i.SystemInit)
    i.TIM2_IRQHandler                        0x080055e8   Section        0  usarthmi.o(i.TIM2_IRQHandler)
    i.UART1_Received                         0x08005670   Section        0  usarthmi.o(i.UART1_Received)
    i.UART1_Send                             0x08005688   Section        0  usarthmi.o(i.UART1_Send)
    i.USART1_IRQHandler                      0x080056a8   Section        0  usarthmi.o(i.USART1_IRQHandler)
    i.USART2Print                            0x0800573c   Section        0  usart.o(i.USART2Print)
    i.USART2_Send                            0x08005770   Section        0  usart.o(i.USART2_Send)
    i.USARTHMIInit                           0x08005788   Section        0  usarthmi.o(i.USARTHMIInit)
    i.USART_ITConfig                         0x080057a8   Section        0  stm32f10x_usart.o(i.USART_ITConfig)
    i.WS100T10_Ctrl                          0x080057f4   Section        0  i2c.o(i.WS100T10_Ctrl)
    i.WS100T10_Init                          0x0800588c   Section        0  i2c.o(i.WS100T10_Init)
    i.__ARM_fpclassify                       0x08005918   Section        0  fpclassify.o(i.__ARM_fpclassify)
    i.__NVIC_EnableIRQ                       0x08005940   Section        0  usarthmi.o(i.__NVIC_EnableIRQ)
    __NVIC_EnableIRQ                         0x08005941   Thumb Code    34  usarthmi.o(i.__NVIC_EnableIRQ)
    i._init_box                              0x08005962   Section        0  rt_membox.o(i._init_box)
    i._is_digit                              0x080059a8   Section        0  __printf_wp.o(i._is_digit)
    i._mutex_acquire                         0x080059b8   Section        0  rtx_conf_cm.o(i._mutex_acquire)
    __tagsym$$used                           0x080059b9   Number         0  rtx_conf_cm.o(i._mutex_acquire)
    i._mutex_release                         0x080059d8   Section        0  rtx_conf_cm.o(i._mutex_release)
    __tagsym$$used                           0x080059d9   Number         0  rtx_conf_cm.o(i._mutex_release)
    i._task_ACCtrl                           0x080059f4   Section        0  ws100t10.o(i._task_ACCtrl)
    i.dbg_init                               0x08005a30   Section        0  hal_cm.o(i.dbg_init)
    i.dbg_task_notify                        0x08005a60   Section        0  hal_cm.o(i.dbg_task_notify)
    i.dbg_task_switch                        0x08005a80   Section        0  hal_cm.o(i.dbg_task_switch)
    i.delay_us                               0x08005a90   Section        0  delay.o(i.delay_us)
    i.isrMessagePut                          0x08005b12   Section        0  rt_cmsis.o(i.isrMessagePut)
    i.isrSemaphoreRelease                    0x08005b3e   Section        0  rt_cmsis.o(i.isrSemaphoreRelease)
    i.isr_mbx_send                           0x08005b66   Section        0  rt_mailbox.o(i.isr_mbx_send)
    i.isr_sem_send                           0x08005b74   Section        0  rt_semaphore.o(i.isr_sem_send)
    i.kalman_filter_init                     0x08005b84   Section        0  max6675.o(i.kalman_filter_init)
    i.kalman_filter_init2                    0x08005b92   Section        0  ad7190.o(i.kalman_filter_init2)
    i.kalman_filter_update                   0x08005ba0   Section        0  max6675.o(i.kalman_filter_update)
    i.kalman_filter_update2                  0x08005bfa   Section        0  ad7190.o(i.kalman_filter_update2)
    i.main                                   0x08005c54   Section        0  moisture.o(i.main)
    i.osDelay                                0x08005df0   Section        0  rt_cmsis.o(i.osDelay)
    i.osKernelInitialize                     0x08005e08   Section        0  rt_cmsis.o(i.osKernelInitialize)
    i.osKernelStart                          0x08005e2c   Section        0  rt_cmsis.o(i.osKernelStart)
    i.osKernelSysTick                        0x08005e98   Section        0  rt_cmsis.o(i.osKernelSysTick)
    i.osMutexCreate                          0x08005eb0   Section        0  rt_cmsis.o(i.osMutexCreate)
    i.osMutexRelease                         0x08005edc   Section        0  rt_cmsis.o(i.osMutexRelease)
    i.osMutexWait                            0x08005ef4   Section        0  rt_cmsis.o(i.osMutexWait)
    i.osSemaphoreCreate                      0x08005f0c   Section        0  rt_cmsis.o(i.osSemaphoreCreate)
    i.osSemaphoreRelease                     0x08005f38   Section        0  rt_cmsis.o(i.osSemaphoreRelease)
    i.osSemaphoreWait                        0x08005f50   Section        0  rt_cmsis.o(i.osSemaphoreWait)
    i.osThreadCreate                         0x08005f68   Section        0  rt_cmsis.o(i.osThreadCreate)
    i.osThreadExit                           0x08005f94   Section        0  rt_cmsis.o(i.osThreadExit)
    i.osThreadGetId                          0x08005fac   Section        0  rt_cmsis.o(i.osThreadGetId)
    i.osThreadTerminate                      0x08005fc4   Section        0  rt_cmsis.o(i.osThreadTerminate)
    i.os_error                               0x08005fdc   Section        0  rtx_conf_cm.o(i.os_error)
    i.os_idle_demon                          0x08005ffe   Section        0  rtx_conf_cm.o(i.os_idle_demon)
    i.os_tick_init                           0x08006004   Section        0  rt_system.o(i.os_tick_init)
    i.os_tick_irqack                         0x0800602c   Section        0  rt_system.o(i.os_tick_irqack)
    i.os_tick_ovf                            0x08006030   Section        0  rt_system.o(i.os_tick_ovf)
    i.os_tick_val                            0x08006040   Section        0  rt_system.o(i.os_tick_val)
    i.rt_alloc_box                           0x08006054   Section        0  rt_membox.o(i.rt_alloc_box)
    i.rt_alloc_mem                           0x0800606e   Section        0  rt_memory.o(i.rt_alloc_mem)
    i.rt_block                               0x080060ac   Section        0  rt_task.o(i.rt_block)
    i.rt_chk_robin                           0x080060e4   Section        0  rt_robin.o(i.rt_chk_robin)
    i.rt_dec_dly                             0x0800612c   Section        0  rt_list.o(i.rt_dec_dly)
    i.rt_dispatch                            0x0800619c   Section        0  rt_task.o(i.rt_dispatch)
    i.rt_dly_wait                            0x080061e0   Section        0  rt_time.o(i.rt_dly_wait)
    i.rt_evt_psh                             0x080061e8   Section        0  rt_event.o(i.rt_evt_psh)
    i.rt_free_box                            0x08006238   Section        0  rt_membox.o(i.rt_free_box)
    i.rt_free_mem                            0x08006264   Section        0  rt_memory.o(i.rt_free_mem)
    i.rt_get_first                           0x0800628c   Section        0  rt_list.o(i.rt_get_first)
    i.rt_id2obj                              0x080062b4   Section        0  rt_cmsis.o(i.rt_id2obj)
    rt_id2obj                                0x080062b5   Thumb Code     8  rt_cmsis.o(i.rt_id2obj)
    i.rt_init_context                        0x080062bc   Section        0  rt_task.o(i.rt_init_context)
    rt_init_context                          0x080062bd   Thumb Code    66  rt_task.o(i.rt_init_context)
    i.rt_init_mem                            0x08006304   Section        0  rt_memory.o(i.rt_init_mem)
    i.rt_init_robin                          0x08006320   Section        0  rt_robin.o(i.rt_init_robin)
    i.rt_init_stack                          0x08006338   Section        0  hal_cm.o(i.rt_init_stack)
    i.rt_mbx_check                           0x080063b8   Section        0  rt_mailbox.o(i.rt_mbx_check)
    i.rt_mbx_init                            0x080063c0   Section        0  rt_mailbox.o(i.rt_mbx_init)
    i.rt_mbx_psh                             0x080063dc   Section        0  rt_mailbox.o(i.rt_mbx_psh)
    i.rt_ms2tick                             0x080064cc   Section        0  rt_cmsis.o(i.rt_ms2tick)
    rt_ms2tick                               0x080064cd   Thumb Code    58  rt_cmsis.o(i.rt_ms2tick)
    i.rt_mut_init                            0x08006510   Section        0  rt_mutex.o(i.rt_mut_init)
    i.rt_mut_release                         0x08006520   Section        0  rt_mutex.o(i.rt_mut_release)
    i.rt_mut_wait                            0x080065f8   Section        0  rt_mutex.o(i.rt_mut_wait)
    i.rt_pop_req                             0x08006670   Section        0  rt_system.o(i.rt_pop_req)
    i.rt_psh_req                             0x080066ec   Section        0  rt_system.o(i.rt_psh_req)
    i.rt_psq_enq                             0x0800670c   Section        0  rt_list.o(i.rt_psq_enq)
    i.rt_put_dly                             0x08006768   Section        0  rt_list.o(i.rt_put_dly)
    i.rt_put_prio                            0x080067b0   Section        0  rt_list.o(i.rt_put_prio)
    i.rt_put_rdy_first                       0x080067e8   Section        0  rt_list.o(i.rt_put_rdy_first)
    i.rt_resort_prio                         0x080067fc   Section        0  rt_list.o(i.rt_resort_prio)
    i.rt_ret_val                             0x08006830   Section        0  hal_cm.o(i.rt_ret_val)
    i.rt_ret_val2                            0x08006836   Section        0  hal_cm.o(i.rt_ret_val2)
    i.rt_rmv_dly                             0x0800683e   Section        0  rt_list.o(i.rt_rmv_dly)
    i.rt_rmv_list                            0x08006868   Section        0  rt_list.o(i.rt_rmv_list)
    i.rt_sem_init                            0x08006898   Section        0  rt_semaphore.o(i.rt_sem_init)
    i.rt_sem_psh                             0x080068a4   Section        0  rt_semaphore.o(i.rt_sem_psh)
    i.rt_sem_send                            0x080068d8   Section        0  rt_semaphore.o(i.rt_sem_send)
    i.rt_sem_wait                            0x08006904   Section        0  rt_semaphore.o(i.rt_sem_wait)
    i.rt_stk_check                           0x08006944   Section        0  rt_system.o(i.rt_stk_check)
    i.rt_switch_req                          0x08006968   Section        0  rt_task.o(i.rt_switch_req)
    i.rt_sys_init                            0x08006990   Section        0  rt_task.o(i.rt_sys_init)
    i.rt_sys_start                           0x08006a5c   Section        0  rt_task.o(i.rt_sys_start)
    i.rt_systick                             0x08006ad4   Section        0  rt_system.o(i.rt_systick)
    i.rt_tid2ptcb                            0x08006b14   Section        0  rt_cmsis.o(i.rt_tid2ptcb)
    rt_tid2ptcb                              0x08006b15   Thumb Code    18  rt_cmsis.o(i.rt_tid2ptcb)
    i.rt_timer_insert                        0x08006b28   Section        0  rt_cmsis.o(i.rt_timer_insert)
    rt_timer_insert                          0x08006b29   Thumb Code    48  rt_cmsis.o(i.rt_timer_insert)
    i.rt_tsk_create                          0x08006b5c   Section        0  rt_task.o(i.rt_tsk_create)
    i.rt_tsk_delete                          0x08006be4   Section        0  rt_task.o(i.rt_tsk_delete)
    i.rt_tsk_prio                            0x08006d60   Section        0  rt_task.o(i.rt_tsk_prio)
    i.rt_tsk_self                            0x08006ddc   Section        0  rt_task.o(i.rt_tsk_self)
    i.svcDelay                               0x08006dec   Section        0  rt_cmsis.o(i.svcDelay)
    i.svcKernelInitialize                    0x08006e00   Section        0  rt_cmsis.o(i.svcKernelInitialize)
    i.svcKernelStart                         0x08006e70   Section        0  rt_cmsis.o(i.svcKernelStart)
    i.svcKernelSysTick                       0x08006eb8   Section        0  rt_cmsis.o(i.svcKernelSysTick)
    i.svcMessageCreate                       0x08006ef0   Section        0  rt_cmsis.o(i.svcMessageCreate)
    i.svcMutexCreate                         0x08006f14   Section        0  rt_cmsis.o(i.svcMutexCreate)
    i.svcMutexRelease                        0x08006f30   Section        0  rt_cmsis.o(i.svcMutexRelease)
    i.svcMutexWait                           0x08006f52   Section        0  rt_cmsis.o(i.svcMutexWait)
    i.svcSemaphoreCreate                     0x08006f8c   Section        0  rt_cmsis.o(i.svcSemaphoreCreate)
    i.svcSemaphoreRelease                    0x08006fb0   Section        0  rt_cmsis.o(i.svcSemaphoreRelease)
    i.svcSemaphoreWait                       0x08006fd8   Section        0  rt_cmsis.o(i.svcSemaphoreWait)
    i.svcThreadCreate                        0x0800700c   Section        0  rt_cmsis.o(i.svcThreadCreate)
    i.svcThreadGetId                         0x08007078   Section        0  rt_cmsis.o(i.svcThreadGetId)
    i.svcThreadTerminate                     0x08007094   Section        0  rt_cmsis.o(i.svcThreadTerminate)
    i.sysTimerTick                           0x080070cc   Section        0  rt_cmsis.o(i.sysTimerTick)
    locale$$code                             0x08007128   Section       44  lc_numeric_c.o(locale$$code)
    x$fpl$d2f                                0x08007154   Section       98  d2f.o(x$fpl$d2f)
    x$fpl$dcmpinf                            0x080071b6   Section       24  dcmpi.o(x$fpl$dcmpinf)
    x$fpl$dflt                               0x080071ce   Section       46  dflt_clz.o(x$fpl$dflt)
    x$fpl$dleqf                              0x080071fc   Section      120  dleqf.o(x$fpl$dleqf)
    x$fpl$dmul                               0x08007274   Section      340  dmul.o(x$fpl$dmul)
    x$fpl$dnaninf                            0x080073c8   Section      156  dnaninf.o(x$fpl$dnaninf)
    x$fpl$dretinf                            0x08007464   Section       12  dretinf.o(x$fpl$dretinf)
    x$fpl$drleqf                             0x08007470   Section      108  drleqf.o(x$fpl$drleqf)
    x$fpl$f2d                                0x080074dc   Section       86  f2d.o(x$fpl$f2d)
    x$fpl$fadd                               0x08007534   Section      196  faddsub_clz.o(x$fpl$fadd)
    _fadd1                                   0x08007543   Thumb Code     0  faddsub_clz.o(x$fpl$fadd)
    x$fpl$fcmpinf                            0x080075f8   Section       24  fcmpi.o(x$fpl$fcmpinf)
    x$fpl$fdiv                               0x08007610   Section      388  fdiv.o(x$fpl$fdiv)
    _fdiv1                                   0x08007611   Thumb Code     0  fdiv.o(x$fpl$fdiv)
    x$fpl$feqf                               0x08007794   Section      104  feqf.o(x$fpl$feqf)
    x$fpl$ffix                               0x080077fc   Section       54  ffix.o(x$fpl$ffix)
    x$fpl$ffixu                              0x08007834   Section       62  ffixu.o(x$fpl$ffixu)
    x$fpl$fflt                               0x08007874   Section       48  fflt_clz.o(x$fpl$fflt)
    x$fpl$ffltu                              0x080078a4   Section       38  fflt_clz.o(x$fpl$ffltu)
    x$fpl$fleqf                              0x080078cc   Section      104  fleqf.o(x$fpl$fleqf)
    x$fpl$fmul                               0x08007934   Section      258  fmul.o(x$fpl$fmul)
    x$fpl$fnaninf                            0x08007a36   Section      140  fnaninf.o(x$fpl$fnaninf)
    x$fpl$fretinf                            0x08007ac2   Section       10  fretinf.o(x$fpl$fretinf)
    x$fpl$frleqf                             0x08007acc   Section       98  frleqf.o(x$fpl$frleqf)
    x$fpl$frsb                               0x08007b2e   Section       20  faddsub_clz.o(x$fpl$frsb)
    x$fpl$fsub                               0x08007b44   Section      234  faddsub_clz.o(x$fpl$fsub)
    _fsub1                                   0x08007b53   Thumb Code     0  faddsub_clz.o(x$fpl$fsub)
    x$fpl$printf1                            0x08007c2e   Section        4  printf1.o(x$fpl$printf1)
    x$fpl$usenofp                            0x08007c32   Section        0  usenofp.o(x$fpl$usenofp)
    .constdata                               0x08007c34   Section       16  ad7190.o(.constdata)
    .constdata                               0x08007c44   Section       32  ws100t10.o(.constdata)
    .constdata                               0x08007c64   Section       16  max6675.o(.constdata)
    .constdata                               0x08007c74   Section        4  usarthmi.o(.constdata)
    .constdata                               0x08007c78   Section      234  hmi.o(.constdata)
    .constdata                               0x08007d64   Section      104  rtx_conf_cm.o(.constdata)
    __tagsym$$used                           0x08007d80   Number         0  rtx_conf_cm.o(.constdata)
    __tagsym$$used                           0x08007d84   Number         0  rtx_conf_cm.o(.constdata)
    __tagsym$$used                           0x08007d88   Number         0  rtx_conf_cm.o(.constdata)
    __tagsym$$used                           0x08007d8c   Number         0  rtx_conf_cm.o(.constdata)
    .constdata                               0x08007dcc   Section       17  __printf_flags_wp.o(.constdata)
    maptable                                 0x08007dcc   Data          17  __printf_flags_wp.o(.constdata)
    .constdata                               0x08007de0   Section      148  bigflt0.o(.constdata)
    tenpwrs_x                                0x08007de0   Data          60  bigflt0.o(.constdata)
    tenpwrs_i                                0x08007e1c   Data          64  bigflt0.o(.constdata)
    locale$$data                             0x08007e94   Section       28  lc_numeric_c.o(locale$$data)
    __lcnum_c_name                           0x08007e98   Data           2  lc_numeric_c.o(locale$$data)
    __lcnum_c_start                          0x08007ea0   Data           0  lc_numeric_c.o(locale$$data)
    __lcnum_c_point                          0x08007eac   Data           0  lc_numeric_c.o(locale$$data)
    __lcnum_c_thousands                      0x08007eae   Data           0  lc_numeric_c.o(locale$$data)
    __lcnum_c_grouping                       0x08007eaf   Data           0  lc_numeric_c.o(locale$$data)
    __lcnum_c_end                            0x08007eb0   Data           0  lc_numeric_c.o(locale$$data)
    .data                                    0x20000000   Section       53  ad7190.o(.data)
    WeightData2Temp                          0x2000000c   Data           4  ad7190.o(.data)
    .data                                    0x20000038   Section       48  ws100t10.o(.data)
    HeatOp_State                             0x2000005c   Data           1  ws100t10.o(.data)
    .data                                    0x20000068   Section        4  max6675.o(.data)
    .data                                    0x2000006c   Section       24  usarthmi.o(.data)
    UsartDelayTime                           0x20000070   Data           2  usarthmi.o(.data)
    RxFlag                                   0x20000072   Data           1  usarthmi.o(.data)
    Datai                                    0x20000073   Data           1  usarthmi.o(.data)
    .data                                    0x20000084   Section       57  hmi.o(.data)
    .data                                    0x200000c0   Section       20  rtx_conf_cm.o(.data)
    nr_mutex                                 0x200000d0   Data           4  rtx_conf_cm.o(.data)
    .data                                    0x200000d4   Section       20  system_stm32f10x.o(.data)
    .data                                    0x200000e8   Section        8  rt_cmsis.o(.data)
    .data                                    0x200000f0   Section        8  rt_task.o(.data)
    .data                                    0x200000f8   Section        8  rt_system.o(.data)
    os_lock                                  0x200000f8   Data           1  rt_system.o(.data)
    os_psh_flag                              0x200000f9   Data           1  rt_system.o(.data)
    pend_flags                               0x200000fa   Data           1  rt_system.o(.data)
    .data                                    0x20000100   Section        4  rt_time.o(.data)
    .data                                    0x20000104   Section        8  rt_robin.o(.data)
    .data                                    0x2000010c   Section        1  hal_cm.o(.data)
    .bss                                     0x20000110   Section       40  ad7190.o(.bss)
    .bss                                     0x20000138   Section       20  max6675.o(.bss)
    .bss                                     0x2000014c   Section      100  usarthmi.o(.bss)
    .bss                                     0x200001b0   Section      356  hmi.o(.bss)
    .bss                                     0x20000314   Section       52  rt_task.o(.bss)
    .bss                                     0x20000348   Section       48  rt_list.o(.bss)
    .bss                                     0x20000378   Section       96  libspace.o(.bss)
    HEAP                                     0x200003d8   Section      512  startup_stm32f10x_md.o(HEAP)
    Heap_Mem                                 0x200003d8   Data         512  startup_stm32f10x_md.o(HEAP)
    STACK                                    0x200005d8   Section     1024  startup_stm32f10x_md.o(STACK)
    Stack_Mem                                0x200005d8   Data        1024  startup_stm32f10x_md.o(STACK)
    __initial_sp                             0x200009d8   Data           0  startup_stm32f10x_md.o(STACK)
    .ARM.__AT_0x20001000                     0x20001000   Section      150  hmi.o(.ARM.__AT_0x20001000)
    buf                                      0x20001000   Data         150  hmi.o(.ARM.__AT_0x20001000)
    .ARM.__AT_0x20001200                     0x20001200   Section      150  hmi.o(.ARM.__AT_0x20001200)
    buf                                      0x20001200   Data         150  hmi.o(.ARM.__AT_0x20001200)
    .bss                                     0x20001298   Section    14148  rtx_conf_cm.o(.bss)
    std_libspace                             0x2000459c   Data         960  rtx_conf_cm.o(.bss)
    std_libmutex                             0x2000495c   Data         128  rtx_conf_cm.o(.bss)

    Global Symbols

    Symbol Name                              Value     Ov Type        Size  Object(Section)

    BuildAttributes$$THM_ISAv4$P$D$K$B$S$PE$A:L22UL41UL21$X:L11$S22US41US21$IEEE1$IW$USESV6$~STKCKD$USESV7$~SHL$OTIME$ROPI$IEEEJ$EBA8$UX$STANDARDLIB$REQ8$PRES8$EABIv2 0x00000000   Number         0  anon$$obj.o ABSOLUTE
    __ARM_use_no_argv                        0x00000000   Number         0  moisture.o ABSOLUTE
    _printf_flags                            0x00000000   Number         0  printf_stubs.o ABSOLUTE
    _printf_return_value                     0x00000000   Number         0  printf_stubs.o ABSOLUTE
    _printf_sizespec                         0x00000000   Number         0  printf_stubs.o ABSOLUTE
    _printf_widthprec                        0x00000000   Number         0  printf_stubs.o ABSOLUTE
    __ARM_exceptions_init                     - Undefined Weak Reference
    __alloca_initialize                       - Undefined Weak Reference
    __arm_fini_                               - Undefined Weak Reference
    __arm_preinit_                            - Undefined Weak Reference
    __cpp_initialize__aeabi_                  - Undefined Weak Reference
    __cxa_finalize                            - Undefined Weak Reference
    __sigvec_lookup                           - Undefined Weak Reference
    _atexit_init                              - Undefined Weak Reference
    _call_atexit_fns                          - Undefined Weak Reference
    _clock_init                               - Undefined Weak Reference
    _fp_trap_init                             - Undefined Weak Reference
    _fp_trap_shutdown                         - Undefined Weak Reference
    _get_lc_collate                           - Undefined Weak Reference
    _get_lc_ctype                             - Undefined Weak Reference
    _get_lc_monetary                          - Undefined Weak Reference
    _get_lc_time                              - Undefined Weak Reference
    _getenv_init                              - Undefined Weak Reference
    _handle_redirection                       - Undefined Weak Reference
    _init_alloc                               - Undefined Weak Reference
    _init_user_alloc                          - Undefined Weak Reference
    _initio                                   - Undefined Weak Reference
    _printf_mbtowc                            - Undefined Weak Reference
    _printf_truncate_signed                   - Undefined Weak Reference
    _printf_truncate_unsigned                 - Undefined Weak Reference
    _rand_init                                - Undefined Weak Reference
    _signal_finish                            - Undefined Weak Reference
    _signal_init                              - Undefined Weak Reference
    _terminate_alloc                          - Undefined Weak Reference
    _terminate_user_alloc                     - Undefined Weak Reference
    _terminateio                              - Undefined Weak Reference
    __Vectors_Size                           0x000000ec   Number         0  startup_stm32f10x_md.o ABSOLUTE
    __RL_RTX_VER                             0x00000482   Number         0  rt_system.o ABSOLUTE
    __Vectors                                0x08000000   Data           4  startup_stm32f10x_md.o(RESET)
    __Vectors_End                            0x080000ec   Data           0  startup_stm32f10x_md.o(RESET)
    __main                                   0x080000ed   Thumb Code     8  __main.o(!!!main)
    __scatterload                            0x080000f5   Thumb Code     0  __scatter.o(!!!scatter)
    __scatterload_rt2                        0x080000f5   Thumb Code    44  __scatter.o(!!!scatter)
    __scatterload_rt2_thumb_only             0x080000f5   Thumb Code     0  __scatter.o(!!!scatter)
    __scatterload_null                       0x08000103   Thumb Code     0  __scatter.o(!!!scatter)
    __scatterload_copy                       0x08000129   Thumb Code    26  __scatter_copy.o(!!handler_copy)
    __scatterload_zeroinit                   0x08000145   Thumb Code    28  __scatter_zi.o(!!handler_zi)
    _printf_f                                0x08000161   Thumb Code     0  _printf_f.o(.ARM.Collect$$_printf_percent$$00000003)
    _printf_percent                          0x08000161   Thumb Code     0  _printf_percent.o(.ARM.Collect$$_printf_percent$$00000000)
    _printf_d                                0x08000167   Thumb Code     0  _printf_d.o(.ARM.Collect$$_printf_percent$$00000009)
    _printf_s                                0x0800016d   Thumb Code     0  _printf_s.o(.ARM.Collect$$_printf_percent$$00000014)
    _printf_percent_end                      0x08000173   Thumb Code     0  _printf_percent_end.o(.ARM.Collect$$_printf_percent$$00000017)
    __rt_lib_init                            0x08000177   Thumb Code     0  libinit.o(.ARM.Collect$$libinit$$00000000)
    __rt_lib_init_fp_1                       0x08000179   Thumb Code     0  libinit2.o(.ARM.Collect$$libinit$$00000002)
    __rt_lib_init_heap_1                     0x08000179   Thumb Code     0  libinit2.o(.ARM.Collect$$libinit$$0000000A)
    __rt_lib_init_lc_common                  0x08000179   Thumb Code     0  libinit2.o(.ARM.Collect$$libinit$$0000000F)
    __rt_lib_init_preinit_1                  0x08000179   Thumb Code     0  libinit2.o(.ARM.Collect$$libinit$$00000004)
    __rt_lib_init_rand_1                     0x08000179   Thumb Code     0  libinit2.o(.ARM.Collect$$libinit$$0000000E)
    __rt_lib_init_user_alloc_1               0x08000179   Thumb Code     0  libinit2.o(.ARM.Collect$$libinit$$0000000C)
    __rt_lib_init_lc_collate_1               0x0800017f   Thumb Code     0  libinit2.o(.ARM.Collect$$libinit$$00000011)
    __rt_lib_init_lc_ctype_1                 0x0800017f   Thumb Code     0  libinit2.o(.ARM.Collect$$libinit$$00000013)
    __rt_lib_init_lc_monetary_1              0x0800017f   Thumb Code     0  libinit2.o(.ARM.Collect$$libinit$$00000015)
    __rt_lib_init_lc_numeric_2               0x0800017f   Thumb Code     0  libinit2.o(.ARM.Collect$$libinit$$00000016)
    __rt_lib_init_alloca_1                   0x08000189   Thumb Code     0  libinit2.o(.ARM.Collect$$libinit$$0000002E)
    __rt_lib_init_argv_1                     0x08000189   Thumb Code     0  libinit2.o(.ARM.Collect$$libinit$$0000002C)
    __rt_lib_init_atexit_1                   0x08000189   Thumb Code     0  libinit2.o(.ARM.Collect$$libinit$$0000001B)
    __rt_lib_init_clock_1                    0x08000189   Thumb Code     0  libinit2.o(.ARM.Collect$$libinit$$00000021)
    __rt_lib_init_cpp_1                      0x08000189   Thumb Code     0  libinit2.o(.ARM.Collect$$libinit$$00000032)
    __rt_lib_init_exceptions_1               0x08000189   Thumb Code     0  libinit2.o(.ARM.Collect$$libinit$$00000030)
    __rt_lib_init_fp_trap_1                  0x08000189   Thumb Code     0  libinit2.o(.ARM.Collect$$libinit$$0000001F)
    __rt_lib_init_getenv_1                   0x08000189   Thumb Code     0  libinit2.o(.ARM.Collect$$libinit$$00000023)
    __rt_lib_init_lc_numeric_1               0x08000189   Thumb Code     0  libinit2.o(.ARM.Collect$$libinit$$00000017)
    __rt_lib_init_lc_time_1                  0x08000189   Thumb Code     0  libinit2.o(.ARM.Collect$$libinit$$00000019)
    __rt_lib_init_return                     0x08000189   Thumb Code     0  libinit2.o(.ARM.Collect$$libinit$$00000033)
    __rt_lib_init_signal_1                   0x08000189   Thumb Code     0  libinit2.o(.ARM.Collect$$libinit$$0000001D)
    __rt_lib_init_stdio_1                    0x08000189   Thumb Code     0  libinit2.o(.ARM.Collect$$libinit$$00000025)
    __rt_lib_shutdown                        0x0800018b   Thumb Code     0  libshutdown.o(.ARM.Collect$$libshutdown$$00000000)
    __rt_lib_shutdown_cpp_1                  0x0800018d   Thumb Code     0  libshutdown2.o(.ARM.Collect$$libshutdown$$00000004)
    __rt_lib_shutdown_fini_1                 0x0800018d   Thumb Code     0  libshutdown2.o(.ARM.Collect$$libshutdown$$00000002)
    __rt_lib_shutdown_fp_trap_1              0x0800018d   Thumb Code     0  libshutdown2.o(.ARM.Collect$$libshutdown$$00000009)
    __rt_lib_shutdown_heap_1                 0x0800018d   Thumb Code     0  libshutdown2.o(.ARM.Collect$$libshutdown$$00000011)
    __rt_lib_shutdown_return                 0x0800018d   Thumb Code     0  libshutdown2.o(.ARM.Collect$$libshutdown$$00000012)
    __rt_lib_shutdown_signal_1               0x0800018d   Thumb Code     0  libshutdown2.o(.ARM.Collect$$libshutdown$$0000000C)
    __rt_lib_shutdown_stdio_1                0x0800018d   Thumb Code     0  libshutdown2.o(.ARM.Collect$$libshutdown$$00000006)
    __rt_lib_shutdown_user_alloc_1           0x0800018d   Thumb Code     0  libshutdown2.o(.ARM.Collect$$libshutdown$$0000000E)
    __rt_entry                               0x0800018f   Thumb Code     0  __rtentry.o(.ARM.Collect$$rtentry$$00000000)
    __rt_entry_presh_1                       0x0800018f   Thumb Code     0  __rtentry2.o(.ARM.Collect$$rtentry$$00000002)
    __rt_entry_sh                            0x0800018f   Thumb Code     0  __rtentry4.o(.ARM.Collect$$rtentry$$00000004)
    __rt_entry_li                            0x08000195   Thumb Code     0  __rtentry2.o(.ARM.Collect$$rtentry$$0000000A)
    __rt_entry_postsh_1                      0x08000195   Thumb Code     0  __rtentry2.o(.ARM.Collect$$rtentry$$00000009)
    __rt_entry_postli_1                      0x08000199   Thumb Code     0  __rtentry2.o(.ARM.Collect$$rtentry$$0000000B)
    __rt_entry_main                          0x080001a1   Thumb Code     0  __rtentry2.o(.ARM.Collect$$rtentry$$0000000D)
    __rt_exit                                0x080001a9   Thumb Code     0  rtexit.o(.ARM.Collect$$rtexit$$00000000)
    __rt_exit_ls                             0x080001ab   Thumb Code     0  rtexit2.o(.ARM.Collect$$rtexit$$00000003)
    __rt_exit_prels_1                        0x080001ab   Thumb Code     0  rtexit2.o(.ARM.Collect$$rtexit$$00000002)
    __rt_exit_exit                           0x080001af   Thumb Code     0  rtexit2.o(.ARM.Collect$$rtexit$$00000004)
    _platform_post_lib_init                  0x080001b5   Thumb Code    24  rtx_conf_cm.o(.emb_text)
    rt_set_PSP                               0x080001d1   Thumb Code     6  hal_cm3.o(.emb_text)
    rt_get_PSP                               0x080001d7   Thumb Code     6  hal_cm3.o(.emb_text)
    os_set_env                               0x080001dd   Thumb Code    24  hal_cm3.o(.emb_text)
    _alloc_box                               0x080001f9   Thumb Code    28  hal_cm3.o(.emb_text)
    _free_box                                0x08000219   Thumb Code    28  hal_cm3.o(.emb_text)
    SVC_Handler                              0x08000239   Thumb Code   108  hal_cm3.o(.emb_text)
    PendSV_Handler                           0x080002b1   Thumb Code    56  hal_cm3.o(.emb_text)
    SysTick_Handler                          0x080002ed   Thumb Code     8  hal_cm3.o(.emb_text)
    OS_Tick_Handler                          0x080002f5   Thumb Code    12  hal_cm3.o(.emb_text)
    Reset_Handler                            0x08000301   Thumb Code     8  startup_stm32f10x_md.o(.text)
    NMI_Handler                              0x08000309   Thumb Code     2  startup_stm32f10x_md.o(.text)
    HardFault_Handler                        0x0800030b   Thumb Code     2  startup_stm32f10x_md.o(.text)
    MemManage_Handler                        0x0800030d   Thumb Code     2  startup_stm32f10x_md.o(.text)
    BusFault_Handler                         0x0800030f   Thumb Code     2  startup_stm32f10x_md.o(.text)
    UsageFault_Handler                       0x08000311   Thumb Code     2  startup_stm32f10x_md.o(.text)
    DebugMon_Handler                         0x08000315   Thumb Code     2  startup_stm32f10x_md.o(.text)
    ADC1_2_IRQHandler                        0x0800031b   Thumb Code     0  startup_stm32f10x_md.o(.text)
    CAN1_RX1_IRQHandler                      0x0800031b   Thumb Code     0  startup_stm32f10x_md.o(.text)
    CAN1_SCE_IRQHandler                      0x0800031b   Thumb Code     0  startup_stm32f10x_md.o(.text)
    DMA1_Channel1_IRQHandler                 0x0800031b   Thumb Code     0  startup_stm32f10x_md.o(.text)
    DMA1_Channel2_IRQHandler                 0x0800031b   Thumb Code     0  startup_stm32f10x_md.o(.text)
    DMA1_Channel3_IRQHandler                 0x0800031b   Thumb Code     0  startup_stm32f10x_md.o(.text)
    DMA1_Channel4_IRQHandler                 0x0800031b   Thumb Code     0  startup_stm32f10x_md.o(.text)
    DMA1_Channel5_IRQHandler                 0x0800031b   Thumb Code     0  startup_stm32f10x_md.o(.text)
    DMA1_Channel6_IRQHandler                 0x0800031b   Thumb Code     0  startup_stm32f10x_md.o(.text)
    DMA1_Channel7_IRQHandler                 0x0800031b   Thumb Code     0  startup_stm32f10x_md.o(.text)
    EXTI0_IRQHandler                         0x0800031b   Thumb Code     0  startup_stm32f10x_md.o(.text)
    EXTI15_10_IRQHandler                     0x0800031b   Thumb Code     0  startup_stm32f10x_md.o(.text)
    EXTI1_IRQHandler                         0x0800031b   Thumb Code     0  startup_stm32f10x_md.o(.text)
    EXTI2_IRQHandler                         0x0800031b   Thumb Code     0  startup_stm32f10x_md.o(.text)
    EXTI3_IRQHandler                         0x0800031b   Thumb Code     0  startup_stm32f10x_md.o(.text)
    EXTI4_IRQHandler                         0x0800031b   Thumb Code     0  startup_stm32f10x_md.o(.text)
    EXTI9_5_IRQHandler                       0x0800031b   Thumb Code     0  startup_stm32f10x_md.o(.text)
    FLASH_IRQHandler                         0x0800031b   Thumb Code     0  startup_stm32f10x_md.o(.text)
    I2C1_ER_IRQHandler                       0x0800031b   Thumb Code     0  startup_stm32f10x_md.o(.text)
    I2C1_EV_IRQHandler                       0x0800031b   Thumb Code     0  startup_stm32f10x_md.o(.text)
    I2C2_ER_IRQHandler                       0x0800031b   Thumb Code     0  startup_stm32f10x_md.o(.text)
    I2C2_EV_IRQHandler                       0x0800031b   Thumb Code     0  startup_stm32f10x_md.o(.text)
    PVD_IRQHandler                           0x0800031b   Thumb Code     0  startup_stm32f10x_md.o(.text)
    RCC_IRQHandler                           0x0800031b   Thumb Code     0  startup_stm32f10x_md.o(.text)
    RTCAlarm_IRQHandler                      0x0800031b   Thumb Code     0  startup_stm32f10x_md.o(.text)
    RTC_IRQHandler                           0x0800031b   Thumb Code     0  startup_stm32f10x_md.o(.text)
    SPI1_IRQHandler                          0x0800031b   Thumb Code     0  startup_stm32f10x_md.o(.text)
    SPI2_IRQHandler                          0x0800031b   Thumb Code     0  startup_stm32f10x_md.o(.text)
    TAMPER_IRQHandler                        0x0800031b   Thumb Code     0  startup_stm32f10x_md.o(.text)
    TIM1_BRK_IRQHandler                      0x0800031b   Thumb Code     0  startup_stm32f10x_md.o(.text)
    TIM1_CC_IRQHandler                       0x0800031b   Thumb Code     0  startup_stm32f10x_md.o(.text)
    TIM1_TRG_COM_IRQHandler                  0x0800031b   Thumb Code     0  startup_stm32f10x_md.o(.text)
    TIM1_UP_IRQHandler                       0x0800031b   Thumb Code     0  startup_stm32f10x_md.o(.text)
    TIM3_IRQHandler                          0x0800031b   Thumb Code     0  startup_stm32f10x_md.o(.text)
    TIM4_IRQHandler                          0x0800031b   Thumb Code     0  startup_stm32f10x_md.o(.text)
    USART2_IRQHandler                        0x0800031b   Thumb Code     0  startup_stm32f10x_md.o(.text)
    USART3_IRQHandler                        0x0800031b   Thumb Code     0  startup_stm32f10x_md.o(.text)
    USBWakeUp_IRQHandler                     0x0800031b   Thumb Code     0  startup_stm32f10x_md.o(.text)
    USB_HP_CAN1_TX_IRQHandler                0x0800031b   Thumb Code     0  startup_stm32f10x_md.o(.text)
    USB_LP_CAN1_RX0_IRQHandler               0x0800031b   Thumb Code     0  startup_stm32f10x_md.o(.text)
    WWDG_IRQHandler                          0x0800031b   Thumb Code     0  startup_stm32f10x_md.o(.text)
    __user_initial_stackheap                 0x0800031d   Thumb Code     0  startup_stm32f10x_md.o(.text)
    __user_libspace                          0x08000341   Thumb Code     8  libspace.o(.text)
    __user_perproc_libspace                  0x08000341   Thumb Code     0  libspace.o(.text)
    __2sprintf                               0x08000349   Thumb Code    34  noretval__2sprintf.o(.text)
    _printf_pre_padding                      0x08000371   Thumb Code    44  _printf_pad.o(.text)
    _printf_post_padding                     0x0800039d   Thumb Code    34  _printf_pad.o(.text)
    _printf_str                              0x080003bf   Thumb Code    82  _printf_str.o(.text)
    _printf_int_dec                          0x08000411   Thumb Code   104  _printf_dec.o(.text)
    __printf                                 0x08000489   Thumb Code   308  __printf_flags_wp.o(.text)
    exit                                     0x080005c1   Thumb Code    18  exit.o(.text)
    strcpy                                   0x080005d3   Thumb Code    72  strcpy.o(.text)
    strlen                                   0x0800061b   Thumb Code    62  strlen.o(.text)
    strcmp                                   0x08000659   Thumb Code   128  strcmpv7m.o(.text)
    __use_two_region_memory                  0x080006d9   Thumb Code     2  heapauxi.o(.text)
    __rt_heap_escrow$2region                 0x080006db   Thumb Code     2  heapauxi.o(.text)
    __rt_heap_expand$2region                 0x080006dd   Thumb Code     2  heapauxi.o(.text)
    _printf_int_common                       0x080006df   Thumb Code   178  _printf_intcommon.o(.text)
    __lib_sel_fp_printf                      0x08000791   Thumb Code     2  _printf_fp_dec.o(.text)
    _printf_fp_dec_real                      0x08000943   Thumb Code   620  _printf_fp_dec.o(.text)
    _printf_char_common                      0x08000bbb   Thumb Code    32  _printf_char_common.o(.text)
    _sputc                                   0x08000be1   Thumb Code    10  _sputc.o(.text)
    _printf_cs_common                        0x08000beb   Thumb Code    20  _printf_char.o(.text)
    _printf_char                             0x08000bff   Thumb Code    16  _printf_char.o(.text)
    _printf_string                           0x08000c0f   Thumb Code     8  _printf_char.o(.text)
    __rt_locale                              0x08000c17   Thumb Code    10  rt_locale_twolibspace.o(.text)
    _ll_udiv10                               0x08000c21   Thumb Code   138  lludiv10.o(.text)
    _printf_fp_infnan                        0x08000cad   Thumb Code   112  _printf_fp_infnan.o(.text)
    _btod_etento                             0x08000d2d   Thumb Code   224  bigflt0.o(.text)
    _sys_exit                                0x08000e11   Thumb Code     8  sys_exit.o(.text)
    __user_setup_stackheap                   0x08000e1d   Thumb Code    74  sys_stackheap_outer.o(.text)
    __I$use$semihosting                      0x08000e67   Thumb Code     0  use_no_semi.o(.text)
    __use_no_semihosting_swi                 0x08000e67   Thumb Code     2  use_no_semi.o(.text)
    __semihosting_library_function           0x08000e69   Thumb Code     0  indicate_semi.o(.text)
    _btod_d2e                                0x08000e69   Thumb Code    62  btod.o(CL$$btod_d2e)
    _d2e_denorm_low                          0x08000ea7   Thumb Code    70  btod.o(CL$$btod_d2e_denorm_low)
    _d2e_norm_op1                            0x08000eed   Thumb Code    96  btod.o(CL$$btod_d2e_norm_op1)
    __btod_div_common                        0x08000f4d   Thumb Code   696  btod.o(CL$$btod_div_common)
    _e2e                                     0x08001285   Thumb Code   220  btod.o(CL$$btod_e2e)
    _btod_ediv                               0x08001361   Thumb Code    42  btod.o(CL$$btod_ediv)
    _btod_emul                               0x0800138b   Thumb Code    42  btod.o(CL$$btod_emul)
    __btod_mult_common                       0x080013b5   Thumb Code   580  btod.o(CL$$btod_mult_common)
    SVC_Count                                0x080015f8   Data           4  svc_table.o(SVC_TABLE)
    ACCMD                                    0x080015fd   Thumb Code    30  ws100t10.o(i.ACCMD)
    SVC_Table                                0x080015fc   Data           0  svc_table.o(SVC_TABLE)
    ACCtrl                                   0x08001621   Thumb Code    64  ws100t10.o(i.ACCtrl)
    AC_CTRL_Init                             0x08001665   Thumb Code    12  ws100t10.o(i.AC_CTRL_Init)
    AD7190_Init                              0x08001675   Thumb Code   208  ad7190.o(i.AD7190_Init)
    AD7190_ReadData                          0x0800175d   Thumb Code   286  ad7190.o(i.AD7190_ReadData)
    AD7190_ReadRegister                      0x0800188d   Thumb Code    46  ad7190.o(i.AD7190_ReadRegister)
    AD7190_ReadRegisterOnce                  0x080018bb   Thumb Code    26  ad7190.o(i.AD7190_ReadRegisterOnce)
    AD7190_Run                               0x080018d5   Thumb Code  1262  ad7190.o(i.AD7190_Run)
    AD7190_WaitForReady                      0x08001dd9   Thumb Code    42  ad7190.o(i.AD7190_WaitForReady)
    AD7190_WriteRegister                     0x08001e09   Thumb Code    36  ad7190.o(i.AD7190_WriteRegister)
    AD7190_WriteRegisterOnce                 0x08001e2d   Thumb Code    20  ad7190.o(i.AD7190_WriteRegisterOnce)
    BIOS_TIM2_TIMER_Init                     0x08001e41   Thumb Code    82  usarthmi.o(i.BIOS_TIM2_TIMER_Init)
    BIOS_USART1_Init                         0x08001ea1   Thumb Code   138  usarthmi.o(i.BIOS_USART1_Init)
    BIOS_USART2_Init                         0x08001f41   Thumb Code    90  usart.o(i.BIOS_USART2_Init)
    DataPrint                                0x08001fad   Thumb Code    66  usarthmi.o(i.DataPrint)
    DataRec                                  0x08001ffd   Thumb Code    12  usarthmi.o(i.DataRec)
    DataUnpack                               0x08002009   Thumb Code  5430  hmi.o(i.DataUnpack)
    FM24DataCRC                              0x080035a1   Thumb Code   252  hmi.o(i.FM24DataCRC)
    FM24Init                                 0x080036ed   Thumb Code     8  fm24.o(i.FM24Init)
    FM24_Read                                0x080036f5   Thumb Code    92  fm24.o(i.FM24_Read)
    FM24_Write                               0x08003751   Thumb Code    72  fm24.o(i.FM24_Write)
    GPIO_InPutset                            0x08003799   Thumb Code    40  bios.o(i.GPIO_InPutset)
    GPIO_Init                                0x080037c5   Thumb Code   278  stm32f10x_gpio.o(i.GPIO_Init)
    GPIO_PinRemapConfig                      0x080038dd   Thumb Code   138  stm32f10x_gpio.o(i.GPIO_PinRemapConfig)
    GPIO_ReadInputDataBit                    0x0800396d   Thumb Code    18  stm32f10x_gpio.o(i.GPIO_ReadInputDataBit)
    GPIO_ResetBits                           0x0800397f   Thumb Code     4  stm32f10x_gpio.o(i.GPIO_ResetBits)
    GPIO_SetBits                             0x08003983   Thumb Code     4  stm32f10x_gpio.o(i.GPIO_SetBits)
    HMICMDInit                               0x08003989   Thumb Code    16  hmi.o(i.HMICMDInit)
    I2C2_ACK                                 0x08003c0d   Thumb Code    56  i2c.o(i.I2C2_ACK)
    I2C2_Init                                0x08003c49   Thumb Code    60  i2c.o(i.I2C2_Init)
    I2C2_NACK                                0x08003c89   Thumb Code    56  i2c.o(i.I2C2_NACK)
    I2C2_ReadByte                            0x08003cc5   Thumb Code    96  i2c.o(i.I2C2_ReadByte)
    I2C2_SendByte                            0x08003d29   Thumb Code    98  i2c.o(i.I2C2_SendByte)
    I2C2_Start                               0x08003d91   Thumb Code    56  i2c.o(i.I2C2_Start)
    I2C2_Stop                                0x08003dcd   Thumb Code    50  i2c.o(i.I2C2_Stop)
    I2C2_Wait_ACK                            0x08003e05   Thumb Code    94  i2c.o(i.I2C2_Wait_ACK)
    InstrumentTypeRead                       0x08003e69   Thumb Code    60  bios.o(i.InstrumentTypeRead)
    MAX6675_ConvertTemperature               0x08003ea9   Thumb Code   108  max6675.o(i.MAX6675_ConvertTemperature)
    MAX6675_Init                             0x08003f29   Thumb Code    96  max6675.o(i.MAX6675_Init)
    MAX6675_ReadData                         0x08003f91   Thumb Code    84  max6675.o(i.MAX6675_ReadData)
    Moisturing                               0x08003fe9   Thumb Code  4648  hmi.o(i.Moisturing)
    MoisturingRun                            0x08005301   Thumb Code    12  hmi.o(i.MoisturingRun)
    Pump_OutCmd                              0x08005311   Thumb Code    34  ws100t10.o(i.Pump_OutCmd)
    RCC_APB2PeriphClockCmd                   0x08005339   Thumb Code    26  stm32f10x_rcc.o(i.RCC_APB2PeriphClockCmd)
    SPI1_Configuration                       0x08005359   Thumb Code   122  spi.o(i.SPI1_Configuration)
    SPI1_ReadWrite                           0x080053dd   Thumb Code    50  spi.o(i.SPI1_ReadWrite)
    SPI_Cmd                                  0x08005415   Thumb Code    24  stm32f10x_spi.o(i.SPI_Cmd)
    SPI_I2S_GetFlagStatus                    0x0800542d   Thumb Code    18  stm32f10x_spi.o(i.SPI_I2S_GetFlagStatus)
    SPI_I2S_ReceiveData                      0x0800543f   Thumb Code     6  stm32f10x_spi.o(i.SPI_I2S_ReceiveData)
    SPI_I2S_SendData                         0x08005445   Thumb Code     4  stm32f10x_spi.o(i.SPI_I2S_SendData)
    SPI_Init                                 0x08005449   Thumb Code    60  stm32f10x_spi.o(i.SPI_Init)
    SafeCheck                                0x08005485   Thumb Code    22  bios.o(i.SafeCheck)
    SystemInit                               0x08005589   Thumb Code    78  system_stm32f10x.o(i.SystemInit)
    TIM2_IRQHandler                          0x080055e9   Thumb Code   116  usarthmi.o(i.TIM2_IRQHandler)
    UART1_Received                           0x08005671   Thumb Code    20  usarthmi.o(i.UART1_Received)
    UART1_Send                               0x08005689   Thumb Code    28  usarthmi.o(i.UART1_Send)
    USART1_IRQHandler                        0x080056a9   Thumb Code   128  usarthmi.o(i.USART1_IRQHandler)
    USART2Print                              0x0800573d   Thumb Code    48  usart.o(i.USART2Print)
    USART2_Send                              0x08005771   Thumb Code    20  usart.o(i.USART2_Send)
    USARTHMIInit                             0x08005789   Thumb Code    24  usarthmi.o(i.USARTHMIInit)
    USART_ITConfig                           0x080057a9   Thumb Code    74  stm32f10x_usart.o(i.USART_ITConfig)
    WS100T10_Ctrl                            0x080057f5   Thumb Code   138  i2c.o(i.WS100T10_Ctrl)
    WS100T10_Init                            0x0800588d   Thumb Code   122  i2c.o(i.WS100T10_Init)
    __ARM_fpclassify                         0x08005919   Thumb Code    40  fpclassify.o(i.__ARM_fpclassify)
    _init_box                                0x08005963   Thumb Code    70  rt_membox.o(i._init_box)
    _is_digit                                0x080059a9   Thumb Code    14  __printf_wp.o(i._is_digit)
    _mutex_acquire                           0x080059b9   Thumb Code    22  rtx_conf_cm.o(i._mutex_acquire)
    _mutex_release                           0x080059d9   Thumb Code    18  rtx_conf_cm.o(i._mutex_release)
    _task_ACCtrl                             0x080059f5   Thumb Code    48  ws100t10.o(i._task_ACCtrl)
    dbg_init                                 0x08005a31   Thumb Code    34  hal_cm.o(i.dbg_init)
    dbg_task_notify                          0x08005a61   Thumb Code    32  hal_cm.o(i.dbg_task_notify)
    dbg_task_switch                          0x08005a81   Thumb Code    16  hal_cm.o(i.dbg_task_switch)
    delay_us                                 0x08005a91   Thumb Code   130  delay.o(i.delay_us)
    isrMessagePut                            0x08005b13   Thumb Code    44  rt_cmsis.o(i.isrMessagePut)
    isrSemaphoreRelease                      0x08005b3f   Thumb Code    40  rt_cmsis.o(i.isrSemaphoreRelease)
    isr_mbx_send                             0x08005b67   Thumb Code    14  rt_mailbox.o(i.isr_mbx_send)
    isr_sem_send                             0x08005b75   Thumb Code    16  rt_semaphore.o(i.isr_sem_send)
    kalman_filter_init                       0x08005b85   Thumb Code    14  max6675.o(i.kalman_filter_init)
    kalman_filter_init2                      0x08005b93   Thumb Code    14  ad7190.o(i.kalman_filter_init2)
    kalman_filter_update                     0x08005ba1   Thumb Code    90  max6675.o(i.kalman_filter_update)
    kalman_filter_update2                    0x08005bfb   Thumb Code    90  ad7190.o(i.kalman_filter_update2)
    main                                     0x08005c55   Thumb Code   362  moisture.o(i.main)
    osDelay                                  0x08005df1   Thumb Code    18  rt_cmsis.o(i.osDelay)
    osKernelInitialize                       0x08005e09   Thumb Code    30  rt_cmsis.o(i.osKernelInitialize)
    osKernelStart                            0x08005e2d   Thumb Code    98  rt_cmsis.o(i.osKernelStart)
    osKernelSysTick                          0x08005e99   Thumb Code    18  rt_cmsis.o(i.osKernelSysTick)
    osMutexCreate                            0x08005eb1   Thumb Code    36  rt_cmsis.o(i.osMutexCreate)
    osMutexRelease                           0x08005edd   Thumb Code    18  rt_cmsis.o(i.osMutexRelease)
    osMutexWait                              0x08005ef5   Thumb Code    18  rt_cmsis.o(i.osMutexWait)
    osSemaphoreCreate                        0x08005f0d   Thumb Code    36  rt_cmsis.o(i.osSemaphoreCreate)
    osSemaphoreRelease                       0x08005f39   Thumb Code    18  rt_cmsis.o(i.osSemaphoreRelease)
    osSemaphoreWait                          0x08005f51   Thumb Code    20  rt_cmsis.o(i.osSemaphoreWait)
    osThreadCreate                           0x08005f69   Thumb Code    36  rt_cmsis.o(i.osThreadCreate)
    osThreadExit                             0x08005f95   Thumb Code    14  rt_cmsis.o(i.osThreadExit)
    osThreadGetId                            0x08005fad   Thumb Code    18  rt_cmsis.o(i.osThreadGetId)
    osThreadTerminate                        0x08005fc5   Thumb Code    18  rt_cmsis.o(i.osThreadTerminate)
    os_error                                 0x08005fdd   Thumb Code    34  rtx_conf_cm.o(i.os_error)
    os_idle_demon                            0x08005fff   Thumb Code     4  rtx_conf_cm.o(i.os_idle_demon)
    os_tick_init                             0x08006005   Thumb Code    32  rt_system.o(i.os_tick_init)
    os_tick_irqack                           0x0800602d   Thumb Code     2  rt_system.o(i.os_tick_irqack)
    os_tick_ovf                              0x08006031   Thumb Code    10  rt_system.o(i.os_tick_ovf)
    os_tick_val                              0x08006041   Thumb Code    14  rt_system.o(i.os_tick_val)
    rt_alloc_box                             0x08006055   Thumb Code    26  rt_membox.o(i.rt_alloc_box)
    rt_alloc_mem                             0x0800606f   Thumb Code    62  rt_memory.o(i.rt_alloc_mem)
    rt_block                                 0x080060ad   Thumb Code    48  rt_task.o(i.rt_block)
    rt_chk_robin                             0x080060e5   Thumb Code    60  rt_robin.o(i.rt_chk_robin)
    rt_dec_dly                               0x0800612d   Thumb Code   102  rt_list.o(i.rt_dec_dly)
    rt_dispatch                              0x0800619d   Thumb Code    60  rt_task.o(i.rt_dispatch)
    rt_dly_wait                              0x080061e1   Thumb Code     6  rt_time.o(i.rt_dly_wait)
    rt_evt_psh                               0x080061e9   Thumb Code    76  rt_event.o(i.rt_evt_psh)
    rt_free_box                              0x08006239   Thumb Code    44  rt_membox.o(i.rt_free_box)
    rt_free_mem                              0x08006265   Thumb Code    40  rt_memory.o(i.rt_free_mem)
    rt_get_first                             0x0800628d   Thumb Code    40  rt_list.o(i.rt_get_first)
    rt_init_mem                              0x08006305   Thumb Code    26  rt_memory.o(i.rt_init_mem)
    rt_init_robin                            0x08006321   Thumb Code    14  rt_robin.o(i.rt_init_robin)
    rt_init_stack                            0x08006339   Thumb Code   118  hal_cm.o(i.rt_init_stack)
    rt_mbx_check                             0x080063b9   Thumb Code     8  rt_mailbox.o(i.rt_mbx_check)
    rt_mbx_init                              0x080063c1   Thumb Code    26  rt_mailbox.o(i.rt_mbx_init)
    rt_mbx_psh                               0x080063dd   Thumb Code   236  rt_mailbox.o(i.rt_mbx_psh)
    rt_mut_init                              0x08006511   Thumb Code    16  rt_mutex.o(i.rt_mut_init)
    rt_mut_release                           0x08006521   Thumb Code   208  rt_mutex.o(i.rt_mut_release)
    rt_mut_wait                              0x080065f9   Thumb Code   114  rt_mutex.o(i.rt_mut_wait)
    rt_pop_req                               0x08006671   Thumb Code   112  rt_system.o(i.rt_pop_req)
    rt_psh_req                               0x080066ed   Thumb Code    22  rt_system.o(i.rt_psh_req)
    rt_psq_enq                               0x0800670d   Thumb Code    88  rt_list.o(i.rt_psq_enq)
    rt_put_dly                               0x08006769   Thumb Code    68  rt_list.o(i.rt_put_dly)
    rt_put_prio                              0x080067b1   Thumb Code    54  rt_list.o(i.rt_put_prio)
    rt_put_rdy_first                         0x080067e9   Thumb Code    14  rt_list.o(i.rt_put_rdy_first)
    rt_resort_prio                           0x080067fd   Thumb Code    46  rt_list.o(i.rt_resort_prio)
    rt_ret_val                               0x08006831   Thumb Code     6  hal_cm.o(i.rt_ret_val)
    rt_ret_val2                              0x08006837   Thumb Code     8  hal_cm.o(i.rt_ret_val2)
    rt_rmv_dly                               0x0800683f   Thumb Code    40  rt_list.o(i.rt_rmv_dly)
    rt_rmv_list                              0x08006869   Thumb Code    44  rt_list.o(i.rt_rmv_list)
    rt_sem_init                              0x08006899   Thumb Code    12  rt_semaphore.o(i.rt_sem_init)
    rt_sem_psh                               0x080068a5   Thumb Code    48  rt_semaphore.o(i.rt_sem_psh)
    rt_sem_send                              0x080068d9   Thumb Code    42  rt_semaphore.o(i.rt_sem_send)
    rt_sem_wait                              0x08006905   Thumb Code    58  rt_semaphore.o(i.rt_sem_wait)
    rt_stk_check                             0x08006945   Thumb Code    28  rt_system.o(i.rt_stk_check)
    rt_switch_req                            0x08006969   Thumb Code    30  rt_task.o(i.rt_switch_req)
    rt_sys_init                              0x08006991   Thumb Code   138  rt_task.o(i.rt_sys_init)
    rt_sys_start                             0x08006a5d   Thumb Code   110  rt_task.o(i.rt_sys_start)
    rt_systick                               0x08006ad5   Thumb Code    50  rt_system.o(i.rt_systick)
    rt_tsk_create                            0x08006b5d   Thumb Code   118  rt_task.o(i.rt_tsk_create)
    rt_tsk_delete                            0x08006be5   Thumb Code   352  rt_task.o(i.rt_tsk_delete)
    rt_tsk_prio                              0x08006d61   Thumb Code   108  rt_task.o(i.rt_tsk_prio)
    rt_tsk_self                              0x08006ddd   Thumb Code    12  rt_task.o(i.rt_tsk_self)
    svcDelay                                 0x08006ded   Thumb Code    18  rt_cmsis.o(i.svcDelay)
    svcKernelInitialize                      0x08006e01   Thumb Code    80  rt_cmsis.o(i.svcKernelInitialize)
    svcKernelStart                           0x08006e71   Thumb Code    62  rt_cmsis.o(i.svcKernelStart)
    svcKernelSysTick                         0x08006eb9   Thumb Code    46  rt_cmsis.o(i.svcKernelSysTick)
    svcMessageCreate                         0x08006ef1   Thumb Code    36  rt_cmsis.o(i.svcMessageCreate)
    svcMutexCreate                           0x08006f15   Thumb Code    28  rt_cmsis.o(i.svcMutexCreate)
    svcMutexRelease                          0x08006f31   Thumb Code    34  rt_cmsis.o(i.svcMutexRelease)
    svcMutexWait                             0x08006f53   Thumb Code    58  rt_cmsis.o(i.svcMutexWait)
    svcSemaphoreCreate                       0x08006f8d   Thumb Code    36  rt_cmsis.o(i.svcSemaphoreCreate)
    svcSemaphoreRelease                      0x08006fb1   Thumb Code    40  rt_cmsis.o(i.svcSemaphoreRelease)
    svcSemaphoreWait                         0x08006fd9   Thumb Code    50  rt_cmsis.o(i.svcSemaphoreWait)
    svcThreadCreate                          0x0800700d   Thumb Code    96  rt_cmsis.o(i.svcThreadCreate)
    svcThreadGetId                           0x08007079   Thumb Code    22  rt_cmsis.o(i.svcThreadGetId)
    svcThreadTerminate                       0x08007095   Thumb Code    50  rt_cmsis.o(i.svcThreadTerminate)
    sysTimerTick                             0x080070cd   Thumb Code    84  rt_cmsis.o(i.sysTimerTick)
    _get_lc_numeric                          0x08007129   Thumb Code    44  lc_numeric_c.o(locale$$code)
    __aeabi_d2f                              0x08007155   Thumb Code     0  d2f.o(x$fpl$d2f)
    _d2f                                     0x08007155   Thumb Code    98  d2f.o(x$fpl$d2f)
    __fpl_dcmp_Inf                           0x080071b7   Thumb Code    24  dcmpi.o(x$fpl$dcmpinf)
    __aeabi_i2d                              0x080071cf   Thumb Code     0  dflt_clz.o(x$fpl$dflt)
    _dflt                                    0x080071cf   Thumb Code    46  dflt_clz.o(x$fpl$dflt)
    __aeabi_cdcmple                          0x080071fd   Thumb Code     0  dleqf.o(x$fpl$dleqf)
    _dcmple                                  0x080071fd   Thumb Code   120  dleqf.o(x$fpl$dleqf)
    __fpl_dcmple_InfNaN                      0x0800725f   Thumb Code     0  dleqf.o(x$fpl$dleqf)
    __aeabi_dmul                             0x08007275   Thumb Code     0  dmul.o(x$fpl$dmul)
    _dmul                                    0x08007275   Thumb Code   332  dmul.o(x$fpl$dmul)
    __fpl_dnaninf                            0x080073c9   Thumb Code   156  dnaninf.o(x$fpl$dnaninf)
    __fpl_dretinf                            0x08007465   Thumb Code    12  dretinf.o(x$fpl$dretinf)
    __aeabi_cdrcmple                         0x08007471   Thumb Code     0  drleqf.o(x$fpl$drleqf)
    _drcmple                                 0x08007471   Thumb Code   108  drleqf.o(x$fpl$drleqf)
    __aeabi_f2d                              0x080074dd   Thumb Code     0  f2d.o(x$fpl$f2d)
    _f2d                                     0x080074dd   Thumb Code    86  f2d.o(x$fpl$f2d)
    __aeabi_fadd                             0x08007535   Thumb Code     0  faddsub_clz.o(x$fpl$fadd)
    _fadd                                    0x08007535   Thumb Code   196  faddsub_clz.o(x$fpl$fadd)
    __fpl_fcmp_Inf                           0x080075f9   Thumb Code    24  fcmpi.o(x$fpl$fcmpinf)
    __aeabi_fdiv                             0x08007611   Thumb Code     0  fdiv.o(x$fpl$fdiv)
    _fdiv                                    0x08007611   Thumb Code   384  fdiv.o(x$fpl$fdiv)
    __aeabi_cfcmpeq                          0x08007795   Thumb Code     0  feqf.o(x$fpl$feqf)
    _fcmpeq                                  0x08007795   Thumb Code   104  feqf.o(x$fpl$feqf)
    __aeabi_f2iz                             0x080077fd   Thumb Code     0  ffix.o(x$fpl$ffix)
    _ffix                                    0x080077fd   Thumb Code    54  ffix.o(x$fpl$ffix)
    __aeabi_f2uiz                            0x08007835   Thumb Code     0  ffixu.o(x$fpl$ffixu)
    _ffixu                                   0x08007835   Thumb Code    62  ffixu.o(x$fpl$ffixu)
    __aeabi_i2f                              0x08007875   Thumb Code     0  fflt_clz.o(x$fpl$fflt)
    _fflt                                    0x08007875   Thumb Code    48  fflt_clz.o(x$fpl$fflt)
    __aeabi_ui2f                             0x080078a5   Thumb Code     0  fflt_clz.o(x$fpl$ffltu)
    _ffltu                                   0x080078a5   Thumb Code    38  fflt_clz.o(x$fpl$ffltu)
    __aeabi_cfcmple                          0x080078cd   Thumb Code     0  fleqf.o(x$fpl$fleqf)
    _fcmple                                  0x080078cd   Thumb Code   104  fleqf.o(x$fpl$fleqf)
    __fpl_fcmple_InfNaN                      0x0800791f   Thumb Code     0  fleqf.o(x$fpl$fleqf)
    __aeabi_fmul                             0x08007935   Thumb Code     0  fmul.o(x$fpl$fmul)
    _fmul                                    0x08007935   Thumb Code   258  fmul.o(x$fpl$fmul)
    __fpl_fnaninf                            0x08007a37   Thumb Code   140  fnaninf.o(x$fpl$fnaninf)
    __fpl_fretinf                            0x08007ac3   Thumb Code    10  fretinf.o(x$fpl$fretinf)
    __aeabi_cfrcmple                         0x08007acd   Thumb Code     0  frleqf.o(x$fpl$frleqf)
    _frcmple                                 0x08007acd   Thumb Code    98  frleqf.o(x$fpl$frleqf)
    __aeabi_frsub                            0x08007b2f   Thumb Code     0  faddsub_clz.o(x$fpl$frsb)
    _frsb                                    0x08007b2f   Thumb Code    20  faddsub_clz.o(x$fpl$frsb)
    __aeabi_fsub                             0x08007b45   Thumb Code     0  faddsub_clz.o(x$fpl$fsub)
    _fsub                                    0x08007b45   Thumb Code   234  faddsub_clz.o(x$fpl$fsub)
    _printf_fp_dec                           0x08007c2f   Thumb Code     4  printf1.o(x$fpl$printf1)
    __I$use$fp                               0x08007c32   Number         0  usenofp.o(x$fpl$usenofp)
    os_thread_def_AD7190_Run                 0x08007c34   Data          16  ad7190.o(.constdata)
    os_thread_def__task_ACCtrl               0x08007c44   Data          16  ws100t10.o(.constdata)
    os_thread_def_HeatTask_Socket            0x08007c54   Data          16  ws100t10.o(.constdata)
    os_thread_def_MAX6675_ConvertTemperature 0x08007c64   Data          16  max6675.o(.constdata)
    os_semaphore_def_semDataBack             0x08007c74   Data           4  usarthmi.o(.constdata)
    os_thread_def_Moisturing                 0x08007c78   Data          16  hmi.o(.constdata)
    os_thread_def_DataUnpack                 0x08007c88   Data          16  hmi.o(.constdata)
    os_maxtaskrun                            0x08007d64   Data           2  rtx_conf_cm.o(.constdata)
    os_stackinfo                             0x08007d68   Data           4  rtx_conf_cm.o(.constdata)
    os_rrobin                                0x08007d6c   Data           4  rtx_conf_cm.o(.constdata)
    os_tickfreq                              0x08007d70   Data           4  rtx_conf_cm.o(.constdata)
    os_tickus_i                              0x08007d74   Data           2  rtx_conf_cm.o(.constdata)
    os_tickus_f                              0x08007d76   Data           2  rtx_conf_cm.o(.constdata)
    os_trv                                   0x08007d78   Data           4  rtx_conf_cm.o(.constdata)
    os_flags                                 0x08007d7c   Data           1  rtx_conf_cm.o(.constdata)
    CMSIS_RTOS_API_Version                   0x08007d80   Data           4  rtx_conf_cm.o(.constdata)
    CMSIS_RTOS_RTX_Version                   0x08007d84   Data           4  rtx_conf_cm.o(.constdata)
    os_clockrate                             0x08007d88   Data           4  rtx_conf_cm.o(.constdata)
    os_timernum                              0x08007d8c   Data           4  rtx_conf_cm.o(.constdata)
    mp_tcb_size                              0x08007d90   Data           2  rtx_conf_cm.o(.constdata)
    mp_stk_size                              0x08007d94   Data           4  rtx_conf_cm.o(.constdata)
    os_stack_sz                              0x08007d98   Data           4  rtx_conf_cm.o(.constdata)
    os_fifo_size                             0x08007d9c   Data           1  rtx_conf_cm.o(.constdata)
    os_thread_def_osTimerThread              0x08007da0   Data          16  rtx_conf_cm.o(.constdata)
    os_messageQ_def_osTimerMessageQ          0x08007db0   Data           8  rtx_conf_cm.o(.constdata)
    mp_tmr_size                              0x08007db8   Data           2  rtx_conf_cm.o(.constdata)
    os_thread_def_main                       0x08007dbc   Data          16  rtx_conf_cm.o(.constdata)
    Region$$Table$$Base                      0x08007e74   Number         0  anon$$obj.o(Region$$Table)
    Region$$Table$$Limit                     0x08007e94   Number         0  anon$$obj.o(Region$$Table)
    ErrCount                                 0x20000000   Data           1  ad7190.o(.data)
    WeightData2                              0x20000004   Data           4  ad7190.o(.data)
    ADvalue2filter                           0x20000008   Data           4  ad7190.o(.data)
    ADvalue2filterOld                        0x20000010   Data           4  ad7190.o(.data)
    ADvalue2                                 0x20000014   Data           4  ad7190.o(.data)
    ic2                                      0x20000018   Data           1  ad7190.o(.data)
    i                                        0x20000019   Data           1  ad7190.o(.data)
    data2                                    0x2000001c   Data           4  ad7190.o(.data)
    FollowCount                              0x20000020   Data           1  ad7190.o(.data)
    TimeCount                                0x20000021   Data           1  ad7190.o(.data)
    WeightZeroOld                            0x20000024   Data           4  ad7190.o(.data)
    modeRega                                 0x20000028   Data           4  ad7190.o(.data)
    configa                                  0x2000002c   Data           4  ad7190.o(.data)
    configao                                 0x20000030   Data           4  ad7190.o(.data)
    weightChanging                           0x20000034   Data           1  ad7190.o(.data)
    Percent                                  0x20000038   Data           8  ws100t10.o(.data)
    GetPercent                               0x20000040   Data           8  ws100t10.o(.data)
    PercentOld                               0x20000048   Data           8  ws100t10.o(.data)
    Kp                                       0x20000050   Data           4  ws100t10.o(.data)
    Ki                                       0x20000054   Data           4  ws100t10.o(.data)
    Kd                                       0x20000058   Data           4  ws100t10.o(.data)
    HeatOutValue                             0x20000060   Data           4  ws100t10.o(.data)
    OutputMax                                0x20000064   Data           4  ws100t10.o(.data)
    Temperature                              0x20000068   Data           4  max6675.o(.data)
    USART_Mutex_ID                           0x2000006c   Data           4  usarthmi.o(.data)
    RxUpToDate                               0x20000074   Data           1  usarthmi.o(.data)
    semDataBack                              0x20000078   Data           4  usarthmi.o(.data)
    os_semaphore_cb_semDataBack              0x2000007c   Data           8  usarthmi.o(.data)
    pageNum                                  0x20000084   Data           1  hmi.o(.data)
    MaxWeight                                0x20000085   Data           1  hmi.o(.data)
    MaxTemp                                  0x20000086   Data           1  hmi.o(.data)
    Resolution                               0x20000088   Data           4  hmi.o(.data)
    ResolutionWater                          0x2000008c   Data           4  hmi.o(.data)
    StartWeight                              0x20000090   Data           4  hmi.o(.data)
    StopWeight                               0x20000094   Data           4  hmi.o(.data)
    WaterPercent                             0x20000098   Data           4  hmi.o(.data)
    WeightOld                                0x2000009c   Data           4  hmi.o(.data)
    CountNochange                            0x200000a0   Data           2  hmi.o(.data)
    CountDelay                               0x200000a2   Data           2  hmi.o(.data)
    SCount                                   0x200000a4   Data           1  hmi.o(.data)
    SRange                                   0x200000a6   Data           2  hmi.o(.data)
    DisData                                  0x200000a8   Data           4  hmi.o(.data)
    Finisflag                                0x200000ac   Data           1  hmi.o(.data)
    t18Dis                                   0x200000ad   Data           1  hmi.o(.data)
    t18DisCount                              0x200000ae   Data           2  hmi.o(.data)
    semDataChange                            0x200000b0   Data           4  hmi.o(.data)
    LastTick                                 0x200000b4   Data           4  hmi.o(.data)
    lostTick                                 0x200000b8   Data           4  hmi.o(.data)
    Err                                      0x200000bc   Data           1  hmi.o(.data)
    osThreadId_osTimerThread                 0x200000c0   Data           4  rtx_conf_cm.o(.data)
    osMessageQId_osTimerMessageQ             0x200000c4   Data           4  rtx_conf_cm.o(.data)
    os_tmr                                   0x200000c8   Data           4  rtx_conf_cm.o(.data)
    m_tmr                                    0x200000cc   Data           4  rtx_conf_cm.o(.data)
    SystemCoreClock                          0x200000d4   Data           4  system_stm32f10x.o(.data)
    AHBPrescTable                            0x200000d8   Data          16  system_stm32f10x.o(.data)
    os_initialized                           0x200000e8   Data           1  rt_cmsis.o(.data)
    os_running                               0x200000e9   Data           1  rt_cmsis.o(.data)
    os_timer_head                            0x200000ec   Data           4  rt_cmsis.o(.data)
    os_tsk                                   0x200000f0   Data           8  rt_task.o(.data)
    os_tick_irqn                             0x200000fc   Data           4  rt_system.o(.data)
    os_time                                  0x20000100   Data           4  rt_time.o(.data)
    os_robin                                 0x20000104   Data           8  rt_robin.o(.data)
    dbg_msg                                  0x2000010c   Data           1  hal_cm.o(.data)
    kf2                                      0x20000110   Data          20  ad7190.o(.bss)
    CalibrateWeight2                         0x20000128   Data          16  ad7190.o(.bss)
    kf                                       0x20000138   Data          20  max6675.o(.bss)
    DataInbuf                                0x2000014c   Data         100  usarthmi.o(.bss)
    Set                                      0x200001b0   Data         196  hmi.o(.bss)
    DataLogValue                             0x20000274   Data         100  hmi.o(.bss)
    NameBuf                                  0x200002d8   Data          40  hmi.o(.bss)
    startTime                                0x20000300   Data          20  hmi.o(.bss)
    os_idle_TCB                              0x20000314   Data          52  rt_task.o(.bss)
    os_rdy                                   0x20000348   Data          24  rt_list.o(.bss)
    os_dly                                   0x20000360   Data          24  rt_list.o(.bss)
    __libspace_start                         0x20000378   Data          96  libspace.o(.bss)
    __temporary_stack_top$libspace           0x200003d8   Data           0  libspace.o(.bss)
    mp_tcb                                   0x20001298   Data         532  rtx_conf_cm.o(.bss)
    mp_stk                                   0x200014b0   Data        9232  rtx_conf_cm.o(.bss)
    os_stack_mem                             0x200038c0   Data        3104  rtx_conf_cm.o(.bss)
    os_fifo                                  0x200044e0   Data         132  rtx_conf_cm.o(.bss)
    os_active_TCB                            0x20004564   Data          40  rtx_conf_cm.o(.bss)
    os_messageQ_q_osTimerMessageQ            0x2000458c   Data          16  rtx_conf_cm.o(.bss)



==============================================================================

Memory Map of the image

  Image Entry point : 0x080000ed

  Load Region LR_IROM1 (Base: 0x08000000, Size: 0x00007fc0, Max: 0x00010000, ABSOLUTE)

    Execution Region ER_IROM1 (Exec base: 0x08000000, Load base: 0x08000000, Size: 0x00007eb0, Max: 0x00010000, ABSOLUTE)

    Exec Addr    Load Addr    Size         Type   Attr      Idx    E Section Name        Object

    0x08000000   0x08000000   0x000000ec   Data   RO         2510    RESET               startup_stm32f10x_md.o
    0x080000ec   0x080000ec   0x00000008   Code   RO         3825  * !!!main             c_w.l(__main.o)
    0x080000f4   0x080000f4   0x00000034   Code   RO         4111    !!!scatter          c_w.l(__scatter.o)
    0x08000128   0x08000128   0x0000001a   Code   RO         4113    !!handler_copy      c_w.l(__scatter_copy.o)
    0x08000142   0x08000142   0x00000002   PAD
    0x08000144   0x08000144   0x0000001c   Code   RO         4115    !!handler_zi        c_w.l(__scatter_zi.o)
    0x08000160   0x08000160   0x00000000   Code   RO         3814    .ARM.Collect$$_printf_percent$$00000000  c_w.l(_printf_percent.o)
    0x08000160   0x08000160   0x00000006   Code   RO         3813    .ARM.Collect$$_printf_percent$$00000003  c_w.l(_printf_f.o)
    0x08000166   0x08000166   0x00000006   Code   RO         3812    .ARM.Collect$$_printf_percent$$00000009  c_w.l(_printf_d.o)
    0x0800016c   0x0800016c   0x00000006   Code   RO         3811    .ARM.Collect$$_printf_percent$$00000014  c_w.l(_printf_s.o)
    0x08000172   0x08000172   0x00000004   Code   RO         3898    .ARM.Collect$$_printf_percent$$00000017  c_w.l(_printf_percent_end.o)
    0x08000176   0x08000176   0x00000002   Code   RO         3995    .ARM.Collect$$libinit$$00000000  c_w.l(libinit.o)
    0x08000178   0x08000178   0x00000000   Code   RO         3997    .ARM.Collect$$libinit$$00000002  c_w.l(libinit2.o)
    0x08000178   0x08000178   0x00000000   Code   RO         3999    .ARM.Collect$$libinit$$00000004  c_w.l(libinit2.o)
    0x08000178   0x08000178   0x00000000   Code   RO         4002    .ARM.Collect$$libinit$$0000000A  c_w.l(libinit2.o)
    0x08000178   0x08000178   0x00000000   Code   RO         4004    .ARM.Collect$$libinit$$0000000C  c_w.l(libinit2.o)
    0x08000178   0x08000178   0x00000000   Code   RO         4006    .ARM.Collect$$libinit$$0000000E  c_w.l(libinit2.o)
    0x08000178   0x08000178   0x00000006   Code   RO         4007    .ARM.Collect$$libinit$$0000000F  c_w.l(libinit2.o)
    0x0800017e   0x0800017e   0x00000000   Code   RO         4009    .ARM.Collect$$libinit$$00000011  c_w.l(libinit2.o)
    0x0800017e   0x0800017e   0x00000000   Code   RO         4011    .ARM.Collect$$libinit$$00000013  c_w.l(libinit2.o)
    0x0800017e   0x0800017e   0x00000000   Code   RO         4013    .ARM.Collect$$libinit$$00000015  c_w.l(libinit2.o)
    0x0800017e   0x0800017e   0x0000000a   Code   RO         4014    .ARM.Collect$$libinit$$00000016  c_w.l(libinit2.o)
    0x08000188   0x08000188   0x00000000   Code   RO         4015    .ARM.Collect$$libinit$$00000017  c_w.l(libinit2.o)
    0x08000188   0x08000188   0x00000000   Code   RO         4017    .ARM.Collect$$libinit$$00000019  c_w.l(libinit2.o)
    0x08000188   0x08000188   0x00000000   Code   RO         4019    .ARM.Collect$$libinit$$0000001B  c_w.l(libinit2.o)
    0x08000188   0x08000188   0x00000000   Code   RO         4021    .ARM.Collect$$libinit$$0000001D  c_w.l(libinit2.o)
    0x08000188   0x08000188   0x00000000   Code   RO         4023    .ARM.Collect$$libinit$$0000001F  c_w.l(libinit2.o)
    0x08000188   0x08000188   0x00000000   Code   RO         4025    .ARM.Collect$$libinit$$00000021  c_w.l(libinit2.o)
    0x08000188   0x08000188   0x00000000   Code   RO         4027    .ARM.Collect$$libinit$$00000023  c_w.l(libinit2.o)
    0x08000188   0x08000188   0x00000000   Code   RO         4029    .ARM.Collect$$libinit$$00000025  c_w.l(libinit2.o)
    0x08000188   0x08000188   0x00000000   Code   RO         4033    .ARM.Collect$$libinit$$0000002C  c_w.l(libinit2.o)
    0x08000188   0x08000188   0x00000000   Code   RO         4035    .ARM.Collect$$libinit$$0000002E  c_w.l(libinit2.o)
    0x08000188   0x08000188   0x00000000   Code   RO         4037    .ARM.Collect$$libinit$$00000030  c_w.l(libinit2.o)
    0x08000188   0x08000188   0x00000000   Code   RO         4039    .ARM.Collect$$libinit$$00000032  c_w.l(libinit2.o)
    0x08000188   0x08000188   0x00000002   Code   RO         4040    .ARM.Collect$$libinit$$00000033  c_w.l(libinit2.o)
    0x0800018a   0x0800018a   0x00000002   Code   RO         4041    .ARM.Collect$$libshutdown$$00000000  c_w.l(libshutdown.o)
    0x0800018c   0x0800018c   0x00000000   Code   RO         4054    .ARM.Collect$$libshutdown$$00000002  c_w.l(libshutdown2.o)
    0x0800018c   0x0800018c   0x00000000   Code   RO         4056    .ARM.Collect$$libshutdown$$00000004  c_w.l(libshutdown2.o)
    0x0800018c   0x0800018c   0x00000000   Code   RO         4058    .ARM.Collect$$libshutdown$$00000006  c_w.l(libshutdown2.o)
    0x0800018c   0x0800018c   0x00000000   Code   RO         4061    .ARM.Collect$$libshutdown$$00000009  c_w.l(libshutdown2.o)
    0x0800018c   0x0800018c   0x00000000   Code   RO         4064    .ARM.Collect$$libshutdown$$0000000C  c_w.l(libshutdown2.o)
    0x0800018c   0x0800018c   0x00000000   Code   RO         4066    .ARM.Collect$$libshutdown$$0000000E  c_w.l(libshutdown2.o)
    0x0800018c   0x0800018c   0x00000000   Code   RO         4069    .ARM.Collect$$libshutdown$$00000011  c_w.l(libshutdown2.o)
    0x0800018c   0x0800018c   0x00000002   Code   RO         4070    .ARM.Collect$$libshutdown$$00000012  c_w.l(libshutdown2.o)
    0x0800018e   0x0800018e   0x00000000   Code   RO         3881    .ARM.Collect$$rtentry$$00000000  c_w.l(__rtentry.o)
    0x0800018e   0x0800018e   0x00000000   Code   RO         3913    .ARM.Collect$$rtentry$$00000002  c_w.l(__rtentry2.o)
    0x0800018e   0x0800018e   0x00000006   Code   RO         3925    .ARM.Collect$$rtentry$$00000004  c_w.l(__rtentry4.o)
    0x08000194   0x08000194   0x00000000   Code   RO         3915    .ARM.Collect$$rtentry$$00000009  c_w.l(__rtentry2.o)
    0x08000194   0x08000194   0x00000004   Code   RO         3916    .ARM.Collect$$rtentry$$0000000A  c_w.l(__rtentry2.o)
    0x08000198   0x08000198   0x00000008   Code   RO         3917    .ARM.Collect$$rtentry$$0000000B  c_w.l(__rtentry2.o)
    0x080001a0   0x080001a0   0x00000008   Code   RO         3919    .ARM.Collect$$rtentry$$0000000D  c_w.l(__rtentry2.o)
    0x080001a8   0x080001a8   0x00000002   Code   RO         3882    .ARM.Collect$$rtexit$$00000000  c_w.l(rtexit.o)
    0x080001aa   0x080001aa   0x00000000   Code   RO         3928    .ARM.Collect$$rtexit$$00000002  c_w.l(rtexit2.o)
    0x080001aa   0x080001aa   0x00000004   Code   RO         3929    .ARM.Collect$$rtexit$$00000003  c_w.l(rtexit2.o)
    0x080001ae   0x080001ae   0x00000006   Code   RO         3930    .ARM.Collect$$rtexit$$00000004  c_w.l(rtexit2.o)
    0x080001b4   0x080001b4   0x0000001c   Code   RO          922    .emb_text           rtx_conf_cm.o
    0x080001d0   0x080001d0   0x00000130   Code   RO         3759    .emb_text           RTX_CM3.lib(hal_cm3.o)
    0x08000300   0x08000300   0x00000040   Code   RO         2511    .text               startup_stm32f10x_md.o
    0x08000340   0x08000340   0x00000008   Code   RO         3774    .text               c_w.l(libspace.o)
    0x08000348   0x08000348   0x00000028   Code   RO         3781    .text               c_w.l(noretval__2sprintf.o)
    0x08000370   0x08000370   0x0000004e   Code   RO         3785    .text               c_w.l(_printf_pad.o)
    0x080003be   0x080003be   0x00000052   Code   RO         3787    .text               c_w.l(_printf_str.o)
    0x08000410   0x08000410   0x00000078   Code   RO         3789    .text               c_w.l(_printf_dec.o)
    0x08000488   0x08000488   0x00000138   Code   RO         3803    .text               c_w.l(__printf_flags_wp.o)
    0x080005c0   0x080005c0   0x00000012   Code   RO         3815    .text               c_w.l(exit.o)
    0x080005d2   0x080005d2   0x00000048   Code   RO         3817    .text               c_w.l(strcpy.o)
    0x0800061a   0x0800061a   0x0000003e   Code   RO         3819    .text               c_w.l(strlen.o)
    0x08000658   0x08000658   0x00000080   Code   RO         3821    .text               c_w.l(strcmpv7m.o)
    0x080006d8   0x080006d8   0x00000006   Code   RO         3823    .text               c_w.l(heapauxi.o)
    0x080006de   0x080006de   0x000000b2   Code   RO         3888    .text               c_w.l(_printf_intcommon.o)
    0x08000790   0x08000790   0x0000041e   Code   RO         3890    .text               c_w.l(_printf_fp_dec.o)
    0x08000bae   0x08000bae   0x00000002   PAD
    0x08000bb0   0x08000bb0   0x00000030   Code   RO         3892    .text               c_w.l(_printf_char_common.o)
    0x08000be0   0x08000be0   0x0000000a   Code   RO         3894    .text               c_w.l(_sputc.o)
    0x08000bea   0x08000bea   0x0000002c   Code   RO         3896    .text               c_w.l(_printf_char.o)
    0x08000c16   0x08000c16   0x0000000a   Code   RO         3941    .text               c_w.l(rt_locale_twolibspace.o)
    0x08000c20   0x08000c20   0x0000008a   Code   RO         3943    .text               c_w.l(lludiv10.o)
    0x08000caa   0x08000caa   0x00000002   PAD
    0x08000cac   0x08000cac   0x00000080   Code   RO         3945    .text               c_w.l(_printf_fp_infnan.o)
    0x08000d2c   0x08000d2c   0x000000e4   Code   RO         3949    .text               c_w.l(bigflt0.o)
    0x08000e10   0x08000e10   0x0000000c   Code   RO         3981    .text               c_w.l(sys_exit.o)
    0x08000e1c   0x08000e1c   0x0000004a   Code   RO         3983    .text               c_w.l(sys_stackheap_outer.o)
    0x08000e66   0x08000e66   0x00000002   Code   RO         4042    .text               c_w.l(use_no_semi.o)
    0x08000e68   0x08000e68   0x00000000   Code   RO         4044    .text               c_w.l(indicate_semi.o)
    0x08000e68   0x08000e68   0x0000003e   Code   RO         3952    CL$$btod_d2e        c_w.l(btod.o)
    0x08000ea6   0x08000ea6   0x00000046   Code   RO         3954    CL$$btod_d2e_denorm_low  c_w.l(btod.o)
    0x08000eec   0x08000eec   0x00000060   Code   RO         3953    CL$$btod_d2e_norm_op1  c_w.l(btod.o)
    0x08000f4c   0x08000f4c   0x00000338   Code   RO         3962    CL$$btod_div_common  c_w.l(btod.o)
    0x08001284   0x08001284   0x000000dc   Code   RO         3959    CL$$btod_e2e        c_w.l(btod.o)
    0x08001360   0x08001360   0x0000002a   Code   RO         3956    CL$$btod_ediv       c_w.l(btod.o)
    0x0800138a   0x0800138a   0x0000002a   Code   RO         3955    CL$$btod_emul       c_w.l(btod.o)
    0x080013b4   0x080013b4   0x00000244   Code   RO         3961    CL$$btod_mult_common  c_w.l(btod.o)
    0x080015f8   0x080015f8   0x00000004   Code   RO         3769    SVC_TABLE           RTX_CM3.lib(svc_table.o)
    0x080015fc   0x080015fc   0x00000024   Code   RO          600    i.ACCMD             ws100t10.o
    0x08001620   0x08001620   0x00000044   Code   RO          601    i.ACCtrl            ws100t10.o
    0x08001664   0x08001664   0x00000010   Code   RO          602    i.AC_CTRL_Init      ws100t10.o
    0x08001674   0x08001674   0x000000e8   Code   RO          509    i.AD7190_Init       ad7190.o
    0x0800175c   0x0800175c   0x00000130   Code   RO          510    i.AD7190_ReadData   ad7190.o
    0x0800188c   0x0800188c   0x0000002e   Code   RO          511    i.AD7190_ReadRegister  ad7190.o
    0x080018ba   0x080018ba   0x0000001a   Code   RO          512    i.AD7190_ReadRegisterOnce  ad7190.o
    0x080018d4   0x080018d4   0x00000504   Code   RO          513    i.AD7190_Run        ad7190.o
    0x08001dd8   0x08001dd8   0x00000030   Code   RO          514    i.AD7190_WaitForReady  ad7190.o
    0x08001e08   0x08001e08   0x00000024   Code   RO          515    i.AD7190_WriteRegister  ad7190.o
    0x08001e2c   0x08001e2c   0x00000014   Code   RO          516    i.AD7190_WriteRegisterOnce  ad7190.o
    0x08001e40   0x08001e40   0x00000060   Code   RO          735    i.BIOS_TIM2_TIMER_Init  usarthmi.o
    0x08001ea0   0x08001ea0   0x000000a0   Code   RO          736    i.BIOS_USART1_Init  usarthmi.o
    0x08001f40   0x08001f40   0x0000006c   Code   RO          341    i.BIOS_USART2_Init  usart.o
    0x08001fac   0x08001fac   0x00000050   Code   RO          737    i.DataPrint         usarthmi.o
    0x08001ffc   0x08001ffc   0x0000000c   Code   RO          738    i.DataRec           usarthmi.o
    0x08002008   0x08002008   0x00001598   Code   RO          854    i.DataUnpack        hmi.o
    0x080035a0   0x080035a0   0x0000014c   Code   RO          855    i.FM24DataCRC       hmi.o
    0x080036ec   0x080036ec   0x00000008   Code   RO          399    i.FM24Init          fm24.o
    0x080036f4   0x080036f4   0x0000005c   Code   RO          400    i.FM24_Read         fm24.o
    0x08003750   0x08003750   0x00000048   Code   RO          401    i.FM24_Write        fm24.o
    0x08003798   0x08003798   0x0000002c   Code   RO            6    i.GPIO_InPutset     bios.o
    0x080037c4   0x080037c4   0x00000116   Code   RO         1271    i.GPIO_Init         stm32f10x_gpio.o
    0x080038da   0x080038da   0x00000002   PAD
    0x080038dc   0x080038dc   0x00000090   Code   RO         1273    i.GPIO_PinRemapConfig  stm32f10x_gpio.o
    0x0800396c   0x0800396c   0x00000012   Code   RO         1275    i.GPIO_ReadInputDataBit  stm32f10x_gpio.o
    0x0800397e   0x0800397e   0x00000004   Code   RO         1278    i.GPIO_ResetBits    stm32f10x_gpio.o
    0x08003982   0x08003982   0x00000004   Code   RO         1279    i.GPIO_SetBits      stm32f10x_gpio.o
    0x08003986   0x08003986   0x00000002   PAD
    0x08003988   0x08003988   0x00000014   Code   RO          856    i.HMICMDInit        hmi.o
    0x0800399c   0x0800399c   0x0000024c   Code   RO          603    i.HeatPID_Task      ws100t10.o
    0x08003be8   0x08003be8   0x00000010   Code   RO          604    i.HeatTask_Init     ws100t10.o
    0x08003bf8   0x08003bf8   0x00000014   Code   RO          605    i.HeatTask_Socket   ws100t10.o
    0x08003c0c   0x08003c0c   0x0000003c   Code   RO          152    i.I2C2_ACK          i2c.o
    0x08003c48   0x08003c48   0x00000040   Code   RO          153    i.I2C2_Init         i2c.o
    0x08003c88   0x08003c88   0x0000003c   Code   RO          154    i.I2C2_NACK         i2c.o
    0x08003cc4   0x08003cc4   0x00000064   Code   RO          155    i.I2C2_ReadByte     i2c.o
    0x08003d28   0x08003d28   0x00000068   Code   RO          156    i.I2C2_SendByte     i2c.o
    0x08003d90   0x08003d90   0x0000003c   Code   RO          157    i.I2C2_Start        i2c.o
    0x08003dcc   0x08003dcc   0x00000038   Code   RO          158    i.I2C2_Stop         i2c.o
    0x08003e04   0x08003e04   0x00000064   Code   RO          159    i.I2C2_Wait_ACK     i2c.o
    0x08003e68   0x08003e68   0x00000040   Code   RO            7    i.InstrumentTypeRead  bios.o
    0x08003ea8   0x08003ea8   0x00000080   Code   RO          678    i.MAX6675_ConvertTemperature  max6675.o
    0x08003f28   0x08003f28   0x00000068   Code   RO          679    i.MAX6675_Init      max6675.o
    0x08003f90   0x08003f90   0x00000058   Code   RO          680    i.MAX6675_ReadData  max6675.o
    0x08003fe8   0x08003fe8   0x00001318   Code   RO          857    i.Moisturing        hmi.o
    0x08005300   0x08005300   0x00000010   Code   RO          858    i.MoisturingRun     hmi.o
    0x08005310   0x08005310   0x00000028   Code   RO          607    i.Pump_OutCmd       ws100t10.o
    0x08005338   0x08005338   0x00000020   Code   RO         1395    i.RCC_APB2PeriphClockCmd  stm32f10x_rcc.o
    0x08005358   0x08005358   0x00000084   Code   RO          281    i.SPI1_Configuration  spi.o
    0x080053dc   0x080053dc   0x00000038   Code   RO          282    i.SPI1_ReadWrite    spi.o
    0x08005414   0x08005414   0x00000018   Code   RO         1608    i.SPI_Cmd           stm32f10x_spi.o
    0x0800542c   0x0800542c   0x00000012   Code   RO         1616    i.SPI_I2S_GetFlagStatus  stm32f10x_spi.o
    0x0800543e   0x0800543e   0x00000006   Code   RO         1619    i.SPI_I2S_ReceiveData  stm32f10x_spi.o
    0x08005444   0x08005444   0x00000004   Code   RO         1620    i.SPI_I2S_SendData  stm32f10x_spi.o
    0x08005448   0x08005448   0x0000003c   Code   RO         1621    i.SPI_Init          stm32f10x_spi.o
    0x08005484   0x08005484   0x0000001c   Code   RO            9    i.SafeCheck         bios.o
    0x080054a0   0x080054a0   0x00000008   Code   RO         2518    i.SetSysClock       system_stm32f10x.o
    0x080054a8   0x080054a8   0x000000e0   Code   RO         2519    i.SetSysClockTo72   system_stm32f10x.o
    0x08005588   0x08005588   0x00000060   Code   RO         2521    i.SystemInit        system_stm32f10x.o
    0x080055e8   0x080055e8   0x00000088   Code   RO          739    i.TIM2_IRQHandler   usarthmi.o
    0x08005670   0x08005670   0x00000018   Code   RO          740    i.UART1_Received    usarthmi.o
    0x08005688   0x08005688   0x00000020   Code   RO          741    i.UART1_Send        usarthmi.o
    0x080056a8   0x080056a8   0x00000094   Code   RO          742    i.USART1_IRQHandler  usarthmi.o
    0x0800573c   0x0800573c   0x00000034   Code   RO          345    i.USART2Print       usart.o
    0x08005770   0x08005770   0x00000018   Code   RO          346    i.USART2_Send       usart.o
    0x08005788   0x08005788   0x00000020   Code   RO          743    i.USARTHMIInit      usarthmi.o
    0x080057a8   0x080057a8   0x0000004a   Code   RO         2329    i.USART_ITConfig    stm32f10x_usart.o
    0x080057f2   0x080057f2   0x00000002   PAD
    0x080057f4   0x080057f4   0x00000098   Code   RO          168    i.WS100T10_Ctrl     i2c.o
    0x0800588c   0x0800588c   0x0000008c   Code   RO          169    i.WS100T10_Init     i2c.o
    0x08005918   0x08005918   0x00000028   Code   RO         3979    i.__ARM_fpclassify  m_ws.l(fpclassify.o)
    0x08005940   0x08005940   0x00000022   Code   RO          744    i.__NVIC_EnableIRQ  usarthmi.o
    0x08005962   0x08005962   0x00000046   Code   RO         3658    i._init_box         RTX_CM3.lib(rt_membox.o)
    0x080059a8   0x080059a8   0x0000000e   Code   RO         3801    i._is_digit         c_w.l(__printf_wp.o)
    0x080059b6   0x080059b6   0x00000002   PAD
    0x080059b8   0x080059b8   0x00000020   Code   RO          924    i._mutex_acquire    rtx_conf_cm.o
    0x080059d8   0x080059d8   0x0000001c   Code   RO          926    i._mutex_release    rtx_conf_cm.o
    0x080059f4   0x080059f4   0x0000003c   Code   RO          608    i._task_ACCtrl      ws100t10.o
    0x08005a30   0x08005a30   0x00000030   Code   RO         3711    i.dbg_init          RTX_CM3.lib(hal_cm.o)
    0x08005a60   0x08005a60   0x00000020   Code   RO         3712    i.dbg_task_notify   RTX_CM3.lib(hal_cm.o)
    0x08005a80   0x08005a80   0x00000010   Code   RO         3713    i.dbg_task_switch   RTX_CM3.lib(hal_cm.o)
    0x08005a90   0x08005a90   0x00000082   Code   RO          124    i.delay_us          delay.o
    0x08005b12   0x08005b12   0x0000002c   Code   RO         2565    i.isrMessagePut     RTX_CM3.lib(rt_cmsis.o)
    0x08005b3e   0x08005b3e   0x00000028   Code   RO         2566    i.isrSemaphoreRelease  RTX_CM3.lib(rt_cmsis.o)
    0x08005b66   0x08005b66   0x0000000e   Code   RO         3514    i.isr_mbx_send      RTX_CM3.lib(rt_mailbox.o)
    0x08005b74   0x08005b74   0x00000010   Code   RO         3561    i.isr_sem_send      RTX_CM3.lib(rt_semaphore.o)
    0x08005b84   0x08005b84   0x0000000e   Code   RO          681    i.kalman_filter_init  max6675.o
    0x08005b92   0x08005b92   0x0000000e   Code   RO          517    i.kalman_filter_init2  ad7190.o
    0x08005ba0   0x08005ba0   0x0000005a   Code   RO          682    i.kalman_filter_update  max6675.o
    0x08005bfa   0x08005bfa   0x0000005a   Code   RO          518    i.kalman_filter_update2  ad7190.o
    0x08005c54   0x08005c54   0x0000019c   Code   RO          825    i.main              moisture.o
    0x08005df0   0x08005df0   0x00000018   Code   RO         2568    i.osDelay           RTX_CM3.lib(rt_cmsis.o)
    0x08005e08   0x08005e08   0x00000024   Code   RO         2569    i.osKernelInitialize  RTX_CM3.lib(rt_cmsis.o)
    0x08005e2c   0x08005e2c   0x0000006c   Code   RO         2571    i.osKernelStart     RTX_CM3.lib(rt_cmsis.o)
    0x08005e98   0x08005e98   0x00000018   Code   RO         2572    i.osKernelSysTick   RTX_CM3.lib(rt_cmsis.o)
    0x08005eb0   0x08005eb0   0x0000002c   Code   RO         2582    i.osMutexCreate     RTX_CM3.lib(rt_cmsis.o)
    0x08005edc   0x08005edc   0x00000018   Code   RO         2584    i.osMutexRelease    RTX_CM3.lib(rt_cmsis.o)
    0x08005ef4   0x08005ef4   0x00000018   Code   RO         2585    i.osMutexWait       RTX_CM3.lib(rt_cmsis.o)
    0x08005f0c   0x08005f0c   0x0000002c   Code   RO         2590    i.osSemaphoreCreate  RTX_CM3.lib(rt_cmsis.o)
    0x08005f38   0x08005f38   0x00000018   Code   RO         2592    i.osSemaphoreRelease  RTX_CM3.lib(rt_cmsis.o)
    0x08005f50   0x08005f50   0x00000018   Code   RO         2593    i.osSemaphoreWait   RTX_CM3.lib(rt_cmsis.o)
    0x08005f68   0x08005f68   0x0000002c   Code   RO         2597    i.osThreadCreate    RTX_CM3.lib(rt_cmsis.o)
    0x08005f94   0x08005f94   0x00000018   Code   RO         2598    i.osThreadExit      RTX_CM3.lib(rt_cmsis.o)
    0x08005fac   0x08005fac   0x00000018   Code   RO         2599    i.osThreadGetId     RTX_CM3.lib(rt_cmsis.o)
    0x08005fc4   0x08005fc4   0x00000018   Code   RO         2602    i.osThreadTerminate  RTX_CM3.lib(rt_cmsis.o)
    0x08005fdc   0x08005fdc   0x00000022   Code   RO          927    i.os_error          rtx_conf_cm.o
    0x08005ffe   0x08005ffe   0x00000004   Code   RO          928    i.os_idle_demon     rtx_conf_cm.o
    0x08006002   0x08006002   0x00000002   PAD
    0x08006004   0x08006004   0x00000028   Code   RO         3305    i.os_tick_init      RTX_CM3.lib(rt_system.o)
    0x0800602c   0x0800602c   0x00000002   Code   RO         3306    i.os_tick_irqack    RTX_CM3.lib(rt_system.o)
    0x0800602e   0x0800602e   0x00000002   PAD
    0x08006030   0x08006030   0x00000010   Code   RO         3307    i.os_tick_ovf       RTX_CM3.lib(rt_system.o)
    0x08006040   0x08006040   0x00000014   Code   RO         3308    i.os_tick_val       RTX_CM3.lib(rt_system.o)
    0x08006054   0x08006054   0x0000001a   Code   RO         3659    i.rt_alloc_box      RTX_CM3.lib(rt_membox.o)
    0x0800606e   0x0800606e   0x0000003e   Code   RO         3687    i.rt_alloc_mem      RTX_CM3.lib(rt_memory.o)
    0x080060ac   0x080060ac   0x00000038   Code   RO         3186    i.rt_block          RTX_CM3.lib(rt_task.o)
    0x080060e4   0x080060e4   0x00000048   Code   RO         3636    i.rt_chk_robin      RTX_CM3.lib(rt_robin.o)
    0x0800612c   0x0800612c   0x00000070   Code   RO         3437    i.rt_dec_dly        RTX_CM3.lib(rt_list.o)
    0x0800619c   0x0800619c   0x00000044   Code   RO         3187    i.rt_dispatch       RTX_CM3.lib(rt_task.o)
    0x080061e0   0x080061e0   0x00000006   Code   RO         3603    i.rt_dly_wait       RTX_CM3.lib(rt_time.o)
    0x080061e6   0x080061e6   0x00000002   PAD
    0x080061e8   0x080061e8   0x00000050   Code   RO         3398    i.rt_evt_psh        RTX_CM3.lib(rt_event.o)
    0x08006238   0x08006238   0x0000002c   Code   RO         3660    i.rt_free_box       RTX_CM3.lib(rt_membox.o)
    0x08006264   0x08006264   0x00000028   Code   RO         3688    i.rt_free_mem       RTX_CM3.lib(rt_memory.o)
    0x0800628c   0x0800628c   0x00000028   Code   RO         3438    i.rt_get_first      RTX_CM3.lib(rt_list.o)
    0x080062b4   0x080062b4   0x00000008   Code   RO         2614    i.rt_id2obj         RTX_CM3.lib(rt_cmsis.o)
    0x080062bc   0x080062bc   0x00000048   Code   RO         3188    i.rt_init_context   RTX_CM3.lib(rt_task.o)
    0x08006304   0x08006304   0x0000001a   Code   RO         3689    i.rt_init_mem       RTX_CM3.lib(rt_memory.o)
    0x0800631e   0x0800631e   0x00000002   PAD
    0x08006320   0x08006320   0x00000018   Code   RO         3637    i.rt_init_robin     RTX_CM3.lib(rt_robin.o)
    0x08006338   0x08006338   0x00000080   Code   RO         3714    i.rt_init_stack     RTX_CM3.lib(hal_cm.o)
    0x080063b8   0x080063b8   0x00000008   Code   RO         3515    i.rt_mbx_check      RTX_CM3.lib(rt_mailbox.o)
    0x080063c0   0x080063c0   0x0000001a   Code   RO         3516    i.rt_mbx_init       RTX_CM3.lib(rt_mailbox.o)
    0x080063da   0x080063da   0x00000002   PAD
    0x080063dc   0x080063dc   0x000000f0   Code   RO         3517    i.rt_mbx_psh        RTX_CM3.lib(rt_mailbox.o)
    0x080064cc   0x080064cc   0x00000044   Code   RO         2615    i.rt_ms2tick        RTX_CM3.lib(rt_cmsis.o)
    0x08006510   0x08006510   0x00000010   Code   RO         3271    i.rt_mut_init       RTX_CM3.lib(rt_mutex.o)
    0x08006520   0x08006520   0x000000d8   Code   RO         3272    i.rt_mut_release    RTX_CM3.lib(rt_mutex.o)
    0x080065f8   0x080065f8   0x00000078   Code   RO         3273    i.rt_mut_wait       RTX_CM3.lib(rt_mutex.o)
    0x08006670   0x08006670   0x0000007c   Code   RO         3309    i.rt_pop_req        RTX_CM3.lib(rt_system.o)
    0x080066ec   0x080066ec   0x00000020   Code   RO         3310    i.rt_psh_req        RTX_CM3.lib(rt_system.o)
    0x0800670c   0x0800670c   0x0000005c   Code   RO         3440    i.rt_psq_enq        RTX_CM3.lib(rt_list.o)
    0x08006768   0x08006768   0x00000048   Code   RO         3441    i.rt_put_dly        RTX_CM3.lib(rt_list.o)
    0x080067b0   0x080067b0   0x00000036   Code   RO         3442    i.rt_put_prio       RTX_CM3.lib(rt_list.o)
    0x080067e6   0x080067e6   0x00000002   PAD
    0x080067e8   0x080067e8   0x00000014   Code   RO         3443    i.rt_put_rdy_first  RTX_CM3.lib(rt_list.o)
    0x080067fc   0x080067fc   0x00000034   Code   RO         3444    i.rt_resort_prio    RTX_CM3.lib(rt_list.o)
    0x08006830   0x08006830   0x00000006   Code   RO         3715    i.rt_ret_val        RTX_CM3.lib(hal_cm.o)
    0x08006836   0x08006836   0x00000008   Code   RO         3716    i.rt_ret_val2       RTX_CM3.lib(hal_cm.o)
    0x0800683e   0x0800683e   0x00000028   Code   RO         3445    i.rt_rmv_dly        RTX_CM3.lib(rt_list.o)
    0x08006866   0x08006866   0x00000002   PAD
    0x08006868   0x08006868   0x00000030   Code   RO         3446    i.rt_rmv_list       RTX_CM3.lib(rt_list.o)
    0x08006898   0x08006898   0x0000000c   Code   RO         3563    i.rt_sem_init       RTX_CM3.lib(rt_semaphore.o)
    0x080068a4   0x080068a4   0x00000034   Code   RO         3564    i.rt_sem_psh        RTX_CM3.lib(rt_semaphore.o)
    0x080068d8   0x080068d8   0x0000002a   Code   RO         3565    i.rt_sem_send       RTX_CM3.lib(rt_semaphore.o)
    0x08006902   0x08006902   0x00000002   PAD
    0x08006904   0x08006904   0x00000040   Code   RO         3566    i.rt_sem_wait       RTX_CM3.lib(rt_semaphore.o)
    0x08006944   0x08006944   0x00000024   Code   RO         3312    i.rt_stk_check      RTX_CM3.lib(rt_system.o)
    0x08006968   0x08006968   0x00000028   Code   RO         3189    i.rt_switch_req     RTX_CM3.lib(rt_task.o)
    0x08006990   0x08006990   0x000000cc   Code   RO         3190    i.rt_sys_init       RTX_CM3.lib(rt_task.o)
    0x08006a5c   0x08006a5c   0x00000078   Code   RO         3191    i.rt_sys_start      RTX_CM3.lib(rt_task.o)
    0x08006ad4   0x08006ad4   0x00000040   Code   RO         3314    i.rt_systick        RTX_CM3.lib(rt_system.o)
    0x08006b14   0x08006b14   0x00000012   Code   RO         2616    i.rt_tid2ptcb       RTX_CM3.lib(rt_cmsis.o)
    0x08006b26   0x08006b26   0x00000002   PAD
    0x08006b28   0x08006b28   0x00000034   Code   RO         2617    i.rt_timer_insert   RTX_CM3.lib(rt_cmsis.o)
    0x08006b5c   0x08006b5c   0x00000088   Code   RO         3192    i.rt_tsk_create     RTX_CM3.lib(rt_task.o)
    0x08006be4   0x08006be4   0x0000017c   Code   RO         3193    i.rt_tsk_delete     RTX_CM3.lib(rt_task.o)
    0x08006d60   0x08006d60   0x0000007c   Code   RO         3195    i.rt_tsk_prio       RTX_CM3.lib(rt_task.o)
    0x08006ddc   0x08006ddc   0x00000010   Code   RO         3196    i.rt_tsk_self       RTX_CM3.lib(rt_task.o)
    0x08006dec   0x08006dec   0x00000012   Code   RO         2619    i.svcDelay          RTX_CM3.lib(rt_cmsis.o)
    0x08006dfe   0x08006dfe   0x00000002   PAD
    0x08006e00   0x08006e00   0x00000070   Code   RO         2620    i.svcKernelInitialize  RTX_CM3.lib(rt_cmsis.o)
    0x08006e70   0x08006e70   0x00000048   Code   RO         2622    i.svcKernelStart    RTX_CM3.lib(rt_cmsis.o)
    0x08006eb8   0x08006eb8   0x00000038   Code   RO         2623    i.svcKernelSysTick  RTX_CM3.lib(rt_cmsis.o)
    0x08006ef0   0x08006ef0   0x00000024   Code   RO         2625    i.svcMessageCreate  RTX_CM3.lib(rt_cmsis.o)
    0x08006f14   0x08006f14   0x0000001c   Code   RO         2628    i.svcMutexCreate    RTX_CM3.lib(rt_cmsis.o)
    0x08006f30   0x08006f30   0x00000022   Code   RO         2630    i.svcMutexRelease   RTX_CM3.lib(rt_cmsis.o)
    0x08006f52   0x08006f52   0x0000003a   Code   RO         2631    i.svcMutexWait      RTX_CM3.lib(rt_cmsis.o)
    0x08006f8c   0x08006f8c   0x00000024   Code   RO         2633    i.svcSemaphoreCreate  RTX_CM3.lib(rt_cmsis.o)
    0x08006fb0   0x08006fb0   0x00000028   Code   RO         2635    i.svcSemaphoreRelease  RTX_CM3.lib(rt_cmsis.o)
    0x08006fd8   0x08006fd8   0x00000032   Code   RO         2636    i.svcSemaphoreWait  RTX_CM3.lib(rt_cmsis.o)
    0x0800700a   0x0800700a   0x00000002   PAD
    0x0800700c   0x0800700c   0x0000006c   Code   RO         2640    i.svcThreadCreate   RTX_CM3.lib(rt_cmsis.o)
    0x08007078   0x08007078   0x0000001c   Code   RO         2641    i.svcThreadGetId    RTX_CM3.lib(rt_cmsis.o)
    0x08007094   0x08007094   0x00000038   Code   RO         2644    i.svcThreadTerminate  RTX_CM3.lib(rt_cmsis.o)
    0x080070cc   0x080070cc   0x0000005c   Code   RO         2655    i.sysTimerTick      RTX_CM3.lib(rt_cmsis.o)
    0x08007128   0x08007128   0x0000002c   Code   RO         3975    locale$$code        c_w.l(lc_numeric_c.o)
    0x08007154   0x08007154   0x00000062   Code   RO         3827    x$fpl$d2f           fz_ws.l(d2f.o)
    0x080071b6   0x080071b6   0x00000018   Code   RO         3899    x$fpl$dcmpinf       fz_ws.l(dcmpi.o)
    0x080071ce   0x080071ce   0x0000002e   Code   RO         3834    x$fpl$dflt          fz_ws.l(dflt_clz.o)
    0x080071fc   0x080071fc   0x00000078   Code   RO         3839    x$fpl$dleqf         fz_ws.l(dleqf.o)
    0x08007274   0x08007274   0x00000154   Code   RO         3841    x$fpl$dmul          fz_ws.l(dmul.o)
    0x080073c8   0x080073c8   0x0000009c   Code   RO         3901    x$fpl$dnaninf       fz_ws.l(dnaninf.o)
    0x08007464   0x08007464   0x0000000c   Code   RO         3903    x$fpl$dretinf       fz_ws.l(dretinf.o)
    0x08007470   0x08007470   0x0000006c   Code   RO         3843    x$fpl$drleqf        fz_ws.l(drleqf.o)
    0x080074dc   0x080074dc   0x00000056   Code   RO         3845    x$fpl$f2d           fz_ws.l(f2d.o)
    0x08007532   0x08007532   0x00000002   PAD
    0x08007534   0x08007534   0x000000c4   Code   RO         3847    x$fpl$fadd          fz_ws.l(faddsub_clz.o)
    0x080075f8   0x080075f8   0x00000018   Code   RO         3905    x$fpl$fcmpinf       fz_ws.l(fcmpi.o)
    0x08007610   0x08007610   0x00000184   Code   RO         3854    x$fpl$fdiv          fz_ws.l(fdiv.o)
    0x08007794   0x08007794   0x00000068   Code   RO         3857    x$fpl$feqf          fz_ws.l(feqf.o)
    0x080077fc   0x080077fc   0x00000036   Code   RO         3859    x$fpl$ffix          fz_ws.l(ffix.o)
    0x08007832   0x08007832   0x00000002   PAD
    0x08007834   0x08007834   0x0000003e   Code   RO         3863    x$fpl$ffixu         fz_ws.l(ffixu.o)
    0x08007872   0x08007872   0x00000002   PAD
    0x08007874   0x08007874   0x00000030   Code   RO         3868    x$fpl$fflt          fz_ws.l(fflt_clz.o)
    0x080078a4   0x080078a4   0x00000026   Code   RO         3867    x$fpl$ffltu         fz_ws.l(fflt_clz.o)
    0x080078ca   0x080078ca   0x00000002   PAD
    0x080078cc   0x080078cc   0x00000068   Code   RO         3873    x$fpl$fleqf         fz_ws.l(fleqf.o)
    0x08007934   0x08007934   0x00000102   Code   RO         3875    x$fpl$fmul          fz_ws.l(fmul.o)
    0x08007a36   0x08007a36   0x0000008c   Code   RO         3907    x$fpl$fnaninf       fz_ws.l(fnaninf.o)
    0x08007ac2   0x08007ac2   0x0000000a   Code   RO         3909    x$fpl$fretinf       fz_ws.l(fretinf.o)
    0x08007acc   0x08007acc   0x00000062   Code   RO         3877    x$fpl$frleqf        fz_ws.l(frleqf.o)
    0x08007b2e   0x08007b2e   0x00000014   Code   RO         3848    x$fpl$frsb          fz_ws.l(faddsub_clz.o)
    0x08007b42   0x08007b42   0x00000002   PAD
    0x08007b44   0x08007b44   0x000000ea   Code   RO         3849    x$fpl$fsub          fz_ws.l(faddsub_clz.o)
    0x08007c2e   0x08007c2e   0x00000004   Code   RO         3879    x$fpl$printf1       fz_ws.l(printf1.o)
    0x08007c32   0x08007c32   0x00000000   Code   RO         3911    x$fpl$usenofp       fz_ws.l(usenofp.o)
    0x08007c32   0x08007c32   0x00000002   PAD
    0x08007c34   0x08007c34   0x00000010   Data   RO          520    .constdata          ad7190.o
    0x08007c44   0x08007c44   0x00000020   Data   RO          609    .constdata          ws100t10.o
    0x08007c64   0x08007c64   0x00000010   Data   RO          684    .constdata          max6675.o
    0x08007c74   0x08007c74   0x00000004   Data   RO          746    .constdata          usarthmi.o
    0x08007c78   0x08007c78   0x000000ea   Data   RO          862    .constdata          hmi.o
    0x08007d62   0x08007d62   0x00000002   PAD
    0x08007d64   0x08007d64   0x00000068   Data   RO          930    .constdata          rtx_conf_cm.o
    0x08007dcc   0x08007dcc   0x00000011   Data   RO         3804    .constdata          c_w.l(__printf_flags_wp.o)
    0x08007ddd   0x08007ddd   0x00000003   PAD
    0x08007de0   0x08007de0   0x00000094   Data   RO         3950    .constdata          c_w.l(bigflt0.o)
    0x08007e74   0x08007e74   0x00000020   Data   RO         4109    Region$$Table       anon$$obj.o
    0x08007e94   0x08007e94   0x0000001c   Data   RO         3974    locale$$data        c_w.l(lc_numeric_c.o)


    Execution Region RW_IRAM1 (Exec base: 0x20000000, Load base: 0x08007eb0, Size: 0x000049dc, Max: 0x00005000, ABSOLUTE)

    Exec Addr    Load Addr    Size         Type   Attr      Idx    E Section Name        Object

    0x20000000   0x08007eb0   0x00000035   Data   RW          521    .data               ad7190.o
    0x20000035   0x08007ee5   0x00000003   PAD
    0x20000038   0x08007ee8   0x00000030   Data   RW          610    .data               ws100t10.o
    0x20000068   0x08007f18   0x00000004   Data   RW          685    .data               max6675.o
    0x2000006c   0x08007f1c   0x00000018   Data   RW          747    .data               usarthmi.o
    0x20000084   0x08007f34   0x00000039   Data   RW          863    .data               hmi.o
    0x200000bd   0x08007f6d   0x00000003   PAD
    0x200000c0   0x08007f70   0x00000014   Data   RW          931    .data               rtx_conf_cm.o
    0x200000d4   0x08007f84   0x00000014   Data   RW         2522    .data               system_stm32f10x.o
    0x200000e8   0x08007f98   0x00000008   Data   RW         2658    .data               RTX_CM3.lib(rt_cmsis.o)
    0x200000f0   0x08007fa0   0x00000008   Data   RW         3198    .data               RTX_CM3.lib(rt_task.o)
    0x200000f8   0x08007fa8   0x00000008   Data   RW         3317    .data               RTX_CM3.lib(rt_system.o)
    0x20000100   0x08007fb0   0x00000004   Data   RW         3607    .data               RTX_CM3.lib(rt_time.o)
    0x20000104   0x08007fb4   0x00000008   Data   RW         3638    .data               RTX_CM3.lib(rt_robin.o)
    0x2000010c   0x08007fbc   0x00000001   Data   RW         3717    .data               RTX_CM3.lib(hal_cm.o)
    0x2000010d   0x08007fbd   0x00000003   PAD
    0x20000110        -       0x00000028   Zero   RW          519    .bss                ad7190.o
    0x20000138        -       0x00000014   Zero   RW          683    .bss                max6675.o
    0x2000014c        -       0x00000064   Zero   RW          745    .bss                usarthmi.o
    0x200001b0        -       0x00000164   Zero   RW          861    .bss                hmi.o
    0x20000314        -       0x00000034   Zero   RW         3197    .bss                RTX_CM3.lib(rt_task.o)
    0x20000348        -       0x00000030   Zero   RW         3447    .bss                RTX_CM3.lib(rt_list.o)
    0x20000378        -       0x00000060   Zero   RW         3775    .bss                c_w.l(libspace.o)
    0x200003d8        -       0x00000200   Zero   RW         2509    HEAP                startup_stm32f10x_md.o
    0x200005d8        -       0x00000400   Zero   RW         2508    STACK               startup_stm32f10x_md.o
    0x200009d8   0x08007fbd   0x00000628   PAD
    0x20001000        -       0x00000096   Zero   RW          859    .ARM.__AT_0x20001000  hmi.o
    0x20001096   0x08007fbd   0x0000016a   PAD
    0x20001200        -       0x00000096   Zero   RW          860    .ARM.__AT_0x20001200  hmi.o
    0x20001296   0x08007fbd   0x00000002   PAD
    0x20001298        -       0x00003744   Zero   RW          929    .bss                rtx_conf_cm.o


==============================================================================

Image component sizes


      Code (inc. data)   RO Data    RW Data    ZI Data      Debug   Object Name

      2100        250         16         53         40      10829   ad7190.o
       136         14          0          0          0     235239   bios.o
       130          0          0          0          0        471   delay.o
       172          0          0          0          0       1988   fm24.o
     10784       2742        234         57        656      14024   hmi.o
       896         70          0          0          0       4820   i2c.o
       424         32         16          4         20       3769   max6675.o
       412         60          0          0          0        631   moisture.o
       126         26        104         20      14148       9123   rtx_conf_cm.o
       188         16          0          0          0       1050   spi.o
        64         26        236          0       1536        796   startup_stm32f10x_md.o
       448          6          0          0          0       5106   stm32f10x_gpio.o
        32          6          0          0          0        641   stm32f10x_rcc.o
       112          0          0          0          0       4446   stm32f10x_spi.o
        74          0          0          0          0       2593   stm32f10x_usart.o
       328         28          0         20          0       2301   system_stm32f10x.o
       184         26          0          0          0       1911   usart.o
       754        106          4         24        100       9796   usarthmi.o
       844        112         32         48          0       5228   ws100t10.o

    ----------------------------------------------------------------------
     18216       3520        676        232      18440     314762   Object Totals
         0          0         32          0          0          0   (incl. Generated)
         8          0          2          6       1940          0   (incl. Padding)

    ----------------------------------------------------------------------

      Code (inc. data)   RO Data    RW Data    ZI Data      Debug   Library Member Name

       238         24          0          1          0       3244   hal_cm.o
       304         36          0          0          0        756   hal_cm3.o
      1546        194          0          8          0      40639   rt_cmsis.o
        80          4          0          0          0        649   rt_event.o
       530         34          0          0         48       8157   rt_list.o
       288          4          0          0          0       2385   rt_mailbox.o
       140          0          0          0          0       1889   rt_membox.o
       128          0          0          0          0       2267   rt_memory.o
       352         14          0          0          0       2073   rt_mutex.o
        96         22          0          8          0       1134   rt_robin.o
       186         10          0          0          0       2862   rt_semaphore.o
       334         64          0          8          0       6991   rt_system.o
      1216        174          0          8         52       9537   rt_task.o
         6          0          0          4          0        636   rt_time.o
         4          4          0          0          0        196   svc_table.o
         8          0          0          0          0         68   __main.o
       312          4         17          0          0         92   __printf_flags_wp.o
        14          0          0          0          0         68   __printf_wp.o
         0          0          0          0          0          0   __rtentry.o
        20          0          0          0          0          0   __rtentry2.o
         6          0          0          0          0          0   __rtentry4.o
        52          8          0          0          0          0   __scatter.o
        26          0          0          0          0          0   __scatter_copy.o
        28          0          0          0          0          0   __scatter_zi.o
        44          0          0          0          0        108   _printf_char.o
        48          6          0          0          0         96   _printf_char_common.o
         6          0          0          0          0          0   _printf_d.o
       120         16          0          0          0         92   _printf_dec.o
         6          0          0          0          0          0   _printf_f.o
      1054          0          0          0          0        216   _printf_fp_dec.o
       128         16          0          0          0         84   _printf_fp_infnan.o
       178          0          0          0          0         88   _printf_intcommon.o
        78          0          0          0          0        108   _printf_pad.o
         0          0          0          0          0          0   _printf_percent.o
         4          0          0          0          0          0   _printf_percent_end.o
         6          0          0          0          0          0   _printf_s.o
        82          0          0          0          0         80   _printf_str.o
        10          0          0          0          0         68   _sputc.o
       228          4        148          0          0         96   bigflt0.o
      1936        128          0          0          0        672   btod.o
        18          0          0          0          0         80   exit.o
         6          0          0          0          0        152   heapauxi.o
         0          0          0          0          0          0   indicate_semi.o
        44         10         28          0          0         76   lc_numeric_c.o
         2          0          0          0          0          0   libinit.o
        18          0          0          0          0          0   libinit2.o
         2          0          0          0          0          0   libshutdown.o
         2          0          0          0          0          0   libshutdown2.o
         8          4          0          0         96         68   libspace.o
       138          0          0          0          0         80   lludiv10.o
        40          6          0          0          0         84   noretval__2sprintf.o
        10          0          0          0          0         76   rt_locale_twolibspace.o
         2          0          0          0          0          0   rtexit.o
        10          0          0          0          0          0   rtexit2.o
       128          0          0          0          0         68   strcmpv7m.o
        72          0          0          0          0         80   strcpy.o
        62          0          0          0          0         76   strlen.o
        12          4          0          0          0         68   sys_exit.o
        74          0          0          0          0         80   sys_stackheap_outer.o
         2          0          0          0          0         68   use_no_semi.o
        98          4          0          0          0         92   d2f.o
        24          0          0          0          0         68   dcmpi.o
        46          0          0          0          0         68   dflt_clz.o
       120          4          0          0          0         92   dleqf.o
       340         12          0          0          0        104   dmul.o
       156          4          0          0          0         92   dnaninf.o
        12          0          0          0          0         68   dretinf.o
       108          0          0          0          0         80   drleqf.o
        86          4          0          0          0         84   f2d.o
       450          8          0          0          0        236   faddsub_clz.o
        24          0          0          0          0         68   fcmpi.o
       388         76          0          0          0         96   fdiv.o
       104          4          0          0          0         84   feqf.o
        54          4          0          0          0         84   ffix.o
        62          4          0          0          0         84   ffixu.o
        86          0          0          0          0        136   fflt_clz.o
       104          4          0          0          0         84   fleqf.o
       258          4          0          0          0         84   fmul.o
       140          4          0          0          0         84   fnaninf.o
        10          0          0          0          0         68   fretinf.o
        98          0          0          0          0         68   frleqf.o
         4          0          0          0          0         68   printf1.o
         0          0          0          0          0          0   usenofp.o
        40          0          0          0          0         68   fpclassify.o

    ----------------------------------------------------------------------
     13344        926        196         40        196      88467   Library Totals
        40          0          3          3          0          0   (incl. Padding)

    ----------------------------------------------------------------------

      Code (inc. data)   RO Data    RW Data    ZI Data      Debug   Library Name

      5448        584          0         37        100      83415   RTX_CM3.lib
      5044        206        193          0         96       2992   c_w.l
      2772        136          0          0          0       1992   fz_ws.l
        40          0          0          0          0         68   m_ws.l

    ----------------------------------------------------------------------
     13344        926        196         40        196      88467   Library Totals

    ----------------------------------------------------------------------

==============================================================================


      Code (inc. data)   RO Data    RW Data    ZI Data      Debug   

     31560       4446        872        272      18636     391785   Grand Totals
     31560       4446        872        272      18636     391785   ELF Image Totals
     31560       4446        872        272          0          0   ROM Totals

==============================================================================

    Total RO  Size (Code + RO Data)                32432 (  31.67kB)
    Total RW  Size (RW Data + ZI Data)             18908 (  18.46kB)
    Total ROM Size (Code + RO Data + RW Data)      32704 (  31.94kB)

==============================================================================

